 cgamex86

 Timestamp is 38ac8946 (Thu Feb 17 16:50:30 2000)

 Preferred load address is 30000000

 Start         Length     Name                   Class
 0001:00000000 0003c2faH .text                   CODE
 0002:00000000 000060a9H .rdata                  DATA
 0002:000060b0 00000059H .edata                  DATA
 0003:00000000 00000004H .CRT$XCA                DATA
 0003:00000004 00000004H .CRT$XCZ                DATA
 0003:00000008 00000004H .CRT$XIA                DATA
 0003:0000000c 00000008H .CRT$XIC                DATA
 0003:00000014 00000004H .CRT$XIZ                DATA
 0003:00000018 00000004H .CRT$XPA                DATA
 0003:0000001c 00000004H .CRT$XPX                DATA
 0003:00000020 00000004H .CRT$XPZ                DATA
 0003:00000024 00000004H .CRT$XTA                DATA
 0003:00000028 00000004H .CRT$XTZ                DATA
 0003:00000030 0000391cH .data                   DATA
 0003:00003950 0013fe58H .bss                    DATA
 0004:00000000 00000014H .idata$2                DATA
 0004:00000014 00000014H .idata$3                DATA
 0004:00000028 0000012cH .idata$4                DATA
 0004:00000154 0000012cH .idata$5                DATA
 0004:00000280 00000542H .idata$6                DATA

  Address         Publics by Value              Rva+Base     Lib:Object

 0001:00000000       _qsort                     30001000 f   bg_lib.obj
 0001:000006c0       _strlen                    300016c0 f   bg_lib.obj
 0001:00000700       _strcat                    30001700 f   bg_lib.obj
 0001:00000760       _strcpy                    30001760 f   bg_lib.obj
 0001:000007b0       _strcmp                    300017b0 f   bg_lib.obj
 0001:00000810       _strchr                    30001810 f   bg_lib.obj
 0001:00000850       _strstr                    30001850 f   bg_lib.obj
 0001:000008d0       _memmove                   300018d0 f   bg_lib.obj
 0001:00000950       _tan                       30001950 f   bg_lib.obj
 0001:00000990       _srand                     30001990 f   bg_lib.obj
 0001:000009b0       _rand                      300019b0 f   bg_lib.obj
 0001:000009e0       _atof                      300019e0 f   bg_lib.obj
 0001:00000b30       __atof                     30001b30 f   bg_lib.obj
 0001:00000c80       _BG_FindItemForPowerup     30001c80 f   bg_misc.obj
 0001:00000cf0       _BG_FindItemForHoldable    30001cf0 f   bg_misc.obj
 0001:00000d60       _BG_FindItemForWeapon      30001d60 f   bg_misc.obj
 0001:00000dc0       _BG_FindAmmoForWeapon      30001dc0 f   bg_misc.obj
 0001:00000e20       _BG_FindItem               30001e20 f   bg_misc.obj
 0001:00000e70       _BG_PlayerTouchesItem      30001e70 f   bg_misc.obj
 0001:00000f30       _BG_CanItemBeGrabbed       30001f30 f   bg_misc.obj
 0001:00001280       _BG_EvaluateTrajectory     30002280 f   bg_misc.obj
 0001:000014e0       _BG_EvaluateTrajectoryDelta 300024e0 f   bg_misc.obj
 0001:000016a0       _BG_AddPredictableEventToPlayerstate 300026a0 f   bg_misc.obj
 0001:000016f0       _BG_PlayerStateToEntityState 300026f0 f   bg_misc.obj
 0001:000019b0       _PM_AddEvent               300029b0 f   bg_pmove.obj
 0001:000019e0       _PM_AddTouchEnt            300029e0 f   bg_pmove.obj
 0001:00001a70       _PM_ClipVelocity           30002a70 f   bg_pmove.obj
 0001:00001b10       _PM_UpdateViewAngles       30002b10 f   bg_pmove.obj
 0001:00001c00       _PmoveSingle               30002c00 f   bg_pmove.obj
 0001:00005770       _Pmove                     30006770 f   bg_pmove.obj
 0001:00005800       _PM_SlideMove              30006800 f   bg_slidemove.obj
 0001:00006040       _PM_StepSlideMove          30007040 f   bg_slidemove.obj
 0001:00006460       _CG_TargetCommand_f        30007460 f   cg_consolecmds.obj
 0001:00006710       _CG_ConsoleCommand         30007710 f   cg_consolecmds.obj
 0001:00006780       _CG_InitConsoleCommands    30007780 f   cg_consolecmds.obj
 0001:00006880       _CG_DrawHead               30007880 f   cg_draw.obj
 0001:00006bf0       _CG_DrawFlagModel          30007bf0 f   cg_draw.obj
 0001:00006d30       _CG_DrawTeamBackground     30007d30 f   cg_draw.obj
 0001:00006dd0       _CG_AddLagometerFrameInfo  30007dd0 f   cg_draw.obj
 0001:00006e10       _CG_AddLagometerSnapshotInfo 30007e10 f   cg_draw.obj
 0001:00006e90       _CG_CenterPrint            30007e90 f   cg_draw.obj
 0001:00006f20       _CG_DrawActive             30007f20 f   cg_draw.obj
 0001:0000a4c0       _CG_AdjustFrom640          3000b4c0 f   cg_drawtools.obj
 0001:0000a510       _CG_FillRect               3000b510 f   cg_drawtools.obj
 0001:0000a580       _CG_DrawPic                3000b580 f   cg_drawtools.obj
 0001:0000a5e0       _CG_DrawChar               3000b5e0 f   cg_drawtools.obj
 0001:0000a6b0       _CG_DrawStringExt          3000b6b0 f   cg_drawtools.obj
 0001:0000a8a0       _CG_DrawBigString          3000b8a0 f   cg_drawtools.obj
 0001:0000a8f0       _CG_DrawBigStringColor     3000b8f0 f   cg_drawtools.obj
 0001:0000a930       _CG_DrawSmallString        3000b930 f   cg_drawtools.obj
 0001:0000a980       _CG_DrawSmallStringColor   3000b980 f   cg_drawtools.obj
 0001:0000a9c0       _CG_DrawStrlen             3000b9c0 f   cg_drawtools.obj
 0001:0000aa40       _CG_TileClear              3000ba40 f   cg_drawtools.obj
 0001:0000abe0       _CG_FadeColor              3000bbe0 f   cg_drawtools.obj
 0001:0000ac70       _CG_TeamColor              3000bc70 f   cg_drawtools.obj
 0001:0000acc0       _CG_GetColorForHealth      3000bcc0 f   cg_drawtools.obj
 0001:0000add0       _CG_ColorForHealth         3000bdd0 f   cg_drawtools.obj
 0001:0000ae10       _UI_DrawBannerString       3000be10 f   cg_drawtools.obj
 0001:0000b0a0       _UI_ProportionalStringWidth 3000c0a0 f   cg_drawtools.obj
 0001:0000b120       _UI_ProportionalSizeScale  3000c120 f   cg_drawtools.obj
 0001:0000b150       _UI_DrawProportionalString 3000c150 f   cg_drawtools.obj
 0001:0000b510       _CG_BubbleTrail            3000c510 f   cg_effects.obj
 0001:0000b7c0       _CG_SmokePuff              3000c7c0 f   cg_effects.obj
 0001:0000b9c0       _CG_SpawnEffect            3000c9c0 f   cg_effects.obj
 0001:0000bae0       _CG_MakeExplosion          3000cae0 f   cg_effects.obj
 0001:0000bd00       _CG_Bleed                  3000cd00 f   cg_effects.obj
 0001:0000bdf0       _CG_RBleed                 3000cdf0 f   cg_effects.obj
 0001:0000bef0       _CG_Bleed2                 3000cef0 f   cg_effects.obj
 0001:0000c010       _CG_LaunchGib              3000d010 f   cg_effects.obj
 0001:0000c150       _CG_GibPlayer              3000d150 f   cg_effects.obj
 0001:0000c7b0       _CG_LaunchGibNoBlood       3000d7b0 f   cg_effects.obj
 0001:0000c8f0       _CG_GibNoBlood             3000d8f0 f   cg_effects.obj
 0001:0000cf50       _CG_PositionEntityOnTag    3000df50 f   cg_ents.obj
 0001:0000d060       _CG_PositionRotatedEntityOnTag 3000e060 f   cg_ents.obj
 0001:0000d180       _CG_SetEntitySoundPosition 3000e180 f   cg_ents.obj
 0001:0000d220       _CG_Beam                   3000e220 f   cg_ents.obj
 0001:0000d2d0       _CG_AdjustPositionForMover 3000e2d0 f   cg_ents.obj
 0001:0000d420       _CG_AddPacketEntities      3000e420 f   cg_ents.obj
 0001:0000ead0       _CG_PlaceString            3000fad0 f   cg_event.obj
 0001:0000ec20       _CG_PainEvent              3000fc20 f   cg_event.obj
 0001:0000ecd0       _CG_EntityEvent            3000fcd0 f   cg_event.obj
 0001:00010b90       _CG_CheckEvents            30011b90 f   cg_event.obj
 0001:00010c60       _CG_LoadingString          30011c60 f   cg_info.obj
 0001:00010c90       _CG_LoadingItem            30011c90 f   cg_info.obj
 0001:00010d00       _CG_LoadingClient          30011d00 f   cg_info.obj
 0001:00010e30       _CG_DrawInformation        30011e30 f   cg_info.obj
 0001:000113a0       _CG_InitLocalEntities      300123a0 f   cg_localents.obj
 0001:00011420       _CG_FreeLocalEntity        30012420 f   cg_localents.obj
 0001:00011480       _CG_AllocLocalEntity       30012480 f   cg_localents.obj
 0001:00011500       _CG_BloodTrail             30012500 f   cg_localents.obj
 0001:000115d0       _CG_FragmentBounceMark     300125d0 f   cg_localents.obj
 0001:00011670       _CG_FragmentBounceSound    30012670 f   cg_localents.obj
 0001:00011700       _CG_ReflectVelocity        30012700 f   cg_localents.obj
 0001:00011880       _CG_AddFragment            30012880 f   cg_localents.obj
 0001:00011ac0       _CG_AddExpandingFade       30012ac0 f   cg_localents.obj
 0001:00011c00       _CG_AddFadeRGB             30012c00 f   cg_localents.obj
 0001:00011ca0       _CG_AddLocalEntities       30012ca0 f   cg_localents.obj
 0001:00012520       _vmMain                    30013520 f   cg_main.obj
 0001:000125c0       _CG_RegisterCvars          300135c0 f   cg_main.obj
 0001:00012660       _CG_UpdateCvars            30013660 f   cg_main.obj
 0001:00012700       _CG_CrosshairPlayer        30013700 f   cg_main.obj
 0001:00012730       _CG_LastAttacker           30013730 f   cg_main.obj
 0001:00012760       _CG_Printf                 30013760 f   cg_main.obj
 0001:000127b0       _CG_Error                  300137b0 f   cg_main.obj
 0001:00012800       _Com_Error                 30013800 f   cg_main.obj
 0001:00012850       _Com_Printf                30013850 f   cg_main.obj
 0001:000128a0       _CG_Argv                   300138a0 f   cg_main.obj
 0001:000128d0       _CG_ConfigString           300138d0 f   cg_main.obj
 0001:00012910       _CG_StartMusic             30013910 f   cg_main.obj
 0001:00012980       _CG_Init                   30013980 f   cg_main.obj
 0001:00013b90       _CG_Shutdown               30014b90 f   cg_main.obj
 0001:00013ba0       _CG_InitMarkPolys          30014ba0 f   cg_marks.obj
 0001:00013c20       _CG_FreeMarkPoly           30014c20 f   cg_marks.obj
 0001:00013c80       _CG_AllocMark              30014c80 f   cg_marks.obj
 0001:00013d30       _CG_ImpactMark             30014d30 f   cg_marks.obj
 0001:00014190       _CG_AddMarks               30015190 f   cg_marks.obj
 0001:000143d0       _CG_CustomSound            300153d0 f   cg_players.obj
 0001:00014490       _CG_NewClientInfo          30015490 f   cg_players.obj
 0001:00015740       _CG_LoadDeferredPlayers    30016740 f   cg_players.obj
 0001:000157d0       _CG_AddRefEntityWithPowerups 300167d0 f   cg_players.obj
 0001:000158b0       _CG_Player                 300168b0 f   cg_players.obj
 0001:00017970       _CG_Player3rd              30018970 f   cg_players.obj
 0001:00018900       _CG_ResetPlayerEntity      30019900 f   cg_players.obj
 0001:00018b70       _CG_CheckAmmo              30019b70 f   cg_playerstate.obj
 0001:00018d20       _CG_DamageFeedback         30019d20 f   cg_playerstate.obj
 0001:00018ff0       _CG_Respawn                30019ff0 f   cg_playerstate.obj
 0001:00019030       _CG_CheckPlayerstateEvents 3001a030 f   cg_playerstate.obj
 0001:00019150       _CG_CheckLocalSounds       3001a150 f   cg_playerstate.obj
 0001:000195e0       _CG_TransitionPlayerState  3001a5e0 f   cg_playerstate.obj
 0001:00019700       _CG_BuildSolidList         3001a700 f   cg_predict.obj
 0001:00019810       _CG_Trace                  3001a810 f   cg_predict.obj
 0001:00019ac0       _CG_PointContents          3001aac0 f   cg_predict.obj
 0001:00019b80       _CG_PredictPlayerState     3001ab80 f   cg_predict.obj
 0001:0001a550       _CG_DrawScoreboard         3001b550 f   cg_scoreboard.obj
 0001:0001b230       _CG_DrawTourneyScoreboard  3001c230 f   cg_scoreboard.obj
 0001:0001b5a0       _CG_ParseServerinfo        3001c5a0 f   cg_servercmds.obj
 0001:0001b6d0       _CG_SetConfigValues        3001c6d0 f   cg_servercmds.obj
 0001:0001b770       _CG_ExecuteNewServerCommands 3001c770 f   cg_servercmds.obj
 0001:0001c270       _CG_SetInitialSnapshot     3001d270 f   cg_snapshot.obj
 0001:0001c400       _CG_ProcessSnapshots       3001d400 f   cg_snapshot.obj
 0001:0001c9e0       _dllEntry                  3001d9e0 f   cg_syscalls.obj
 0001:0001ca00       _PASSFLOAT                 3001da00 f   cg_syscalls.obj
 0001:0001ca20       _trap_Print                3001da20 f   cg_syscalls.obj
 0001:0001ca40       _trap_Error                3001da40 f   cg_syscalls.obj
 0001:0001ca60       _trap_Milliseconds         3001da60 f   cg_syscalls.obj
 0001:0001ca80       _trap_Cvar_Register        3001da80 f   cg_syscalls.obj
 0001:0001cab0       _trap_Cvar_Update          3001dab0 f   cg_syscalls.obj
 0001:0001cad0       _trap_Cvar_Set             3001dad0 f   cg_syscalls.obj
 0001:0001cb00       _trap_Cvar_VariableStringBuffer 3001db00 f   cg_syscalls.obj
 0001:0001cb30       _trap_Argc                 3001db30 f   cg_syscalls.obj
 0001:0001cb50       _trap_Argv                 3001db50 f   cg_syscalls.obj
 0001:0001cb80       _trap_Args                 3001db80 f   cg_syscalls.obj
 0001:0001cbb0       _trap_FS_FOpenFile         3001dbb0 f   cg_syscalls.obj
 0001:0001cbe0       _trap_FS_Read              3001dbe0 f   cg_syscalls.obj
 0001:0001cc10       _trap_FS_Write             3001dc10 f   cg_syscalls.obj
 0001:0001cc40       _trap_FS_FCloseFile        3001dc40 f   cg_syscalls.obj
 0001:0001cc60       _trap_SendConsoleCommand   3001dc60 f   cg_syscalls.obj
 0001:0001cc80       _trap_AddCommand           3001dc80 f   cg_syscalls.obj
 0001:0001cca0       _trap_SendClientCommand    3001dca0 f   cg_syscalls.obj
 0001:0001ccc0       _trap_UpdateScreen         3001dcc0 f   cg_syscalls.obj
 0001:0001cce0       _trap_CM_LoadMap           3001dce0 f   cg_syscalls.obj
 0001:0001cd00       _trap_CM_NumInlineModels   3001dd00 f   cg_syscalls.obj
 0001:0001cd20       _trap_CM_InlineModel       3001dd20 f   cg_syscalls.obj
 0001:0001cd40       _trap_CM_TempBoxModel      3001dd40 f   cg_syscalls.obj
 0001:0001cd70       _trap_CM_PointContents     3001dd70 f   cg_syscalls.obj
 0001:0001cda0       _trap_CM_TransformedPointContents 3001dda0 f   cg_syscalls.obj
 0001:0001cdd0       _trap_CM_BoxTrace          3001ddd0 f   cg_syscalls.obj
 0001:0001ce10       _trap_CM_TransformedBoxTrace 3001de10 f   cg_syscalls.obj
 0001:0001ce50       _trap_CM_MarkFragments     3001de50 f   cg_syscalls.obj
 0001:0001ce90       _trap_S_StartSound         3001de90 f   cg_syscalls.obj
 0001:0001cec0       _trap_S_StartLocalSound    3001dec0 f   cg_syscalls.obj
 0001:0001cef0       _trap_S_ClearLoopingSounds 3001def0 f   cg_syscalls.obj
 0001:0001cf10       _trap_S_AddLoopingSound    3001df10 f   cg_syscalls.obj
 0001:0001cf40       _trap_S_UpdateEntityPosition 3001df40 f   cg_syscalls.obj
 0001:0001cf70       _trap_S_Respatialize       3001df70 f   cg_syscalls.obj
 0001:0001cfa0       _trap_S_RegisterSound      3001dfa0 f   cg_syscalls.obj
 0001:0001cfc0       _trap_S_StartBackgroundTrack 3001dfc0 f   cg_syscalls.obj
 0001:0001cff0       _trap_R_LoadWorldMap       3001dff0 f   cg_syscalls.obj
 0001:0001d010       _trap_R_RegisterModel      3001e010 f   cg_syscalls.obj
 0001:0001d030       _trap_R_RegisterSkin       3001e030 f   cg_syscalls.obj
 0001:0001d050       _trap_R_RegisterShader     3001e050 f   cg_syscalls.obj
 0001:0001d070       _trap_R_RegisterShaderNoMip 3001e070 f   cg_syscalls.obj
 0001:0001d090       _trap_R_ClearScene         3001e090 f   cg_syscalls.obj
 0001:0001d0b0       _trap_R_AddRefEntityToScene 3001e0b0 f   cg_syscalls.obj
 0001:0001d0d0       _trap_R_AddPolyToScene     3001e0d0 f   cg_syscalls.obj
 0001:0001d100       _trap_R_AddLightToScene    3001e100 f   cg_syscalls.obj
 0001:0001d160       _trap_R_RenderScene        3001e160 f   cg_syscalls.obj
 0001:0001d180       _trap_R_SetColor           3001e180 f   cg_syscalls.obj
 0001:0001d1a0       _trap_R_DrawStretchPic     3001e1a0 f   cg_syscalls.obj
 0001:0001d230       _trap_R_ModelBounds        3001e230 f   cg_syscalls.obj
 0001:0001d260       _trap_R_LerpTag            3001e260 f   cg_syscalls.obj
 0001:0001d2a0       _trap_GetGlconfig          3001e2a0 f   cg_syscalls.obj
 0001:0001d2c0       _trap_GetGameState         3001e2c0 f   cg_syscalls.obj
 0001:0001d2e0       _trap_GetCurrentSnapshotNumber 3001e2e0 f   cg_syscalls.obj
 0001:0001d310       _trap_GetSnapshot          3001e310 f   cg_syscalls.obj
 0001:0001d340       _trap_GetServerCommand     3001e340 f   cg_syscalls.obj
 0001:0001d360       _trap_GetCurrentCmdNumber  3001e360 f   cg_syscalls.obj
 0001:0001d380       _trap_GetUserCmd           3001e380 f   cg_syscalls.obj
 0001:0001d3b0       _trap_SetUserCmdValue      3001e3b0 f   cg_syscalls.obj
 0001:0001d3e0       _testPrintInt              3001e3e0 f   cg_syscalls.obj
 0001:0001d410       _testPrintFloat            3001e410 f   cg_syscalls.obj
 0001:0001d440       _trap_MemoryRemaining      3001e440 f   cg_syscalls.obj
 0001:0001d460       _CG_TestModel_f            3001e460 f   cg_view.obj
 0001:0001d5a0       _CG_TestGun_f              3001e5a0 f   cg_view.obj
 0001:0001d5d0       _CG_TestModelNextFrame_f   3001e5d0 f   cg_view.obj
 0001:0001d610       _CG_TestModelPrevFrame_f   3001e610 f   cg_view.obj
 0001:0001d660       _CG_TestModelNextSkin_f    3001e660 f   cg_view.obj
 0001:0001d6a0       _CG_TestModelPrevSkin_f    3001e6a0 f   cg_view.obj
 0001:0001d6f0       _CG_ZoomDown_f             3001e6f0 f   cg_view.obj
 0001:0001d720       _CG_ZoomUp_f               3001e720 f   cg_view.obj
 0001:0001d750       _CG_DrawActiveFrame        3001e750 f   cg_view.obj
 0001:0001ea40       _CG_RailTrail              3001fa40 f   cg_weapons.obj
 0001:0001ef30       _CG_GrappleTrail           3001ff30 f   cg_weapons.obj
 0001:0001f0b0       _CG_RegisterWeapon         300200b0 f   cg_weapons.obj
 0001:000201d0       _CG_RegisterItemVisuals    300211d0 f   cg_weapons.obj
 0001:000202b0       _CG_AddPlayerWeapon        300212b0 f   cg_weapons.obj
 0001:00020f40       _CG_AddViewWeapon          30021f40 f   cg_weapons.obj
 0001:000214e0       _CG_DrawWeaponSelect       300224e0 f   cg_weapons.obj
 0001:00021770       _CG_NextWeapon_f           30022770 f   cg_weapons.obj
 0001:00021880       _CG_PrevWeapon_f           30022880 f   cg_weapons.obj
 0001:00021930       _CG_Weapon_f               30022930 f   cg_weapons.obj
 0001:000219c0       _CG_OutOfAmmoChange        300229c0 f   cg_weapons.obj
 0001:00021a30       _CG_FireWeapon             30022a30 f   cg_weapons.obj
 0001:00021b70       _CG_MissileHitWall         30022b70 f   cg_weapons.obj
 0001:00022150       _CG_MissileHitPlayer       30023150 f   cg_weapons.obj
 0001:000221a0       _CG_MissileHitRPlayer      300231a0 f   cg_weapons.obj
 0001:000221f0       _CG_ShotgunFire            300231f0 f   cg_weapons.obj
 0001:000225d0       _CG_Tracer                 300235d0 f   cg_weapons.obj
 0001:000229a0       _CG_Bullet                 300239a0 f   cg_weapons.obj
 0001:00022b00       _Q_rand                    30023b00 f   q_math.obj
 0001:00022b30       _Q_random                  30023b30 f   q_math.obj
 0001:00022b60       _Q_crandom                 30023b60 f   q_math.obj
 0001:00022b90       _ClampChar                 30023b90 f   q_math.obj
 0001:00022bc0       _ClampShort                30023bc0 f   q_math.obj
 0001:00022c00       _DirToByte                 30023c00 f   q_math.obj
 0001:00022ca0       _ByteToDir                 30023ca0 f   q_math.obj
 0001:00022d20       _ColorBytes3               30023d20 f   q_math.obj
 0001:00022d70       _ColorBytes4               30023d70 f   q_math.obj
 0001:00022dd0       _NormalizeColor            30023dd0 f   q_math.obj
 0001:00022e80       _PlaneFromPoints           30023e80 f   q_math.obj
 0001:00022f50       _RotatePointAroundVector   30023f50 f   q_math.obj
 0001:00023180       _RotateAroundDirection     30024180 f   q_math.obj
 0001:00023210       _vectoangles               30024210 f   q_math.obj
 0001:00023380       _AxisMult                  30024380 f   q_math.obj
 0001:00023450       _AnglesToAxis              30024450 f   q_math.obj
 0001:000234b0       _AxisClear                 300244b0 f   q_math.obj
 0001:00023520       _AxisCopy                  30024520 f   q_math.obj
 0001:000235a0       _ProjectPointOnPlane       300245a0 f   q_math.obj
 0001:00023670       _MakeNormalVectors         30024670 f   q_math.obj
 0001:00023730       _VectorRotate              30024730 f   q_math.obj
 0001:000237d0       _Q_rsqrt                   300247d0 f   q_math.obj
 0001:00023830       _Q_fabs                    30024830 f   q_math.obj
 0001:00023860       _LerpAngle                 30024860 f   q_math.obj
 0001:000238c0       _AngleSubtract             300248c0 f   q_math.obj
 0001:00023920       _AnglesSubtract            30024920 f   q_math.obj
 0001:00023990       _AngleMod                  30024990 f   q_math.obj
 0001:000239d0       _AngleNormalize360         300249d0 f   q_math.obj
 0001:00023a10       _AngleNormalize180         30024a10 f   q_math.obj
 0001:00023a50       _AngleDelta                30024a50 f   q_math.obj
 0001:00023a80       _SetPlaneSignbits          30024a80 f   q_math.obj
 0001:00023af0       _BoxOnPlaneSide            30024af0 f   q_math.obj
 0001:00023d30       _RadiusFromBounds          30024d30 f   q_math.obj
 0001:00023dc0       _ClearBounds               30024dc0 f   q_math.obj
 0001:00023e10       _AddPointToBounds          30024e10 f   q_math.obj
 0001:00023ee0       _VectorCompare             30024ee0 f   q_math.obj
 0001:00023f30       _VectorNormalize           30024f30 f   q_math.obj
 0001:00023fd0       _VectorNormalizeFast       30024fd0 f   q_math.obj
 0001:00024040       _VectorNormalize2          30025040 f   q_math.obj
 0001:000240f0       __VectorMA                 300250f0 f   q_math.obj
 0001:00024140       __DotProduct               30025140 f   q_math.obj
 0001:00024180       __VectorSubtract           30025180 f   q_math.obj
 0001:000241d0       __VectorAdd                300251d0 f   q_math.obj
 0001:00024220       __VectorCopy               30025220 f   q_math.obj
 0001:00024260       __VectorScale              30025260 f   q_math.obj
 0001:000242a0       _CrossProduct              300252a0 f   q_math.obj
 0001:00024310       _VectorLength              30025310 f   q_math.obj
 0001:00024360       _Distance                  30025360 f   q_math.obj
 0001:000243b0       _DistanceSquared           300253b0 f   q_math.obj
 0001:00024410       _VectorInverse             30025410 f   q_math.obj
 0001:00024450       _Vector4Scale              30025450 f   q_math.obj
 0001:000244a0       _Q_log2                    300254a0 f   q_math.obj
 0001:000244e0       _PlaneTypeForNormal        300254e0 f   q_math.obj
 0001:00024540       _MatrixMultiply            30025540 f   q_math.obj
 0001:000246f0       _AngleVectors              300256f0 f   q_math.obj
 0001:000248e0       _PerpendicularVector       300258e0 f   q_math.obj
 0001:000249a0       _Com_Clamp                 300259a0 f   q_shared.obj
 0001:000249e0       _COM_SkipPath              300259e0 f   q_shared.obj
 0001:00024a30       _COM_StripExtension        30025a30 f   q_shared.obj
 0001:00024a80       _COM_DefaultExtension      30025a80 f   q_shared.obj
 0001:00024b10       _BigShort                  30025b10 f   q_shared.obj
 0001:00024b30       _LittleShort               30025b30 f   q_shared.obj
 0001:00024b50       _BigLong                   30025b50 f   q_shared.obj
 0001:00024b70       _LittleLong                30025b70 f   q_shared.obj
 0001:00024b90       _BigFloat                  30025b90 f   q_shared.obj
 0001:00024bb0       _LittleFloat               30025bb0 f   q_shared.obj
 0001:00024bd0       _ShortSwap                 30025bd0 f   q_shared.obj
 0001:00024c20       _ShortNoSwap               30025c20 f   q_shared.obj
 0001:00024c40       _LongSwap                  30025c40 f   q_shared.obj
 0001:00024cc0       _LongNoSwap                30025cc0 f   q_shared.obj
 0001:00024ce0       _FloatSwap                 30025ce0 f   q_shared.obj
 0001:00024d20       _FloatNoSwap               30025d20 f   q_shared.obj
 0001:00024d40       _Swap_Init                 30025d40 f   q_shared.obj
 0001:00024de0       _COM_BeginParseSession     30025de0 f   q_shared.obj
 0001:00024e00       _COM_GetCurrentParseLine   30025e00 f   q_shared.obj
 0001:00024e20       _COM_Parse                 30025e20 f   q_shared.obj
 0001:00024e40       _COM_ParseExt              30025e40 f   q_shared.obj
 0001:000250c0       _COM_MatchToken            300260c0 f   q_shared.obj
 0001:00025110       _SkipBracedSection         30026110 f   q_shared.obj
 0001:00025180       _SkipRestOfLine            30026180 f   q_shared.obj
 0001:000251d0       _Parse1DMatrix             300261d0 f   q_shared.obj
 0001:00025250       _Parse2DMatrix             30026250 f   q_shared.obj
 0001:000252c0       _Parse3DMatrix             300262c0 f   q_shared.obj
 0001:00025340       _Q_isprint                 30026340 f   q_shared.obj
 0001:00025370       _Q_islower                 30026370 f   q_shared.obj
 0001:000253a0       _Q_isupper                 300263a0 f   q_shared.obj
 0001:000253d0       _Q_isalpha                 300263d0 f   q_shared.obj
 0001:00025410       _Q_strrchr                 30026410 f   q_shared.obj
 0001:00025470       _Q_strncpyz                30026470 f   q_shared.obj
 0001:000254d0       _Q_stricmpn                300264d0 f   q_shared.obj
 0001:00025580       _Q_strncmp                 30026580 f   q_shared.obj
 0001:000255f0       _Q_stricmp                 300265f0 f   q_shared.obj
 0001:00025620       _Q_strlwr                  30026620 f   q_shared.obj
 0001:00025670       _Q_strupr                  30026670 f   q_shared.obj
 0001:000256c0       _Q_strcat                  300266c0 f   q_shared.obj
 0001:00025710       _Q_PrintStrlen             30026710 f   q_shared.obj
 0001:00025790       _Q_CleanStr                30026790 f   q_shared.obj
 0001:00025820       _Com_sprintf               30026820 f   q_shared.obj
 0001:000258b0       _va                        300268b0 f   q_shared.obj
 0001:00025910       _Info_ValueForKey          30026910 f   q_shared.obj
 0001:00025a90       _Info_NextPair             30026a90 f   q_shared.obj
 0001:00025b70       _Info_RemoveKey            30026b70 f   q_shared.obj
 0001:00025ce0       _Info_Validate             30026ce0 f   q_shared.obj
 0001:00025d30       _Info_SetValueForKey       30026d30 f   q_shared.obj
 0001:00025ea0       __CIcos                    30026ea0 f   LIBCMTD:cos.obj
 0001:00025eb4       _cos                       30026eb4 f   LIBCMTD:cos.obj
 0001:00025f50       __CIsin                    30026f50 f   LIBCMTD:sin.obj
 0001:00025f64       _sin                       30026f64 f   LIBCMTD:sin.obj
 0001:00026000       __fpmath                   30027000 f   LIBCMTD:fpinit.obj
 0001:00026030       __fpclear                  30027030 f   LIBCMTD:fpinit.obj
 0001:00026040       __cfltcvt_init             30027040 f   LIBCMTD:fpinit.obj
 0001:00026090       ___setfflag                30027090 f   LIBCMTD:fpinit.obj
 0001:000260ac       __ftol                     300270ac f   LIBCMTD:ftol.obj
 0001:000260e0       _memset                    300270e0 f   LIBCMTD:memset.obj
 0001:00026140       _abs                       30027140 f   LIBCMTD:abs.obj
 0001:00026170       __CIsqrt                   30027170 f   LIBCMTD:sqrt.obj
 0001:00026184       _sqrt                      30027184 f   LIBCMTD:sqrt.obj
 0001:00026230       _atol                      30027230 f   LIBCMTD:atox.obj
 0001:00026330       _atoi                      30027330 f   LIBCMTD:atox.obj
 0001:00026350       __atoi64                   30027350 f   LIBCMTD:atox.obj
 0001:00026480       _memcpy                    30027480 f   LIBCMTD:memcpy.obj
 0001:000267c0       _fabs                      300277c0 f   LIBCMTD:fabs.obj
 0001:000268c0       _vsprintf                  300278c0 f   LIBCMTD:vsprintf.obj
 0001:000269c0       __alloca_probe             300279c0 f   LIBCMTD:chkstk.obj
 0001:000269c0       __chkstk                   300279c0 f   LIBCMTD:chkstk.obj
 0001:000269f0       _atan2                     300279f0 f   LIBCMTD:87ctriga.obj
 0001:000269fa       __CIatan2                  300279fa f   LIBCMTD:87ctriga.obj
 0001:00026a10       _strncpy                   30027a10 f   LIBCMTD:strncpy.obj
 0001:00026b10       __tolower                  30027b10 f   LIBCMTD:tolower.obj
 0001:00026b20       _tolower                   30027b20 f   LIBCMTD:tolower.obj
 0001:00026bc0       __tolower_lk               30027bc0 f   LIBCMTD:tolower.obj
 0001:00026cf0       __toupper                  30027cf0 f   LIBCMTD:toupper.obj
 0001:00026d00       _toupper                   30027d00 f   LIBCMTD:toupper.obj
 0001:00026da0       __toupper_lk               30027da0 f   LIBCMTD:toupper.obj
 0001:00026ed0       __CRT_INIT@12              30027ed0 f   LIBCMTD:dllcrt0.obj
 0001:00027010       __DllMainCRTStartup@12     30028010 f   LIBCMTD:dllcrt0.obj
 0001:00027110       __amsg_exit                30028110 f   LIBCMTD:dllcrt0.obj
 0001:00027150       __trandisp1                30028150 f   LIBCMTD:87disp.obj
 0001:000271b7       __trandisp2                300281b7 f   LIBCMTD:87disp.obj
 0001:00027243       __rttospopde               30028243 f   LIBCMTD:87disp.obj
 0001:00027248       __rttospop                 30028248 f   LIBCMTD:87disp.obj
 0001:0002724a       __rtnospop                 3002824a f   LIBCMTD:87disp.obj
 0001:0002724c       __rttosnpop                3002824c f   LIBCMTD:87disp.obj
 0001:0002724d       __rtnospopde               3002824d f   LIBCMTD:87disp.obj
 0001:00027254       __rtzeropop                30028254 f   LIBCMTD:87disp.obj
 0001:00027256       __rtzeronpop               30028256 f   LIBCMTD:87disp.obj
 0001:0002725b       __rtonepop                 3002825b f   LIBCMTD:87disp.obj
 0001:0002725d       __rtonenpop                3002825d f   LIBCMTD:87disp.obj
 0001:00027262       __tosnan1                  30028262 f   LIBCMTD:87disp.obj
 0001:0002728d       __nosnan2                  3002828d f   LIBCMTD:87disp.obj
 0001:0002728f       __tosnan2                  3002828f f   LIBCMTD:87disp.obj
 0001:000272b7       __nan2                     300282b7 f   LIBCMTD:87disp.obj
 0001:000272f6       __rtindfpop                300282f6 f   LIBCMTD:87disp.obj
 0001:000272f8       __rtindfnpop               300282f8 f   LIBCMTD:87disp.obj
 0001:00027309       __rttosnpopde              30028309 f   LIBCMTD:87disp.obj
 0001:00027313       __rtchsifneg               30028313 f   LIBCMTD:87disp.obj
 0001:00027320       __twoToTOS                 30028320 f   LIBCMTD:common.obj
 0001:00027335       __load_CW                  30028335 f   LIBCMTD:common.obj
 0001:0002734c       __convertTOStoQNaN         3002834c f   LIBCMTD:common.obj
 0001:00027365       __fload_withFB             30028365 f   LIBCMTD:common.obj
 0001:000273a8       __checkTOS_withFB          300283a8 f   LIBCMTD:common.obj
 0001:000273be       __fast_exit                300283be f   LIBCMTD:common.obj
 0001:000273cb       __math_exit                300283cb f   LIBCMTD:common.obj
 0001:000273f5       __check_overflow_exit      300283f5 f   LIBCMTD:common.obj
 0001:00027409       __check_range_exit         30028409 f   LIBCMTD:common.obj
 0001:000274b0       __startTwoArgErrorHandling 300284b0 f   LIBCMTD:genexcep.obj
 0001:000274c7       __startOneArgErrorHandling 300284c7 f   LIBCMTD:genexcep.obj
 0001:00027510       __setdefaultprecision      30028510 f   LIBCMTD:fp8.obj
 0001:00027530       __ms_p5_test_fdiv          30028530 f   LIBCMTD:testfdiv.obj
 0001:00027590       __ms_p5_mp_test_fdiv       30028590 f   LIBCMTD:testfdiv.obj
 0001:000275e0       __forcdecpt                300285e0 f   LIBCMTD:cvt.obj
 0001:00027690       __cropzeros                30028690 f   LIBCMTD:cvt.obj
 0001:00027770       __positive                 30028770 f   LIBCMTD:cvt.obj
 0001:000277a0       __fassign                  300287a0 f   LIBCMTD:cvt.obj
 0001:000277f0       __cftoe                    300287f0 f   LIBCMTD:cvt.obj
 0001:000279e0       __cftof                    300289e0 f   LIBCMTD:cvt.obj
 0001:00027b90       __cftog                    30028b90 f   LIBCMTD:cvt.obj
 0001:00027c80       __cfltcvt                  30028c80 f   LIBCMTD:cvt.obj
 0001:00027d10       __isctype                  30028d10 f   LIBCMTD:isctype.obj
 0001:00027dd0       __allmul                   30028dd0 f   LIBCMTD:llmul.obj
 0001:00027e10       __handle_qnan1             30028e10 f   LIBCMTD:fpexcept.obj
 0001:00027e70       __handle_qnan2             30028e70 f   LIBCMTD:fpexcept.obj
 0001:00027ee0       __except1                  30028ee0 f   LIBCMTD:fpexcept.obj
 0001:00027fa0       __except2                  30028fa0 f   LIBCMTD:fpexcept.obj
 0001:00028070       __raise_exc                30029070 f   LIBCMTD:fpexcept.obj
 0001:00028540       __handle_exc               30029540 f   LIBCMTD:fpexcept.obj
 0001:000288c0       __umatherr                 300298c0 f   LIBCMTD:fpexcept.obj
 0001:00028960       __set_errno                30029960 f   LIBCMTD:fpexcept.obj
 0001:000289e0       __errcode                  300299e0 f   LIBCMTD:fpexcept.obj
 0001:00028a60       __set_exp                  30029a60 f   LIBCMTD:util.obj
 0001:00028aa0       __get_exp                  30029aa0 f   LIBCMTD:util.obj
 0001:00028ad0       __add_exp                  30029ad0 f   LIBCMTD:util.obj
 0001:00028b10       __set_bexp                 30029b10 f   LIBCMTD:util.obj
 0001:00028b50       __sptype                   30029b50 f   LIBCMTD:util.obj
 0001:00028bd0       __decomp                   30029bd0 f   LIBCMTD:util.obj
 0001:00028d10       __statfp                   30029d10 f   LIBCMTD:fpctrl.obj
 0001:00028d30       __clrfp                    30029d30 f   LIBCMTD:fpctrl.obj
 0001:00028d50       __ctrlfp                   30029d50 f   LIBCMTD:fpctrl.obj
 0001:00028d90       __set_statfp               30029d90 f   LIBCMTD:fpctrl.obj
 0001:00028e10       __flsbuf                   30029e10 f   LIBCMTD:_flsbuf.obj
 0001:00029090       __output                   3002a090 f   LIBCMTD:output.obj
 0001:00029f30       __CrtDbgBreak              3002af30 f   LIBCMTD:dbgrpt.obj
 0001:00029f40       __CrtSetReportMode         3002af40 f   LIBCMTD:dbgrpt.obj
 0001:00029fa0       __CrtSetReportFile         3002afa0 f   LIBCMTD:dbgrpt.obj
 0001:0002a020       __CrtSetReportHook         3002b020 f   LIBCMTD:dbgrpt.obj
 0001:0002a040       __CrtDbgReport             3002b040 f   LIBCMTD:dbgrpt.obj
 0001:0002a6fc       __fFATN2                   3002b6fc f   LIBCMTD:87triga.obj
 0001:0002a74c       __rtpiby2                  3002b74c f   LIBCMTD:87triga.obj
 0001:0002a790       __cintrindisp2             3002b790 f   LIBCMTD:87cdisp.obj
 0001:0002a7ce       __cintrindisp1             3002b7ce f   LIBCMTD:87cdisp.obj
 0001:0002a80b       __ctrandisp2               3002b80b f   LIBCMTD:87cdisp.obj
 0001:0002a98b       __ctrandisp1               3002b98b f   LIBCMTD:87cdisp.obj
 0001:0002a9be       __fload                    3002b9be f   LIBCMTD:87cdisp.obj
 0001:0002aa00       __mtinitlocks              3002ba00 f   LIBCMTD:mlock.obj
 0001:0002aa40       __mtdeletelocks            3002ba40 f   LIBCMTD:mlock.obj
 0001:0002aae0       __lock                     3002bae0 f   LIBCMTD:mlock.obj
 0001:0002ab80       __unlock                   3002bb80 f   LIBCMTD:mlock.obj
 0001:0002aba0       __lockerr_exit             3002bba0 f   LIBCMTD:mlock.obj
 0001:0002abc0       _setlocale                 3002bbc0 f   LIBCMTD:setlocal.obj
 0001:0002b250       __expandlocale             3002c250 f   LIBCMTD:setlocal.obj
 0001:0002b3e0       ___init_dummy              3002c3e0 f   LIBCMTD:setlocal.obj
 0001:0002b3f0       __strcats                  3002c3f0 f   LIBCMTD:setlocal.obj
 0001:0002b440       ___lc_strtolc              3002c440 f   LIBCMTD:setlocal.obj
 0001:0002b5a0       ___lc_lctostr              3002c5a0 f   LIBCMTD:setlocal.obj
 0001:0002b610       ___crtLCMapStringA         3002c610 f   LIBCMTD:a_map.obj
 0001:0002b970       __cinit                    3002c970 f   LIBCMTD:crt0dat.obj
 0001:0002b9b0       _exit                      3002c9b0 f   LIBCMTD:crt0dat.obj
 0001:0002b9d0       __exit                     3002c9d0 f   LIBCMTD:crt0dat.obj
 0001:0002b9f0       __cexit                    3002c9f0 f   LIBCMTD:crt0dat.obj
 0001:0002ba10       __c_exit                   3002ca10 f   LIBCMTD:crt0dat.obj
 0001:0002bb20       __lockexit                 3002cb20 f   LIBCMTD:crt0dat.obj
 0001:0002bb30       __unlockexit               3002cb30 f   LIBCMTD:crt0dat.obj
 0001:0002bb70       __mtinit                   3002cb70 f   LIBCMTD:tidtable.obj
 0001:0002bc00       __mtterm                   3002cc00 f   LIBCMTD:tidtable.obj
 0001:0002bc30       __initptd                  3002cc30 f   LIBCMTD:tidtable.obj
 0001:0002bc50       __getptd                   3002cc50 f   LIBCMTD:tidtable.obj
 0001:0002bcf0       __freeptd                  3002ccf0 f   LIBCMTD:tidtable.obj
 0001:0002be00       ___threadid                3002ce00 f   LIBCMTD:tidtable.obj
 0001:0002be10       ___threadhandle            3002ce10 f   LIBCMTD:tidtable.obj
 0001:0002be20       __ioinit                   3002ce20 f   LIBCMTD:ioinit.obj
 0001:0002c150       __ioterm                   3002d150 f   LIBCMTD:ioinit.obj
 0001:0002c1f0       _malloc                    3002d1f0 f   LIBCMTD:dbgheap.obj
 0001:0002c210       __malloc_dbg               3002d210 f   LIBCMTD:dbgheap.obj
 0001:0002c240       __nh_malloc                3002d240 f   LIBCMTD:dbgheap.obj
 0001:0002c260       __nh_malloc_dbg            3002d260 f   LIBCMTD:dbgheap.obj
 0001:0002c2c0       __heap_alloc               3002d2c0 f   LIBCMTD:dbgheap.obj
 0001:0002c2e0       __heap_alloc_dbg           3002d2e0 f   LIBCMTD:dbgheap.obj
 0001:0002c600       _calloc                    3002d600 f   LIBCMTD:dbgheap.obj
 0001:0002c620       __calloc_dbg               3002d620 f   LIBCMTD:dbgheap.obj
 0001:0002c680       _realloc                   3002d680 f   LIBCMTD:dbgheap.obj
 0001:0002c6a0       __realloc_dbg              3002d6a0 f   LIBCMTD:dbgheap.obj
 0001:0002cc00       __expand                   3002dc00 f   LIBCMTD:dbgheap.obj
 0001:0002cc20       __expand_dbg               3002dc20 f   LIBCMTD:dbgheap.obj
 0001:0002cc60       _free                      3002dc60 f   LIBCMTD:dbgheap.obj
 0001:0002cc80       __free_lk                  3002dc80 f   LIBCMTD:dbgheap.obj
 0001:0002cca0       __free_dbg                 3002dca0 f   LIBCMTD:dbgheap.obj
 0001:0002ccd0       __free_dbg_lk              3002dcd0 f   LIBCMTD:dbgheap.obj
 0001:0002d0c0       __msize                    3002e0c0 f   LIBCMTD:dbgheap.obj
 0001:0002d0e0       __msize_dbg                3002e0e0 f   LIBCMTD:dbgheap.obj
 0001:0002d240       __CrtSetBreakAlloc         3002e240 f   LIBCMTD:dbgheap.obj
 0001:0002d260       __CrtSetDbgBlockType       3002e260 f   LIBCMTD:dbgheap.obj
 0001:0002d300       __CrtSetAllocHook          3002e300 f   LIBCMTD:dbgheap.obj
 0001:0002d3b0       __CrtCheckMemory           3002e3b0 f   LIBCMTD:dbgheap.obj
 0001:0002d720       __CrtSetDbgFlag            3002e720 f   LIBCMTD:dbgheap.obj
 0001:0002d750       __CrtDoForAllClientObjects 3002e750 f   LIBCMTD:dbgheap.obj
 0001:0002d7c0       __CrtIsValidPointer        3002e7c0 f   LIBCMTD:dbgheap.obj
 0001:0002d810       __CrtIsValidHeapPointer    3002e810 f   LIBCMTD:dbgheap.obj
 0001:0002d8a0       __CrtIsMemoryBlock         3002e8a0 f   LIBCMTD:dbgheap.obj
 0001:0002d990       __CrtSetDumpClient         3002e990 f   LIBCMTD:dbgheap.obj
 0001:0002d9b0       __CrtMemCheckpoint         3002e9b0 f   LIBCMTD:dbgheap.obj
 0001:0002db20       __CrtMemDifference         3002eb20 f   LIBCMTD:dbgheap.obj
 0001:0002dc50       __CrtMemDumpAllObjectsSince 3002ec50 f   LIBCMTD:dbgheap.obj
 0001:0002e030       __CrtDumpMemoryLeaks       3002f030 f   LIBCMTD:dbgheap.obj
 0001:0002e0b0       __CrtMemDumpStatistics     3002f0b0 f   LIBCMTD:dbgheap.obj
 0001:0002e180       __setenvp                  3002f180 f   LIBCMTD:stdenvp.obj
 0001:0002e2d0       __setargv                  3002f2d0 f   LIBCMTD:stdargv.obj
 0001:0002e7e0       ___crtGetEnvironmentStringsA 3002f7e0 f   LIBCMTD:a_env.obj
 0001:0002ea00       __heap_init                3002fa00 f   LIBCMTD:heapinit.obj
 0001:0002ea50       __heap_term                3002fa50 f   LIBCMTD:heapinit.obj
 0001:0002eaf0       _DllMain@12                3002faf0 f   LIBCMTD:dllmain.obj
 0001:0002eb00       __FF_MSGBANNER             3002fb00 f   LIBCMTD:crt0msg.obj
 0001:0002eb50       __NMSG_WRITE               3002fb50 f   LIBCMTD:crt0msg.obj
 0001:0002ed10       __GET_RTERRMSG             3002fd10 f   LIBCMTD:crt0msg.obj
 0001:0002ed60       __87except                 3002fd60 f   LIBCMTD:87except.obj
 0001:0002eee0       __statusfp                 3002fee0 f   LIBCMTD:ieee87.obj
 0001:0002ef00       __clearfp                  3002ff00 f   LIBCMTD:ieee87.obj
 0001:0002ef20       __control87                3002ff20 f   LIBCMTD:ieee87.obj
 0001:0002ef70       __controlfp                3002ff70 f   LIBCMTD:ieee87.obj
 0001:0002ef90       __fpreset                  3002ff90 f   LIBCMTD:ieee87.obj
 0001:0002f380       __ZeroTail                 30030380 f   LIBCMTD:intrncvt.obj
 0001:0002f410       __IncMan                   30030410 f   LIBCMTD:intrncvt.obj
 0001:0002f4c0       __RoundMan                 300304c0 f   LIBCMTD:intrncvt.obj
 0001:0002f5a0       __CopyMan                  300305a0 f   LIBCMTD:intrncvt.obj
 0001:0002f5f0       __FillZeroMan              300305f0 f   LIBCMTD:intrncvt.obj
 0001:0002f620       __IsZeroMan                30030620 f   LIBCMTD:intrncvt.obj
 0001:0002f660       __ShrMan                   30030660 f   LIBCMTD:intrncvt.obj
 0001:0002f750       __ld12cvt                  30030750 f   LIBCMTD:intrncvt.obj
 0001:0002f9a0       __ld12tod                  300309a0 f   LIBCMTD:intrncvt.obj
 0001:0002f9c0       __ld12tof                  300309c0 f   LIBCMTD:intrncvt.obj
 0001:0002f9e0       __ld12told                 300309e0 f   LIBCMTD:intrncvt.obj
 0001:0002faa0       __atodbl                   30030aa0 f   LIBCMTD:intrncvt.obj
 0001:0002fae0       __atoldbl                  30030ae0 f   LIBCMTD:intrncvt.obj
 0001:0002fb20       __atoflt                   30030b20 f   LIBCMTD:intrncvt.obj
 0001:0002fb60       __fptostr                  30030b60 f   LIBCMTD:_fptostr.obj
 0001:0002fc60       __fltout2                  30030c60 f   LIBCMTD:cfout.obj
 0001:0002fce0       ___dtold                   30030ce0 f   LIBCMTD:cfout.obj
 0001:0002fe50       __fptrap                   30030e50 f   LIBCMTD:crt0fp.obj
 0001:0002fe60       ___crtGetStringTypeA       30030e60 f   LIBCMTD:a_str.obj
 0001:00030020       __dosmaperr                30031020 f   LIBCMTD:dosmap.obj
 0001:000300c0       __errno                    300310c0 f   LIBCMTD:dosmap.obj
 0001:000300d0       ___doserrno                300310d0 f   LIBCMTD:dosmap.obj
 0001:000300e0       __matherr                  300310e0 f   LIBCMTD:matherr.obj
 0001:000300f0       __lseek                    300310f0 f   LIBCMTD:lseek.obj
 0001:00030180       __lseek_lk                 30031180 f   LIBCMTD:lseek.obj
 0001:00030240       __write                    30031240 f   LIBCMTD:write.obj
 0001:000302d0       __write_lk                 300312d0 f   LIBCMTD:write.obj
 0001:00030550       __getbuf                   30031550 f   LIBCMTD:_getbuf.obj
 0001:00030620       __isatty                   30031620 f   LIBCMTD:isatty.obj
 0001:00030660       ___initstdio               30031660 f   LIBCMTD:_file.obj
 0001:00030790       ___endstdio                30031790 f   LIBCMTD:_file.obj
 0001:000307b0       __lock_file                300317b0 f   LIBCMTD:_file.obj
 0001:000307f0       __lock_file2               300317f0 f   LIBCMTD:_file.obj
 0001:00030820       __unlock_file              30031820 f   LIBCMTD:_file.obj
 0001:00030860       __unlock_file2             30031860 f   LIBCMTD:_file.obj
 0001:00030890       _wctomb                    30031890 f   LIBCMTD:wctomb.obj
 0001:00030910       __wctomb_lk                30031910 f   LIBCMTD:wctomb.obj
 0001:000309b0       __aulldiv                  300319b0 f   LIBCMTD:ulldiv.obj
 0001:00030a20       __aullrem                  30031a20 f   LIBCMTD:ullrem.obj
 0001:00030aa0       __itoa                     30031aa0 f   LIBCMTD:xtoa.obj
 0001:00030bc0       __ltoa                     30031bc0 f   LIBCMTD:xtoa.obj
 0001:00030c00       __ultoa                    30031c00 f   LIBCMTD:xtoa.obj
 0001:00030c20       __i64toa                   30031c20 f   LIBCMTD:xtoa.obj
 0001:00030d70       __ui64toa                  30031d70 f   LIBCMTD:xtoa.obj
 0001:00030d90       __snprintf                 30031d90 f   LIBCMTD:snprintf.obj
 0001:00030e90       __vsnprintf                30031e90 f   LIBCMTD:vsnprint.obj
 0001:00030f90       _signal                    30031f90 f   LIBCMTD:winsig.obj
 0001:00031260       _raise                     30032260 f   LIBCMTD:winsig.obj
 0001:00031500       ___fpecode                 30032500 f   LIBCMTD:winsig.obj
 0001:00031510       ___pxcptinfoptrs           30032510 f   LIBCMTD:winsig.obj
 0001:00031520       ___crtMessageBoxA          30032520 f   LIBCMTD:crtmbox.obj
 0001:000315e0       ___init_time               300325e0 f   LIBCMTD:inittime.obj
 0001:00031f60       ___init_numeric            30032f60 f   LIBCMTD:initnum.obj
 0001:00032290       ___init_monetary           30033290 f   LIBCMTD:initmon.obj
 0001:000326f0       ___init_ctype              300336f0 f   LIBCMTD:initctyp.obj
 0001:00032a90       ___init_collate            30033a90 f   LIBCMTD:initcoll.obj
 0001:00032aa0       _strcspn                   30033aa0 f   LIBCMTD:strcspn.obj
 0001:00032ae0       _strncmp                   30033ae0 f   LIBCMTD:strncmp.obj
 0001:00032b20       _strpbrk                   30033b20 f   LIBCMTD:strpbrk.obj
 0001:00032b60       ___get_qualified_locale    30033b60 f   LIBCMTD:getqloc.obj
 0001:000338f8       __global_unwind2           300348f8 f   LIBCMTD:exsup.obj
 0001:0003393a       __local_unwind2            3003493a f   LIBCMTD:exsup.obj
 0001:00033992       __NLG_Return2              30034992 f   LIBCMTD:exsup.obj
 0001:000339a2       __abnormal_termination     300349a2 f   LIBCMTD:exsup.obj
 0001:000339c5       __NLG_Notify1              300349c5 f   LIBCMTD:exsup.obj
 0001:000339ce       __NLG_Notify               300349ce f   LIBCMTD:exsup.obj
 0001:000339e1       __NLG_Dispatch             300349e1 f   LIBCMTD:exsup.obj
 0001:000339f0       __except_handler3          300349f0 f   LIBCMTD:exsup3.obj
 0001:00033aad       __seh_longjmp_unwind@4     30034aad f   LIBCMTD:exsup3.obj
 0001:00033ad0       __XcptFilter               30034ad0 f   LIBCMTD:winxfltr.obj
 0001:00033cf0       ?_set_new_handler@@YAP6AHI@ZP6AHI@Z@Z 30034cf0 f   LIBCMTD:handler.obj
 0001:00033d20       ?_query_new_handler@@YAP6AHI@ZXZ 30034d20 f   LIBCMTD:handler.obj
 0001:00033d30       __callnewh                 30034d30 f   LIBCMTD:handler.obj
 0001:00033d60       __malloc_base              30034d60 f   LIBCMTD:malloc.obj
 0001:00033d80       __nh_malloc_base           30034d80 f   LIBCMTD:malloc.obj
 0001:00033de0       __heap_alloc_base          30034de0 f   LIBCMTD:malloc.obj
 0001:00033e50       __CrtDefaultAllocHook      30034e50 f   LIBCMTD:dbghook.obj
 0001:00033e60       __expand_base              30034e60 f   LIBCMTD:expand.obj
 0001:00033f10       __realloc_base             30034f10 f   LIBCMTD:realloc.obj
 0001:00034100       __free_base                30035100 f   LIBCMTD:free.obj
 0001:00034170       __heapchk                  30035170 f   LIBCMTD:heapchk.obj
 0001:000341f0       __heapset                  300351f0 f   LIBCMTD:heapchk.obj
 0001:00034200       __get_sbh_threshold        30035200 f   LIBCMTD:sbheap.obj
 0001:00034210       __set_sbh_threshold        30035210 f   LIBCMTD:sbheap.obj
 0001:00034230       ___sbh_heap_init           30035230 f   LIBCMTD:sbheap.obj
 0001:00034290       ___sbh_find_block          30035290 f   LIBCMTD:sbheap.obj
 0001:000342f0       ___sbh_verify_block        300352f0 f   LIBCMTD:sbheap.obj
 0001:00034350       ___sbh_free_block          30035350 f   LIBCMTD:sbheap.obj
 0001:00034920       ___sbh_alloc_block         30035920 f   LIBCMTD:sbheap.obj
 0001:00034e60       ___sbh_alloc_new_region    30035e60 f   LIBCMTD:sbheap.obj
 0001:00034f70       ___sbh_alloc_new_group     30035f70 f   LIBCMTD:sbheap.obj
 0001:00035160       ___sbh_resize_block        30036160 f   LIBCMTD:sbheap.obj
 0001:00035750       ___sbh_heapmin             30036750 f   LIBCMTD:sbheap.obj
 0001:00035880       ___sbh_heap_check          30036880 f   LIBCMTD:sbheap.obj
 0001:00035ea0       _sprintf                   30036ea0 f   LIBCMTD:sprintf.obj
 0001:00035fa0       __setmbcp                  30036fa0 f   LIBCMTD:mbctype.obj
 0001:00036760       __getmbcp                  30037760 f   LIBCMTD:mbctype.obj
 0001:00036780       ___initmbctable            30037780 f   LIBCMTD:mbctype.obj
 0001:000367b0       ___addl                    300377b0 f   LIBCMTD:mantold.obj
 0001:000367f0       ___add_12                  300377f0 f   LIBCMTD:mantold.obj
 0001:000368a0       ___shl_12                  300378a0 f   LIBCMTD:mantold.obj
 0001:00036900       ___shr_12                  30037900 f   LIBCMTD:mantold.obj
 0001:00036970       ___mtold12                 30037970 f   LIBCMTD:mantold.obj
 0001:00036ab0       ___strgtold12              30037ab0 f   LIBCMTD:strgtold.obj
 0001:000375e0       ___STRINGTOLD              300385e0 f   LIBCMTD:strgtold.obj
 0001:00037630       _$I10_OUTPUT               30038630 f   LIBCMTD:x10fout.obj
 0001:00037b50       __alloc_osfhnd             30038b50 f   LIBCMTD:osfinfo.obj
 0001:00037d40       __set_osfhnd               30038d40 f   LIBCMTD:osfinfo.obj
 0001:00037e00       __free_osfhnd              30038e00 f   LIBCMTD:osfinfo.obj
 0001:00037ee0       __get_osfhandle            30038ee0 f   LIBCMTD:osfinfo.obj
 0001:00037f50       __open_osfhandle           30038f50 f   LIBCMTD:osfinfo.obj
 0001:00038060       __lock_fhandle             30039060 f   LIBCMTD:osfinfo.obj
 0001:000380f0       __unlock_fhandle           300390f0 f   LIBCMTD:osfinfo.obj
 0001:00038120       __fcloseall                30039120 f   LIBCMTD:closeall.obj
 0001:00038200       _fflush                    30039200 f   LIBCMTD:fflush.obj
 0001:00038250       __fflush_lk                30039250 f   LIBCMTD:fflush.obj
 0001:000382a0       __flush                    300392a0 f   LIBCMTD:fflush.obj
 0001:00038360       __flushall                 30039360 f   LIBCMTD:fflush.obj
 0001:000384b0       __Getdays                  300394b0 f   LIBCMTD:strftime.obj
 0001:000385e0       __Getmonths                300395e0 f   LIBCMTD:strftime.obj
 0001:00038710       __Gettnames                30039710 f   LIBCMTD:strftime.obj
 0001:00038a80       _strftime                  30039a80 f   LIBCMTD:strftime.obj
 0001:00038aa0       __Strftime                 30039aa0 f   LIBCMTD:strftime.obj
 0001:00039920       ___getlocaleinfo           3003a920 f   LIBCMTD:inithelp.obj
 0001:00039bb0       _localeconv                3003abb0 f   LIBCMTD:lconv.obj
 0001:00039bc0       ___crtGetStringTypeW       3003abc0 f   LIBCMTD:w_str.obj
 0001:00039e30       __stricmp                  3003ae30 f   LIBCMTD:stricmp.obj
 0001:00039e30       __strcmpi                  3003ae30 f   LIBCMTD:stricmp.obj
 0001:00039f00       __strnicmp                 3003af00 f   LIBCMTD:strnicmp.obj
 0001:0003a010       ___ld12mul                 3003b010 f   LIBCMTD:tenpow.obj
 0001:0003a450       ___multtenpow12            3003b450 f   LIBCMTD:tenpow.obj
 0001:0003a520       _fclose                    3003b520 f   LIBCMTD:fclose.obj
 0001:0003a5b0       __fclose_lk                3003b5b0 f   LIBCMTD:fclose.obj
 0001:0003a670       __commit                   3003b670 f   LIBCMTD:commit.obj
 0001:0003a750       ___tzset                   3003b750 f   LIBCMTD:tzset.obj
 0001:0003a790       __tzset                    3003b790 f   LIBCMTD:tzset.obj
 0001:0003ab60       __isindst                  3003bb60 f   LIBCMTD:tzset.obj
 0001:0003b090       ___crtGetLocaleInfoW       3003c090 f   LIBCMTD:w_loc.obj
 0001:0003b230       ___crtGetLocaleInfoA       3003c230 f   LIBCMTD:a_loc.obj
 0001:0003b3e0       __close                    3003c3e0 f   LIBCMTD:close.obj
 0001:0003b460       __close_lk                 3003c460 f   LIBCMTD:close.obj
 0001:0003b510       __freebuf                  3003c510 f   LIBCMTD:_freebuf.obj
 0001:0003b5b0       _getenv                    3003c5b0 f   LIBCMTD:getenv.obj
 0001:0003b5e0       __getenv_lk                3003c5e0 f   LIBCMTD:getenv.obj
 0001:0003b6b0       __mbsnbicoll               3003c6b0 f   LIBCMTD:mbsnbico.obj
 0001:0003b700       ___wtomb_environ           3003c700 f   LIBCMTD:wtombenv.obj
 0001:0003b7b0       ___crtCompareStringA       3003c7b0 f   LIBCMTD:a_cmp.obj
 0001:0003bc00       ___crtsetenv               3003cc00 f   LIBCMTD:setenv.obj
 0001:0003c050       __mbschr                   3003d050 f   LIBCMTD:mbschr.obj
 0001:0003c13e       _InterlockedDecrement@4    3003d13e f   kernel32:KERNEL32.dll
 0001:0003c144       _InterlockedIncrement@4    3003d144 f   kernel32:KERNEL32.dll
 0001:0003c14a       _GetCommandLineA@0         3003d14a f   kernel32:KERNEL32.dll
 0001:0003c150       _GetVersion@0              3003d150 f   kernel32:KERNEL32.dll
 0001:0003c156       _GetProcAddress@8          3003d156 f   kernel32:KERNEL32.dll
 0001:0003c15c       _GetModuleHandleA@4        3003d15c f   kernel32:KERNEL32.dll
 0001:0003c162       _RaiseException@16         3003d162 f   kernel32:KERNEL32.dll
 0001:0003c168       _DebugBreak@0              3003d168 f   kernel32:KERNEL32.dll
 0001:0003c16e       _GetStdHandle@4            3003d16e f   kernel32:KERNEL32.dll
 0001:0003c174       _WriteFile@20              3003d174 f   kernel32:KERNEL32.dll
 0001:0003c17a       _OutputDebugStringA@4      3003d17a f   kernel32:KERNEL32.dll
 0001:0003c180       _LoadLibraryA@4            3003d180 f   kernel32:KERNEL32.dll
 0001:0003c186       _GetModuleFileNameA@12     3003d186 f   kernel32:KERNEL32.dll
 0001:0003c18c       _InitializeCriticalSection@4 3003d18c f   kernel32:KERNEL32.dll
 0001:0003c192       _DeleteCriticalSection@4   3003d192 f   kernel32:KERNEL32.dll
 0001:0003c198       _EnterCriticalSection@4    3003d198 f   kernel32:KERNEL32.dll
 0001:0003c19e       _LeaveCriticalSection@4    3003d19e f   kernel32:KERNEL32.dll
 0001:0003c1a4       _ExitProcess@4             3003d1a4 f   kernel32:KERNEL32.dll
 0001:0003c1aa       _FatalAppExitA@8           3003d1aa f   kernel32:KERNEL32.dll
 0001:0003c1b0       _Sleep@4                   3003d1b0 f   kernel32:KERNEL32.dll
 0001:0003c1b6       _WideCharToMultiByte@32    3003d1b6 f   kernel32:KERNEL32.dll
 0001:0003c1bc       _MultiByteToWideChar@24    3003d1bc f   kernel32:KERNEL32.dll
 0001:0003c1c2       _LCMapStringA@24           3003d1c2 f   kernel32:KERNEL32.dll
 0001:0003c1c8       _LCMapStringW@24           3003d1c8 f   kernel32:KERNEL32.dll
 0001:0003c1ce       _TerminateProcess@8        3003d1ce f   kernel32:KERNEL32.dll
 0001:0003c1d4       _GetCurrentProcess@0       3003d1d4 f   kernel32:KERNEL32.dll
 0001:0003c1da       _GetCurrentThreadId@0      3003d1da f   kernel32:KERNEL32.dll
 0001:0003c1e0       _TlsSetValue@8             3003d1e0 f   kernel32:KERNEL32.dll
 0001:0003c1e6       _TlsAlloc@0                3003d1e6 f   kernel32:KERNEL32.dll
 0001:0003c1ec       _TlsFree@4                 3003d1ec f   kernel32:KERNEL32.dll
 0001:0003c1f2       _SetLastError@4            3003d1f2 f   kernel32:KERNEL32.dll
 0001:0003c1f8       _TlsGetValue@4             3003d1f8 f   kernel32:KERNEL32.dll
 0001:0003c1fe       _GetLastError@0            3003d1fe f   kernel32:KERNEL32.dll
 0001:0003c204       _GetCurrentThread@0        3003d204 f   kernel32:KERNEL32.dll
 0001:0003c20a       _SetHandleCount@4          3003d20a f   kernel32:KERNEL32.dll
 0001:0003c210       _GetFileType@4             3003d210 f   kernel32:KERNEL32.dll
 0001:0003c216       _GetStartupInfoA@4         3003d216 f   kernel32:KERNEL32.dll
 0001:0003c21c       _IsBadWritePtr@8           3003d21c f   kernel32:KERNEL32.dll
 0001:0003c222       _IsBadReadPtr@8            3003d222 f   kernel32:KERNEL32.dll
 0001:0003c228       _HeapValidate@12           3003d228 f   kernel32:KERNEL32.dll
 0001:0003c22e       _FreeEnvironmentStringsA@4 3003d22e f   kernel32:KERNEL32.dll
 0001:0003c234       _FreeEnvironmentStringsW@4 3003d234 f   kernel32:KERNEL32.dll
 0001:0003c23a       _GetEnvironmentStrings@0   3003d23a f   kernel32:KERNEL32.dll
 0001:0003c240       _GetEnvironmentStringsW@0  3003d240 f   kernel32:KERNEL32.dll
 0001:0003c246       _HeapDestroy@4             3003d246 f   kernel32:KERNEL32.dll
 0001:0003c24c       _HeapCreate@12             3003d24c f   kernel32:KERNEL32.dll
 0001:0003c252       _HeapFree@12               3003d252 f   kernel32:KERNEL32.dll
 0001:0003c258       _VirtualFree@12            3003d258 f   kernel32:KERNEL32.dll
 0001:0003c25e       _GetStringTypeA@20         3003d25e f   kernel32:KERNEL32.dll
 0001:0003c264       _GetStringTypeW@16         3003d264 f   kernel32:KERNEL32.dll
 0001:0003c26a       _SetFilePointer@16         3003d26a f   kernel32:KERNEL32.dll
 0001:0003c270       _SetConsoleCtrlHandler@8   3003d270 f   kernel32:KERNEL32.dll
 0001:0003c276       _GetCPInfo@8               3003d276 f   kernel32:KERNEL32.dll
 0001:0003c27c       _IsValidLocale@8           3003d27c f   kernel32:KERNEL32.dll
 0001:0003c282       _IsValidCodePage@4         3003d282 f   kernel32:KERNEL32.dll
 0001:0003c288       _GetLocaleInfoA@16         3003d288 f   kernel32:KERNEL32.dll
 0001:0003c28e       _EnumSystemLocalesA@8      3003d28e f   kernel32:KERNEL32.dll
 0001:0003c294       _GetUserDefaultLCID@0      3003d294 f   kernel32:KERNEL32.dll
 0001:0003c29a       _GetVersionExA@4           3003d29a f   kernel32:KERNEL32.dll
 0001:0003c2a0       _RtlUnwind@16              3003d2a0 f   kernel32:KERNEL32.dll
 0001:0003c2a6       _UnhandledExceptionFilter@4 3003d2a6 f   kernel32:KERNEL32.dll
 0001:0003c2ac       _HeapAlloc@12              3003d2ac f   kernel32:KERNEL32.dll
 0001:0003c2b2       _HeapReAlloc@16            3003d2b2 f   kernel32:KERNEL32.dll
 0001:0003c2b8       _VirtualAlloc@16           3003d2b8 f   kernel32:KERNEL32.dll
 0001:0003c2be       _GetACP@0                  3003d2be f   kernel32:KERNEL32.dll
 0001:0003c2c4       _GetOEMCP@0                3003d2c4 f   kernel32:KERNEL32.dll
 0001:0003c2ca       _SetStdHandle@8            3003d2ca f   kernel32:KERNEL32.dll
 0001:0003c2d0       _FlushFileBuffers@4        3003d2d0 f   kernel32:KERNEL32.dll
 0001:0003c2d6       _GetTimeZoneInformation@4  3003d2d6 f   kernel32:KERNEL32.dll
 0001:0003c2dc       _GetLocaleInfoW@16         3003d2dc f   kernel32:KERNEL32.dll
 0001:0003c2e2       _CloseHandle@4             3003d2e2 f   kernel32:KERNEL32.dll
 0001:0003c2e8       _CompareStringA@24         3003d2e8 f   kernel32:KERNEL32.dll
 0001:0003c2ee       _CompareStringW@24         3003d2ee f   kernel32:KERNEL32.dll
 0001:0003c2f4       _SetEnvironmentVariableA@8 3003d2f4 f   kernel32:KERNEL32.dll
 0002:00000020       __real@8@3ffbccccccccccccd000 3003e020     bg_lib.obj
 0002:00000028       __real@4@4002a000000000000000 3003e028     bg_lib.obj
 0002:00000030       __real@8@00000000000000000000 3003e030     bg_lib.obj
 0002:00000038       ??_C@_0FM@ILPP@sound?1teamplay?1flagcap_blu?4wav?5s@ 3003e038     bg_misc.obj
 0002:00000094       ??_C@_09DHIB@Blue?5Flag?$AA@ 3003e094     bg_misc.obj
 0002:000000a0       ??_C@_0BB@NLLL@icons?1iconf_blu1?$AA@ 3003e0a0     bg_misc.obj
 0002:000000b4       ??_C@_0BI@ILPD@models?1flags?1b_flag?4md3?$AA@ 3003e0b4     bg_misc.obj
 0002:000000cc       ??_C@_0BO@HCGD@sound?1teamplay?1flagtk_blu?4wav?$AA@ 3003e0cc     bg_misc.obj
 0002:000000ec       ??_C@_0BC@GPLF@team_CTF_blueflag?$AA@ 3003e0ec     bg_misc.obj
 0002:00000100       ??_C@_0FM@LMNP@sound?1teamplay?1flagcap_red?4wav?5s@ 3003e100     bg_misc.obj
 0002:0000015c       ??_C@_08CLEI@Red?5Flag?$AA@ 3003e15c     bg_misc.obj
 0002:00000168       ??_C@_0BB@DADK@icons?1iconf_red1?$AA@ 3003e168     bg_misc.obj
 0002:0000017c       ??_C@_0BI@HHNH@models?1flags?1r_flag?4md3?$AA@ 3003e17c     bg_misc.obj
 0002:00000194       ??_C@_0BO@BOI@sound?1teamplay?1flagtk_red?4wav?$AA@ 3003e194     bg_misc.obj
 0002:000001b4       ??_C@_0BB@FOCB@team_CTF_redflag?$AA@ 3003e1b4     bg_misc.obj
 0002:000001c8       ??_C@_06CPDM@Flight?$AA@   3003e1c8     bg_misc.obj
 0002:000001d0       ??_C@_0N@DFIJ@icons?1flight?$AA@ 3003e1d0     bg_misc.obj
 0002:000001e0       ??_C@_0CI@PHJ@models?1powerups?1instant?1flight_r@ 3003e1e0     bg_misc.obj
 0002:00000208       ??_C@_0CD@MKAO@models?1powerups?1instant?1flight?4m@ 3003e208     bg_misc.obj
 0002:0000022c       ??_C@_0BH@FEAN@sound?1items?1flight?4wav?$AA@ 3003e22c     bg_misc.obj
 0002:00000244       ??_C@_0M@NKLB@item_flight?$AA@ 3003e244     bg_misc.obj
 0002:00000250       ??_C@_0BG@JFPE@sound?1items?1regen?4wav?$AA@ 3003e250     bg_misc.obj
 0002:00000268       ??_C@_0N@KKJF@Regeneration?$AA@ 3003e268     bg_misc.obj
 0002:00000278       ??_C@_0M@KGFF@icons?1regen?$AA@ 3003e278     bg_misc.obj
 0002:00000284       ??_C@_0CH@LMHA@models?1powerups?1instant?1regen_ri@ 3003e284     bg_misc.obj
 0002:000002ac       ??_C@_0CC@JDKK@models?1powerups?1instant?1regen?4md@ 3003e2ac     bg_misc.obj
 0002:000002d0       ??_C@_0BN@ELHM@sound?1items?1regeneration?4wav?$AA@ 3003e2d0     bg_misc.obj
 0002:000002f0       ??_C@_0L@JOKD@item_regen?$AA@ 3003e2f0     bg_misc.obj
 0002:000002fc       ??_C@_0N@PHMD@Invisibility?$AA@ 3003e2fc     bg_misc.obj
 0002:0000030c       ??_C@_0M@GBKC@icons?1invis?$AA@ 3003e30c     bg_misc.obj
 0002:00000318       ??_C@_0CH@FMDJ@models?1powerups?1instant?1invis_ri@ 3003e318     bg_misc.obj
 0002:00000340       ??_C@_0CC@GFDH@models?1powerups?1instant?1invis?4md@ 3003e340     bg_misc.obj
 0002:00000364       ??_C@_0BN@JBDA@sound?1items?1invisibility?4wav?$AA@ 3003e364     bg_misc.obj
 0002:00000384       ??_C@_0L@FJFE@item_invis?$AA@ 3003e384     bg_misc.obj
 0002:00000390       ??_C@_05PDDA@Speed?$AA@    3003e390     bg_misc.obj
 0002:00000398       ??_C@_0M@MOBK@icons?1haste?$AA@ 3003e398     bg_misc.obj
 0002:000003a4       ??_C@_0CH@HLNN@models?1powerups?1instant?1haste_ri@ 3003e3a4     bg_misc.obj
 0002:000003cc       ??_C@_0CC@HMKI@models?1powerups?1instant?1haste?4md@ 3003e3cc     bg_misc.obj
 0002:000003f0       ??_C@_0BG@HKPG@sound?1items?1haste?4wav?$AA@ 3003e3f0     bg_misc.obj
 0002:00000408       ??_C@_0L@PGOM@item_haste?$AA@ 3003e408     bg_misc.obj
 0002:00000414       ??_C@_0DA@KGOL@sound?1items?1airout?4wav?5sound?1ite@ 3003e414     bg_misc.obj
 0002:00000444       ??_C@_0M@LDNA@Battle?5Suit?$AA@ 3003e444     bg_misc.obj
 0002:00000450       ??_C@_0BB@LIEJ@icons?1envirosuit?$AA@ 3003e450     bg_misc.obj
 0002:00000464       ??_C@_0CI@BLEN@models?1powerups?1instant?1enviro_r@ 3003e464     bg_misc.obj
 0002:0000048c       ??_C@_0CD@EJAP@models?1powerups?1instant?1enviro?4m@ 3003e48c     bg_misc.obj
 0002:000004b0       ??_C@_0BI@LHNB@sound?1items?1protect?4wav?$AA@ 3003e4b0     bg_misc.obj
 0002:000004c8       ??_C@_0M@CNAP@item_enviro?$AA@ 3003e4c8     bg_misc.obj
 0002:000004d4       ??_C@_0DA@MMGJ@sound?1items?1damage2?4wav?5sound?1it@ 3003e4d4     bg_misc.obj
 0002:00000504       ??_C@_0M@MLLH@Quad?5Damage?$AA@ 3003e504     bg_misc.obj
 0002:00000510       ??_C@_0L@CMEC@icons?1quad?$AA@ 3003e510     bg_misc.obj
 0002:0000051c       ??_C@_0CG@HCKJ@models?1powerups?1instant?1quad_rin@ 3003e51c     bg_misc.obj
 0002:00000544       ??_C@_0CB@LCDA@models?1powerups?1instant?1quad?4md3@ 3003e544     bg_misc.obj
 0002:00000568       ??_C@_0BL@FBJD@sound?1items?1quaddamage?4wav?$AA@ 3003e568     bg_misc.obj
 0002:00000584       ??_C@_09NKAN@item_quad?$AA@ 3003e584     bg_misc.obj
 0002:00000590       ??_C@_0BL@LIGH@sound?1items?1use_medkit?4wav?$AA@ 3003e590     bg_misc.obj
 0002:000005ac       ??_C@_06MJBN@Medkit?$AA@   3003e5ac     bg_misc.obj
 0002:000005b4       ??_C@_0N@NDKI@icons?1medkit?$AA@ 3003e5b4     bg_misc.obj
 0002:000005c4       ??_C@_0CL@EEMI@models?1powerups?1holdable?1medkit_@ 3003e5c4     bg_misc.obj
 0002:000005f0       ??_C@_0CE@BLCG@models?1powerups?1holdable?1medkit?4@ 3003e5f0     bg_misc.obj
 0002:00000614       ??_C@_0BA@HJCK@holdable_medkit?$AA@ 3003e614     bg_misc.obj
 0002:00000624       ??_C@_0BE@NHOP@Personal?5Teleporter?$AA@ 3003e624     bg_misc.obj
 0002:00000638       ??_C@_0BB@EOIF@icons?1teleporter?$AA@ 3003e638     bg_misc.obj
 0002:0000064c       ??_C@_0CI@EJIK@models?1powerups?1holdable?1telepor@ 3003e64c     bg_misc.obj
 0002:00000674       ??_C@_0BJ@PMCF@sound?1items?1holdable?4wav?$AA@ 3003e674     bg_misc.obj
 0002:00000690       ??_C@_0BE@EFDD@holdable_teleporter?$AA@ 3003e690     bg_misc.obj
 0002:000006a4       ??_C@_0M@PLAB@ammo_energy?$AA@ 3003e6a4     bg_misc.obj
 0002:000006b0       ??_C@_08HHBB@Bfg?5Ammo?$AA@ 3003e6b0     bg_misc.obj
 0002:000006bc       ??_C@_0BA@LIKB@icons?1icona_bfg?$AA@ 3003e6bc     bg_misc.obj
 0002:000006cc       ??_C@_0BP@KGME@models?1powerups?1ammo?1bfgam?4md3?$AA@ 3003e6cc     bg_misc.obj
 0002:000006ec       ??_C@_08BHPM@ammo_bfg?$AA@ 3003e6ec     bg_misc.obj
 0002:000006f8       ??_C@_05OJGD@Slugs?$AA@    3003e6f8     bg_misc.obj
 0002:00000700       ??_C@_0BE@KFKB@icons?1icona_railgun?$AA@ 3003e700     bg_misc.obj
 0002:00000714       ??_C@_0CD@BHHI@models?1powerups?1ammo?1railgunam?4m@ 3003e714     bg_misc.obj
 0002:00000738       ??_C@_0L@PCJD@ammo_slugs?$AA@ 3003e738     bg_misc.obj
 0002:00000744       ??_C@_07ONGL@Rockets?$AA@  3003e744     bg_misc.obj
 0002:0000074c       ??_C@_0BD@NDBD@icons?1icona_rocket?$AA@ 3003e74c     bg_misc.obj
 0002:00000760       ??_C@_0CC@JMHP@models?1powerups?1ammo?1rocketam?4md@ 3003e760     bg_misc.obj
 0002:00000784       ??_C@_0N@DEF@ammo_rockets?$AA@ 3003e784     bg_misc.obj
 0002:00000794       ??_C@_09NPLP@Lightning?$AA@ 3003e794     bg_misc.obj
 0002:000007a0       ??_C@_0BG@BLCM@icons?1icona_lightning?$AA@ 3003e7a0     bg_misc.obj
 0002:000007b8       ??_C@_0CF@DECD@models?1powerups?1ammo?1lightningam@ 3003e7b8     bg_misc.obj
 0002:000007e0       ??_C@_0P@FNDL@ammo_lightning?$AA@ 3003e7e0     bg_misc.obj
 0002:000007f0       ??_C@_05IJJG@Cells?$AA@    3003e7f0     bg_misc.obj
 0002:000007f8       ??_C@_0BD@PPKI@icons?1icona_plasma?$AA@ 3003e7f8     bg_misc.obj
 0002:0000080c       ??_C@_0CC@GNJA@models?1powerups?1ammo?1plasmaam?4md@ 3003e80c     bg_misc.obj
 0002:00000830       ??_C@_0L@JCGG@ammo_cells?$AA@ 3003e830     bg_misc.obj
 0002:0000083c       ??_C@_08CFEJ@Grenades?$AA@ 3003e83c     bg_misc.obj
 0002:00000848       ??_C@_0BE@MMLE@icons?1icona_grenade?$AA@ 3003e848     bg_misc.obj
 0002:0000085c       ??_C@_0CD@NMEK@models?1powerups?1ammo?1grenadeam?4m@ 3003e85c     bg_misc.obj
 0002:00000880       ??_C@_0O@KBKH@ammo_grenades?$AA@ 3003e880     bg_misc.obj
 0002:00000890       ??_C@_07EDBM@Bullets?$AA@  3003e890     bg_misc.obj
 0002:00000898       ??_C@_0BH@DHGM@icons?1icona_machinegun?$AA@ 3003e898     bg_misc.obj
 0002:000008b0       ??_C@_0CG@KHPE@models?1powerups?1ammo?1machineguna@ 3003e8b0     bg_misc.obj
 0002:000008d8       ??_C@_0N@KNDC@ammo_bullets?$AA@ 3003e8d8     bg_misc.obj
 0002:000008e8       ??_C@_06OAJC@Shells?$AA@   3003e8e8     bg_misc.obj
 0002:000008f0       ??_C@_0BE@MPL@icons?1icona_shotgun?$AA@ 3003e8f0     bg_misc.obj
 0002:00000904       ??_C@_0CD@LJLN@models?1powerups?1ammo?1shotgunam?4m@ 3003e904     bg_misc.obj
 0002:00000928       ??_C@_0BH@EMHN@sound?1misc?1am_pkup?4wav?$AA@ 3003e928     bg_misc.obj
 0002:00000940       ??_C@_0M@MOIJ@ammo_shells?$AA@ 3003e940     bg_misc.obj
 0002:0000094c       ??_C@_0P@MANM@Grappling?5Hook?$AA@ 3003e94c     bg_misc.obj
 0002:0000095c       ??_C@_0BE@IDGG@icons?1iconw_grapple?$AA@ 3003e95c     bg_misc.obj
 0002:00000970       ??_C@_0CE@LPMO@models?1weapons2?1grapple?1grapple?4@ 3003e970     bg_misc.obj
 0002:00000994       ??_C@_0BF@GCPL@weapon_grapplinghook?$AA@ 3003e994     bg_misc.obj
 0002:000009ac       ??_C@_06KEGK@BFG10K?$AA@   3003e9ac     bg_misc.obj
 0002:000009b4       ??_C@_0BA@HKCL@icons?1iconw_bfg?$AA@ 3003e9b4     bg_misc.obj
 0002:000009c4       ??_C@_0BM@MFN@models?1weapons2?1bfg?1bfg?4md3?$AA@ 3003e9c4     bg_misc.obj
 0002:000009e0       ??_C@_0L@NOHL@weapon_bfg?$AA@ 3003e9e0     bg_misc.obj
 0002:000009ec       ??_C@_0L@OMHC@Plasma?5Gun?$AA@ 3003e9ec     bg_misc.obj
 0002:000009f8       ??_C@_0BD@MNKG@icons?1iconw_plasma?$AA@ 3003e9f8     bg_misc.obj
 0002:00000a0c       ??_C@_0CC@DOHF@models?1weapons2?1plasma?1plasma?4md@ 3003ea0c     bg_misc.obj
 0002:00000a30       ??_C@_0BB@IMNM@weapon_plasmagun?$AA@ 3003ea30     bg_misc.obj
 0002:00000a44       ??_C@_07MJPA@Railgun?$AA@  3003ea44     bg_misc.obj
 0002:00000a4c       ??_C@_0BE@MJD@icons?1iconw_railgun?$AA@ 3003ea4c     bg_misc.obj
 0002:00000a60       ??_C@_0CE@GDNL@models?1weapons2?1railgun?1railgun?4@ 3003ea60     bg_misc.obj
 0002:00000a84       ??_C@_0P@FOOL@weapon_railgun?$AA@ 3003ea84     bg_misc.obj
 0002:00000a94       ??_C@_0O@JANJ@Lightning?5Gun?$AA@ 3003ea94     bg_misc.obj
 0002:00000aa4       ??_C@_0BG@MMPA@icons?1iconw_lightning?$AA@ 3003eaa4     bg_misc.obj
 0002:00000abc       ??_C@_0CI@OODD@models?1weapons2?1lightning?1lightn@ 3003eabc     bg_misc.obj
 0002:00000ae4       ??_C@_0BB@GAKO@weapon_lightning?$AA@ 3003eae4     bg_misc.obj
 0002:00000af8       ??_C@_0BA@JFMN@Rocket?5Launcher?$AA@ 3003eaf8     bg_misc.obj
 0002:00000b08       ??_C@_0BD@OBBN@icons?1iconw_rocket?$AA@ 3003eb08     bg_misc.obj
 0002:00000b1c       ??_C@_0CE@CDMO@models?1weapons2?1rocketl?1rocketl?4@ 3003eb1c     bg_misc.obj
 0002:00000b40       ??_C@_0BG@EKMA@weapon_rocketlauncher?$AA@ 3003eb40     bg_misc.obj
 0002:00000b58       ??_C@_0EG@FCJ@sound?1weapons?1grenade?1hgrenb1a?4w@ 3003eb58     bg_misc.obj
 0002:00000ba0       ??_C@_0BB@KEFG@Grenade?5Launcher?$AA@ 3003eba0     bg_misc.obj
 0002:00000bb4       ??_C@_0BE@GFIG@icons?1iconw_grenade?$AA@ 3003ebb4     bg_misc.obj
 0002:00000bc8       ??_C@_0CG@MONC@models?1weapons2?1grenadel?1grenade@ 3003ebc8     bg_misc.obj
 0002:00000bf0       ??_C@_0BH@FDFB@weapon_grenadelauncher?$AA@ 3003ebf0     bg_misc.obj
 0002:00000c08       ??_C@_0L@OIKI@Machinegun?$AA@ 3003ec08     bg_misc.obj
 0002:00000c14       ??_C@_0BH@IFLL@icons?1iconw_machinegun?$AA@ 3003ec14     bg_misc.obj
 0002:00000c2c       ??_C@_0CK@BP@models?1weapons2?1machinegun?1machi@ 3003ec2c     bg_misc.obj
 0002:00000c58       ??_C@_0BC@JMBH@weapon_machinegun?$AA@ 3003ec58     bg_misc.obj
 0002:00000c6c       ??_C@_07GAKK@Shotgun?$AA@  3003ec6c     bg_misc.obj
 0002:00000c74       ??_C@_0BE@KFMJ@icons?1iconw_shotgun?$AA@ 3003ec74     bg_misc.obj
 0002:00000c88       ??_C@_0CE@FIBC@models?1weapons2?1shotgun?1shotgun?4@ 3003ec88     bg_misc.obj
 0002:00000cac       ??_C@_0P@PHLB@weapon_shotgun?$AA@ 3003ecac     bg_misc.obj
 0002:00000cbc       ??_C@_08MFME@Gauntlet?$AA@ 3003ecbc     bg_misc.obj
 0002:00000cc8       ??_C@_0CG@ENLL@models?1weapons2?1gauntlet?1gauntle@ 3003ecc8     bg_misc.obj
 0002:00000cf0       ??_C@_0BA@NEFD@weapon_gauntlet?$AA@ 3003ecf0     bg_misc.obj
 0002:00000d00       ??_C@_04FEBI@Fist?$AA@     3003ed00     bg_misc.obj
 0002:00000d08       ??_C@_0BF@IKAB@icons?1iconw_gauntlet?$AA@ 3003ed08     bg_misc.obj
 0002:00000d20       ??_C@_0BG@OBIE@sound?1misc?1w_pkup?4wav?$AA@ 3003ed20     bg_misc.obj
 0002:00000d38       ??_C@_0M@OGLA@weapon_none?$AA@ 3003ed38     bg_misc.obj
 0002:00000d44       ??_C@_0M@MPBK@Mega?5Health?$AA@ 3003ed44     bg_misc.obj
 0002:00000d50       ??_C@_0BB@FCLL@icons?1iconh_mega?$AA@ 3003ed50     bg_misc.obj
 0002:00000d64       ??_C@_0CH@HNCC@models?1powerups?1health?1mega_sphe@ 3003ed64     bg_misc.obj
 0002:00000d8c       ??_C@_0CG@GJOF@models?1powerups?1health?1mega_cros@ 3003ed8c     bg_misc.obj
 0002:00000db4       ??_C@_0BJ@GHGJ@sound?1items?1m_health?4wav?$AA@ 3003edb4     bg_misc.obj
 0002:00000dd0       ??_C@_0BB@KJE@item_health_mega?$AA@ 3003edd0     bg_misc.obj
 0002:00000de4       ??_C@_09DDEP@50?5Health?$AA@ 3003ede4     bg_misc.obj
 0002:00000df0       ??_C@_0BA@PMIC@icons?1iconh_red?$AA@ 3003edf0     bg_misc.obj
 0002:00000e00       ??_C@_0CI@LKJF@models?1powerups?1health?1large_sph@ 3003ee00     bg_misc.obj
 0002:00000e28       ??_C@_0CH@NOLN@models?1powerups?1health?1large_cro@ 3003ee28     bg_misc.obj
 0002:00000e50       ??_C@_0BJ@KID@sound?1items?1l_health?4wav?$AA@ 3003ee50     bg_misc.obj
 0002:00000e6c       ??_C@_0BC@KFF@item_health_large?$AA@ 3003ee6c     bg_misc.obj
 0002:00000e80       ??_C@_09BECD@25?5Health?$AA@ 3003ee80     bg_misc.obj
 0002:00000e8c       ??_C@_0BD@IBDP@icons?1iconh_yellow?$AA@ 3003ee8c     bg_misc.obj
 0002:00000ea0       ??_C@_0CJ@KCHG@models?1powerups?1health?1medium_sp@ 3003eea0     bg_misc.obj
 0002:00000ecc       ??_C@_0CI@DNPD@models?1powerups?1health?1medium_cr@ 3003eecc     bg_misc.obj
 0002:00000ef4       ??_C@_0BJ@NBFG@sound?1items?1n_health?4wav?$AA@ 3003eef4     bg_misc.obj
 0002:00000f10       ??_C@_0M@DFKC@item_health?$AA@ 3003ef10     bg_misc.obj
 0002:00000f1c       ??_C@_08PNDE@5?5Health?$AA@ 3003ef1c     bg_misc.obj
 0002:00000f28       ??_C@_0BC@CNMA@icons?1iconh_green?$AA@ 3003ef28     bg_misc.obj
 0002:00000f3c       ??_C@_0CI@MNOG@models?1powerups?1health?1small_sph@ 3003ef3c     bg_misc.obj
 0002:00000f64       ??_C@_0CH@KNOH@models?1powerups?1health?1small_cro@ 3003ef64     bg_misc.obj
 0002:00000f8c       ??_C@_0BJ@LKOK@sound?1items?1s_health?4wav?$AA@ 3003ef8c     bg_misc.obj
 0002:00000fa8       ??_C@_0BC@HBNN@item_health_small?$AA@ 3003efa8     bg_misc.obj
 0002:00000fbc       ??_C@_0M@LPCG@Heavy?5Armor?$AA@ 3003efbc     bg_misc.obj
 0002:00000fc8       ??_C@_0BA@LPLH@icons?1iconr_red?$AA@ 3003efc8     bg_misc.obj
 0002:00000fd8       ??_C@_0CE@HDBK@models?1powerups?1armor?1armor_red?4@ 3003efd8     bg_misc.obj
 0002:00000ffc       ??_C@_0BI@JMAI@sound?1misc?1ar3_pkup?4wav?$AA@ 3003effc     bg_misc.obj
 0002:00001014       ??_C@_0BA@GFMA@item_armor_body?$AA@ 3003f014     bg_misc.obj
 0002:00001024       ??_C@_05KFDN@Armor?$AA@    3003f024     bg_misc.obj
 0002:0000102c       ??_C@_0BD@NCPP@icons?1iconr_yellow?$AA@ 3003f02c     bg_misc.obj
 0002:00001040       ??_C@_0CE@HFCD@models?1powerups?1armor?1armor_yel?4@ 3003f040     bg_misc.obj
 0002:00001064       ??_C@_0BI@BDMK@sound?1misc?1ar2_pkup?4wav?$AA@ 3003f064     bg_misc.obj
 0002:0000107c       ??_C@_0BC@GPNI@item_armor_combat?$AA@ 3003f07c     bg_misc.obj
 0002:00001090       ??_C@_0M@KPGH@Armor?5Shard?$AA@ 3003f090     bg_misc.obj
 0002:0000109c       ??_C@_0BC@BIPJ@icons?1iconr_shard?$AA@ 3003f09c     bg_misc.obj
 0002:000010b0       ??_C@_0CH@FIOC@models?1powerups?1armor?1shard_sphe@ 3003f0b0     bg_misc.obj
 0002:000010d8       ??_C@_0CA@DPKE@models?1powerups?1armor?1shard?4md3?$AA@ 3003f0d8     bg_misc.obj
 0002:000010f8       ??_C@_0BI@IDIM@sound?1misc?1ar1_pkup?4wav?$AA@ 3003f0f8     bg_misc.obj
 0002:00001110       ??_C@_0BB@JODA@item_armor_shard?$AA@ 3003f110     bg_misc.obj
 0002:00001124       ??_C@_00A@?$AA@            3003f124     bg_misc.obj
 0002:00001128       ??_C@_0BH@HPPA@HoldableItem?5not?5found?$AA@ 3003f128     bg_misc.obj
 0002:00001140       ??_C@_0CB@NJCB@Couldn?8t?5find?5item?5for?5weapon?5?$CFi@ 3003f140     bg_misc.obj
 0002:00001164       ??_C@_0CB@OKOG@Couldn?8t?5find?5ammo?5for?5weapon?5?$CFi@ 3003f164     bg_misc.obj
 0002:00001188       __real@4@c0049000000000000000 3003f188     bg_misc.obj
 0002:0000118c       __real@4@40049000000000000000 3003f18c     bg_misc.obj
 0002:00001190       __real@4@c004c800000000000000 3003f190     bg_misc.obj
 0002:00001194       __real@4@4004b000000000000000 3003f194     bg_misc.obj
 0002:00001198       ??_C@_0BM@HEIN@BG_CanItemBeGrabbed?3?5IT_BAD?$AA@ 3003f198     bg_misc.obj
 0002:000011b4       ??_C@_0CI@DJME@BG_CanItemBeGrabbed?3?5index?5out?5o@ 3003f1b4     bg_misc.obj
 0002:000011dc       ??_C@_0CK@CFCO@BG_EvaluateTrajectory?3?5unknown?5t@ 3003f1dc     bg_misc.obj
 0002:00001208       __real@8@4007c800000000000000 3003f208     bg_misc.obj
 0002:00001210       __real@4@00000000000000000000 3003f210     bg_misc.obj
 0002:00001218       __real@8@4000c90fdaa22168c000 3003f218     bg_misc.obj
 0002:00001220       __real@8@3ff583126e978d4fe000 3003f220     bg_misc.obj
 0002:00001228       ??_C@_0CP@HAJH@BG_EvaluateTrajectoryDelta?3?5unkn@ 3003f228     bg_misc.obj
 0002:00001258       __real@4@4008c800000000000000 3003f258     bg_misc.obj
 0002:00001260       __real@8@3ffe8000000000000000 3003f260     bg_misc.obj
 0002:00001268       __real@8@3ff7b400000000000000 3003f268     bg_pmove.obj
 0002:00001270       __real@4@3fff8000000000000000 3003f270     bg_pmove.obj
 0002:00001278       __real@8@4005fe00000000000000 3003f278     bg_pmove.obj
 0002:00001280       __real@4@4006c800000000000000 3003f280     bg_pmove.obj
 0002:00001284       __real@4@40038000000000000000 3003f284     bg_pmove.obj
 0002:00001288       __real@4@40018000000000000000 3003f288     bg_pmove.obj
 0002:0000128c       __real@4@4003f000000000000000 3003f28c     bg_pmove.obj
 0002:00001290       __real@4@4005c800000000000000 3003f290     bg_pmove.obj
 0002:00001294       __real@4@c0038000000000000000 3003f294     bg_pmove.obj
 0002:00001298       __real@8@3fff8000000000000000 3003f298     bg_pmove.obj
 0002:000012a0       __real@8@4000c000000000000000 3003f2a0     bg_pmove.obj
 0002:000012a8       __real@4@4003a000000000000000 3003f2a8     bg_pmove.obj
 0002:000012b0       __real@8@3fffc000000000000000 3003f2b0     bg_pmove.obj
 0002:000012b8       __real@4@c006c800000000000000 3003f2b8     bg_pmove.obj
 0002:000012bc       ??_C@_08OEON@?$CFi?3Land?6?$AA@ 3003f2bc     bg_pmove.obj
 0002:000012c8       ??_C@_09KHNP@?$CFi?3steep?6?$AA@ 3003f2c8     bg_pmove.obj
 0002:000012d8       __real@8@3ffeb333333333333000 3003f2d8     bg_pmove.obj
 0002:000012e0       ??_C@_0M@CLKI@?$CFi?3kickoff?6?$AA@ 3003f2e0     bg_pmove.obj
 0002:000012f0       __real@8@3ffd8000000000000000 3003f2f0     bg_pmove.obj
 0002:000012f8       __real@4@4001e000000000000000 3003f2f8     bg_pmove.obj
 0002:000012fc       __real@4@4004a000000000000000 3003f2fc     bg_pmove.obj
 0002:00001300       __real@4@4004f000000000000000 3003f300     bg_pmove.obj
 0002:00001308       __real@8@4002e000000000000000 3003f308     bg_pmove.obj
 0002:00001310       __real@8@3ff1d1b71758e2196800 3003f310     bg_pmove.obj
 0002:00001318       __real@4@40008000000000000000 3003f318     bg_pmove.obj
 0002:0000131c       ??_C@_0N@LFAC@?$CFi?3allsolid?6?$AA@ 3003f31c     bg_pmove.obj
 0002:0000132c       __real@4@40058000000000000000 3003f32c     bg_pmove.obj
 0002:00001330       ??_C@_08DAML@?$CFi?3lift?6?$AA@ 3003f330     bg_pmove.obj
 0002:0000133c       __real@4@c003c000000000000000 3003f33c     bg_pmove.obj
 0002:00001340       __real@4@4001a000000000000000 3003f340     bg_pmove.obj
 0002:00001348       __real@8@3fffa666666666666800 3003f348     bg_pmove.obj
 0002:00001350       __real@8@3ffefd70a3d70a3d7000 3003f350     bg_slidemove.obj
 0002:00001358       ??_C@_0M@CBLA@?$CFi?3stepped?6?$AA@ 3003f358     bg_slidemove.obj
 0002:00001364       __real@4@4002f000000000000000 3003f364     bg_slidemove.obj
 0002:00001368       __real@4@4002b000000000000000 3003f368     bg_slidemove.obj
 0002:0000136c       ??_C@_0BE@CFBB@?$CFi?3bend?5can?8t?5step?6?$AA@ 3003f36c     bg_slidemove.obj
 0002:00001380       ??_C@_0M@JPKM@loaddefered?$AA@ 3003f380     cg_consolecmds.obj
 0002:0000138c       ??_C@_04NEDF@tcmd?$AA@     3003f38c     cg_consolecmds.obj
 0002:00001394       ??_C@_0O@IBDB@tell_attacker?$AA@ 3003f394     cg_consolecmds.obj
 0002:000013a4       ??_C@_0M@DEIJ@tell_target?$AA@ 3003f3a4     cg_consolecmds.obj
 0002:000013b0       ??_C@_06IJLN@weapon?$AA@   3003f3b0     cg_consolecmds.obj
 0002:000013b8       ??_C@_08KKEF@weapprev?$AA@ 3003f3b8     cg_consolecmds.obj
 0002:000013c4       ??_C@_08FDMA@weapnext?$AA@ 3003f3c4     cg_consolecmds.obj
 0002:000013d0       ??_C@_08POMM@sizedown?$AA@ 3003f3d0     cg_consolecmds.obj
 0002:000013dc       ??_C@_06IFPB@sizeup?$AA@   3003f3dc     cg_consolecmds.obj
 0002:000013e4       ??_C@_05POM@?9zoom?$AA@    3003f3e4     cg_consolecmds.obj
 0002:000013ec       ??_C@_05MPDD@?$CLzoom?$AA@ 3003f3ec     cg_consolecmds.obj
 0002:000013f4       ??_C@_07BJGL@?9scores?$AA@ 3003f3f4     cg_consolecmds.obj
 0002:000013fc       ??_C@_07POBG@?$CLscores?$AA@ 3003f3fc     cg_consolecmds.obj
 0002:00001404       ??_C@_07NEL@viewpos?$AA@   3003f404     cg_consolecmds.obj
 0002:0000140c       ??_C@_08HKGI@prevskin?$AA@ 3003f40c     cg_consolecmds.obj
 0002:00001418       ??_C@_08FNMJ@nextskin?$AA@ 3003f418     cg_consolecmds.obj
 0002:00001424       ??_C@_09DDNN@prevframe?$AA@ 3003f424     cg_consolecmds.obj
 0002:00001430       ??_C@_09NAPK@nextframe?$AA@ 3003f430     cg_consolecmds.obj
 0002:0000143c       ??_C@_09BKGD@testmodel?$AA@ 3003f43c     cg_consolecmds.obj
 0002:00001448       ??_C@_07JGDN@testgun?$AA@  3003f448     cg_consolecmds.obj
 0002:00001450       ??_C@_08EBEP@gc?5?$CFi?5?$CFi?$AA@ 3003f450     cg_consolecmds.obj
 0002:0000145c       ??_C@_0M@FLKF@cg_viewsize?$AA@ 3003f45c     cg_consolecmds.obj
 0002:00001468       ??_C@_02JAFN@?$CFi?$AA@    3003f468     cg_consolecmds.obj
 0002:0000146c       ??_C@_0BB@DJMJ@?$CI?$CFi?5?$CFi?5?$CFi?$CJ?5?3?5?$CFi?6?$AA@ 3003f46c     cg_consolecmds.obj
 0002:00001480       ??_C@_05FILO@score?$AA@    3003f480     cg_consolecmds.obj
 0002:00001488       ??_C@_0L@BGHL@tell?5?$CFi?5?$CFs?$AA@ 3003f488     cg_consolecmds.obj
 0002:00001494       ??_C@_08BDO@callvote?$AA@  3003f494     cg_consolecmds.obj
 0002:000014a0       ??_C@_04CFLO@vote?$AA@     3003f4a0     cg_consolecmds.obj
 0002:000014a8       ??_C@_0L@NFLA@setviewpos?$AA@ 3003f4a8     cg_consolecmds.obj
 0002:000014b4       ??_C@_06JDOB@addbot?$AA@   3003f4b4     cg_consolecmds.obj
 0002:000014bc       ??_C@_09IADL@levelshot?$AA@ 3003f4bc     cg_consolecmds.obj
 0002:000014c8       ??_C@_06DDCP@follow?$AA@   3003f4c8     cg_consolecmds.obj
 0002:000014d0       ??_C@_04CJJD@team?$AA@     3003f4d0     cg_consolecmds.obj
 0002:000014d8       ??_C@_06GMBK@noclip?$AA@   3003f4d8     cg_consolecmds.obj
 0002:000014e0       ??_C@_08BHIO@notarget?$AA@ 3003f4e0     cg_consolecmds.obj
 0002:000014ec       ??_C@_03IPJE@god?$AA@      3003f4ec     cg_consolecmds.obj
 0002:000014f0       ??_C@_04JEOP@give?$AA@     3003f4f0     cg_consolecmds.obj
 0002:000014f8       ??_C@_08PAEI@say_team?$AA@ 3003f4f8     cg_consolecmds.obj
 0002:00001504       ??_C@_03NJAM@say?$AA@      3003f504     cg_consolecmds.obj
 0002:00001508       ??_C@_04CHLA@kill?$AA@     3003f508     cg_consolecmds.obj
 0002:00001510       __real@8@3ffd89374bc6a7efa000 3003f510     cg_draw.obj
 0002:00001518       __real@8@bffe8000000000000000 3003f518     cg_draw.obj
 0002:00001520       ??_C@_0L@BGKG@tag_barrel?$AA@ 3003f520     cg_draw.obj
 0002:00001530       __real@8@4004f000000000000000 3003f530     cg_draw.obj
 0002:00001538       __real@8@4009fa00000000000000 3003f538     cg_draw.obj
 0002:00001540       ??_C@_0CE@ILIC@CG_DrawActive?3?5Undefined?5stereoV@ 3003f540     cg_draw.obj
 0002:00001568       __real@8@3ffec000000000000000 3003f568     cg_draw.obj
 0002:00001570       __real@8@3ffaa3d70a3d70a3d800 3003f570     cg_draw.obj
 0002:00001578       __real@8@3ff9ccccccccccccd000 3003f578     cg_draw.obj
 0002:00001580       __real@8@3ffb8f5c28f5c28f6000 3003f580     cg_draw.obj
 0002:00001588       __real@8@3ff8a3d70a3d70a3d800 3003f588     cg_draw.obj
 0002:00001590       __real@8@400a8000000000000000 3003f590     cg_draw.obj
 0002:00001598       __real@8@40078700000000000000 3003f598     cg_draw.obj
 0002:000015a0       __real@8@4003a000000000000000 3003f5a0     cg_draw.obj
 0002:000015a8       __real@8@4008fa00000000000000 3003f5a8     cg_draw.obj
 0002:000015b0       __real@4@4007f000000000000000 3003f5b0     cg_draw.obj
 0002:000015b4       __real@4@4000c000000000000000 3003f5b4     cg_draw.obj
 0002:000015b8       __real@4@4009fa00000000000000 3003f5b8     cg_draw.obj
 0002:000015c0       __real@8@4001a000000000000000 3003f5c0     cg_draw.obj
 0002:000015c8       __real@8@4006b400000000000000 3003f5c8     cg_draw.obj
 0002:000015d0       __real@4@400dfffe000000000000 3003f5d0     cg_draw.obj
 0002:000015d4       __real@4@4006b400000000000000 3003f5d4     cg_draw.obj
 0002:000015d8       __real@4@4004b400000000000000 3003f5d8     cg_draw.obj
 0002:000015dc       __real@4@4007fa00000000000000 3003f5dc     cg_draw.obj
 0002:000015e0       ??_C@_01FMOK@n?$AA@        3003f5e0     cg_draw.obj
 0002:000015e4       __real@4@4008a000000000000000 3003f5e4     cg_draw.obj
 0002:000015e8       ??_C@_0BH@JKEJ@time?3?$CFi?5snap?3?$CFi?5cmd?3?$CFi?$AA@ 3003f5e8     cg_draw.obj
 0002:00001600       ??_C@_05EKKA@?$CFifps?$AA@ 3003f600     cg_draw.obj
 0002:00001608       ??_C@_07GKJN@?$CFi?3?$CFi?$CFi?$AA@ 3003f608     cg_draw.obj
 0002:00001610       __real@4@40028000000000000000 3003f610     cg_draw.obj
 0002:00001614       ??_C@_07MFLA@?$CF3i?5?$CF3i?$AA@ 3003f614     cg_draw.obj
 0002:0000161c       ??_C@_07CAMD@unknown?$AA@  3003f61c     cg_draw.obj
 0002:00001624       ??_C@_03MDDI@?$CF2i?$AA@   3003f624     cg_draw.obj
 0002:00001628       __real@4@4003c000000000000000 3003f628     cg_draw.obj
 0002:00001630       __real@8@4004c000000000000000 3003f630     cg_draw.obj
 0002:00001638       __real@4@4008fa00000000000000 3003f638     cg_draw.obj
 0002:0000163c       __real@4@4004c000000000000000 3003f63c     cg_draw.obj
 0002:00001640       ??_C@_03KFOL@snc?$AA@      3003f640     cg_draw.obj
 0002:00001644       __real@4@4008e100000000000000 3003f644     cg_draw.obj
 0002:00001648       __real@4@40079600000000000000 3003f648     cg_draw.obj
 0002:0000164c       ??_C@_0P@LLJP@gfx?12d?1net?4tga?$AA@ 3003f64c     cg_draw.obj
 0002:0000165c       ??_C@_0BH@MGLK@Connection?5Interrupted?$AA@ 3003f65c     cg_draw.obj
 0002:00001674       __real@4@4007a000000000000000 3003f674     cg_draw.obj
 0002:00001678       __real@4@400c8000000000000000 3003f678     cg_draw.obj
 0002:0000167c       ??_C@_0BK@BHOD@use?5the?5TEAM?5menu?5to?5play?$AA@ 3003f67c     cg_draw.obj
 0002:00001698       ??_C@_0BA@GILD@waiting?5to?5play?$AA@ 3003f698     cg_draw.obj
 0002:000016a8       ??_C@_09KPLM@SPECTATOR?$AA@ 3003f6a8     cg_draw.obj
 0002:000016b4       ??_C@_0CB@GGK@VOTE?$CI?$CFi?$CJ?3?$CFs?5yes?$CIF1?$CJ?3?$CFi?5no?$CIF2?$CJ?3?$CFi@ 3003f6b4     cg_draw.obj
 0002:000016d8       ??_C@_09FIOM@following?$AA@ 3003f6d8     cg_draw.obj
 0002:000016e4       ??_C@_0BB@ENDJ@LOW?5AMMO?5WARNING?$AA@ 3003f6e4     cg_draw.obj
 0002:000016f8       ??_C@_0M@OEIB@OUT?5OF?5AMMO?$AA@ 3003f6f8     cg_draw.obj
 0002:00001704       ??_C@_0O@PGJD@Starts?5in?3?5?$CFi?$AA@ 3003f704     cg_draw.obj
 0002:00001714       ??_C@_0BB@EEMI@Capture?5the?5Flag?$AA@ 3003f714     cg_draw.obj
 0002:00001728       ??_C@_0BA@MBBA@Team?5Deathmatch?$AA@ 3003f728     cg_draw.obj
 0002:00001738       ??_C@_0N@EEDI@Free?5For?5All?$AA@ 3003f738     cg_draw.obj
 0002:00001748       ??_C@_08EFHA@?$CFs?5vs?5?$CFs?$AA@ 3003f748     cg_draw.obj
 0002:00001754       ??_C@_0BE@BHPN@Waiting?5for?5players?$AA@ 3003f754     cg_draw.obj
 0002:00001768       __real@8@3ffb8000000000000000 3003f768     cg_drawtools.obj
 0002:00001770       __real@8@40058000000000000000 3003f770     cg_drawtools.obj
 0002:00001778       __real@8@4006c800000000000000 3003f778     cg_drawtools.obj
 0002:00001780       __real@8@4003f000000000000000 3003f780     cg_drawtools.obj
 0002:00001788       __real@8@40048400000000000000 3003f788     cg_drawtools.obj
 0002:00001790       __real@8@3ffdae147ae147ae1000 3003f790     cg_drawtools.obj
 0002:00001798       __real@8@3ffea8f5c28f5c28f800 3003f798     cg_drawtools.obj
 0002:000017a0       __real@4@40078000000000000000 3003f7a0     cg_drawtools.obj
 0002:000017a4       __real@4@3ffec000000000000000 3003f7a4     cg_drawtools.obj
 0002:000017a8       __real@8@3ffeccccccccccccd000 3003f7a8     cg_drawtools.obj
 0002:000017b0       __real@4@4003d800000000000000 3003f7b0     cg_drawtools.obj
 0002:000017b8       __real@8@4001c000000000000000 3003f7b8     cg_effects.obj
 0002:000017c0       __real@4@4006fa00000000000000 3003f7c0     cg_effects.obj
 0002:000017c4       __real@4@4006ff00000000000000 3003f7c4     cg_effects.obj
 0002:000017c8       __real@4@4007b400000000000000 3003f7c8     cg_effects.obj
 0002:000017cc       ??_C@_0BM@JAPN@CG_MakeExplosion?3?5msec?5?$DN?5?$CFi?$AA@ 3003f7cc     cg_effects.obj
 0002:000017e8       __real@4@400abb80000000000000 3003f7e8     cg_effects.obj
 0002:000017f0       __real@8@4006fa00000000000000 3003f7f0     cg_effects.obj
 0002:000017f8       __real@4@40098000000000000000 3003f7f8     cg_ents.obj
 0002:000017fc       ??_C@_0DB@DJJL@CG_InterpoateEntityPosition?3?5cg?4@ 3003f7fc     cg_ents.obj
 0002:00001830       ??_C@_0BF@EHGG@Bad?5entity?5type?3?5?$CFi?6?$AA@ 3003f830     cg_ents.obj
 0002:00001848       __real@4@c0098000000000000000 3003f848     cg_ents.obj
 0002:0000184c       __real@4@4002c000000000000000 3003f84c     cg_ents.obj
 0002:00001850       __real@8@4005c800000000000000 3003f850     cg_ents.obj
 0002:00001858       __real@4@40039000000000000000 3003f858     cg_ents.obj
 0002:00001860       __real@8@40018000000000000000 3003f860     cg_ents.obj
 0002:00001868       __real@8@3ff7a3d70a3d70a3d800 3003f868     cg_ents.obj
 0002:00001870       __real@8@3feea7c5ac471b478800 3003f870     cg_ents.obj
 0002:00001878       ??_C@_0BM@PKOK@Bad?5item?5index?5?$CFi?5on?5entity?$AA@ 3003f878     cg_ents.obj
 0002:00001898       __real@8@40069600000000000000 3003f898     cg_ents.obj
 0002:000018a0       __real@8@4007b400000000000000 3003f8a0     cg_ents.obj
 0002:000018a8       __real@8@40078000000000000000 3003f8a8     cg_ents.obj
 0002:000018b0       ??_C@_04DCMN@?$CFs?$CFs?$AA@ 3003f8b0     cg_event.obj
 0002:000018b8       ??_C@_04PDOI@?$CFith?$AA@  3003f8b8     cg_event.obj
 0002:000018c0       ??_C@_04HKPD@?$CFird?$AA@  3003f8c0     cg_event.obj
 0002:000018c8       ??_C@_04PPKE@?$CFind?$AA@  3003f8c8     cg_event.obj
 0002:000018d0       ??_C@_04MFCJ@?$CFist?$AA@  3003f8d0     cg_event.obj
 0002:000018d8       ??_C@_04KDNJ@13th?$AA@     3003f8d8     cg_event.obj
 0002:000018e0       ??_C@_04PBMP@12th?$AA@     3003f8e0     cg_event.obj
 0002:000018e8       ??_C@_04HPE@11th?$AA@      3003f8e8     cg_event.obj
 0002:000018f0       ??_C@_07KLCB@?$FO33rd?$FO7?$AA@ 3003f8f0     cg_event.obj
 0002:000018f8       ??_C@_07MKLN@?$FO12nd?$FO7?$AA@ 3003f8f8     cg_event.obj
 0002:00001900       ??_C@_07HDD@?$FO41st?$FO7?$AA@ 3003f900     cg_event.obj
 0002:00001908       ??_C@_09HHNH@Tied?5for?5?$AA@ 3003f908     cg_event.obj
 0002:00001914       ??_C@_0P@JFCH@?$CKpain100_1?4wav?$AA@ 3003f914     cg_event.obj
 0002:00001924       ??_C@_0O@HGHK@?$CKpain75_1?4wav?$AA@ 3003f924     cg_event.obj
 0002:00001934       ??_C@_0O@HCOE@?$CKpain50_1?4wav?$AA@ 3003f934     cg_event.obj
 0002:00001944       ??_C@_0O@BOOO@?$CKpain25_1?4wav?$AA@ 3003f944     cg_event.obj
 0002:00001954       ??_C@_0BC@OMBO@Unknown?5event?3?5?$CFi?$AA@ 3003f954     cg_event.obj
 0002:00001968       ??_C@_08JDLL@UNKNOWN?6?$AA@ 3003f968     cg_event.obj
 0002:00001974       ??_C@_0P@DNIF@EV_DEBUG_LINE?6?$AA@ 3003f974     cg_event.obj
 0002:00001984       ??_C@_0BA@FFLB@EV_GIB_NOBLOOD?6?$AA@ 3003f984     cg_event.obj
 0002:00001994       ??_C@_0P@EPLO@EV_GIB_PLAYER?6?$AA@ 3003f994     cg_event.obj
 0002:000019a4       ??_C@_0BC@BBCM@EV_POWERUP_REGEN?6?$AA@ 3003f9a4     cg_event.obj
 0002:000019b8       ??_C@_0BJ@HHNN@sound?1items?1protect3?4wav?$AA@ 3003f9b8     cg_event.obj
 0002:000019d4       ??_C@_0BH@BDJM@EV_POWERUP_BATTLESUIT?6?$AA@ 3003f9d4     cg_event.obj
 0002:000019ec       ??_C@_0BB@PKNK@EV_POWERUP_QUAD?6?$AA@ 3003f9ec     cg_event.obj
 0002:00001a00       ??_C@_0N@POFK@EV_OBITUARY?6?$AA@ 3003fa00     cg_event.obj
 0002:00001a10       ??_C@_0N@ELAE@?$CKdeath?$CFi?4wav?$AA@ 3003fa10     cg_event.obj
 0002:00001a20       ??_C@_0L@HGJI@EV_DEATHx?6?$AA@ 3003fa20     cg_event.obj
 0002:00001a2c       ??_C@_08OLFD@EV_PAIN?6?$AA@ 3003fa2c     cg_event.obj
 0002:00001a38       __real@4@40068000000000000000 3003fa38     cg_event.obj
 0002:00001a40       __real@8@40028000000000000000 3003fa40     cg_event.obj
 0002:00001a48       ??_C@_0BB@PNKO@EV_GLOBAL_SOUND?6?$AA@ 3003fa48     cg_event.obj
 0002:00001a5c       ??_C@_0BC@HLGB@EV_GENERAL_SOUND?6?$AA@ 3003fa5c     cg_event.obj
 0002:00001a70       ??_C@_0M@HLGC@EV_SHOTGUN?6?$AA@ 3003fa70     cg_event.obj
 0002:00001a7c       ??_C@_0BG@BLKG@EV_BULLET_HIT_CORPSE?6?$AA@ 3003fa7c     cg_event.obj
 0002:00001a94       ??_C@_0BF@KHP@EV_BULLET_HIT_FLESH?6?$AA@ 3003fa94     cg_event.obj
 0002:00001aac       ??_C@_0BE@FNME@EV_BULLET_HIT_WALL?6?$AA@ 3003faac     cg_event.obj
 0002:00001ac0       ??_C@_0BF@GAPO@EV_BULLET_HIT_ROBOT?6?$AA@ 3003fac0     cg_event.obj
 0002:00001ad8       ??_C@_0O@DKMH@EV_RAILTRAIL?6?$AA@ 3003fad8     cg_event.obj
 0002:00001ae8       ??_C@_0BB@IMB@EV_MISSILE_MISS?6?$AA@ 3003fae8     cg_event.obj
 0002:00001afc       ??_C@_0BA@HEPK@EV_MISSILE_HIT?6?$AA@ 3003fafc     cg_event.obj
 0002:00001b0c       ??_C@_0CD@KOIH@sound?1weapons?1grenade?1hgrenb2a?4w@ 3003fb0c     cg_event.obj
 0002:00001b30       ??_C@_0CD@BAGH@sound?1weapons?1grenade?1hgrenb1a?4w@ 3003fb30     cg_event.obj
 0002:00001b54       ??_C@_0BD@GMFL@EV_GRENADE_BOUNCE?6?$AA@ 3003fb54     cg_event.obj
 0002:00001b68       ??_C@_0BB@KAJM@EV_ITEM_RESPAWN?6?$AA@ 3003fb68     cg_event.obj
 0002:00001b7c       ??_C@_0N@NEMC@EV_ITEM_POP?6?$AA@ 3003fb7c     cg_event.obj
 0002:00001b8c       ??_C@_0BI@LJLH@EV_PLAYER_TELEPORT_OUT?6?$AA@ 3003fb8c     cg_event.obj
 0002:00001ba4       ??_C@_0BH@IOAG@EV_PLAYER_TELEPORT_IN?6?$AA@ 3003fba4     cg_event.obj
 0002:00001bbc       ??_C@_0P@ECMN@EV_USE_ITEM14?6?$AA@ 3003fbbc     cg_event.obj
 0002:00001bcc       ??_C@_0P@CDJI@EV_USE_ITEM13?6?$AA@ 3003fbcc     cg_event.obj
 0002:00001bdc       ??_C@_0P@DFDC@EV_USE_ITEM12?6?$AA@ 3003fbdc     cg_event.obj
 0002:00001bec       ??_C@_0P@OMN@EV_USE_ITEM11?6?$AA@ 3003fbec     cg_event.obj
 0002:00001bfc       ??_C@_0P@BIGH@EV_USE_ITEM10?6?$AA@ 3003fbfc     cg_event.obj
 0002:00001c0c       ??_C@_0O@LOAA@EV_USE_ITEM9?6?$AA@ 3003fc0c     cg_event.obj
 0002:00001c1c       ??_C@_0O@KIKK@EV_USE_ITEM8?6?$AA@ 3003fc1c     cg_event.obj
 0002:00001c2c       ??_C@_0O@HMKL@EV_USE_ITEM7?6?$AA@ 3003fc2c     cg_event.obj
 0002:00001c3c       ??_C@_0O@GKAB@EV_USE_ITEM6?6?$AA@ 3003fc3c     cg_event.obj
 0002:00001c4c       ??_C@_0O@FBPO@EV_USE_ITEM5?6?$AA@ 3003fc4c     cg_event.obj
 0002:00001c5c       ??_C@_0O@EHFE@EV_USE_ITEM4?6?$AA@ 3003fc5c     cg_event.obj
 0002:00001c6c       ??_C@_0O@CGAB@EV_USE_ITEM3?6?$AA@ 3003fc6c     cg_event.obj
 0002:00001c7c       ??_C@_0O@DAKL@EV_USE_ITEM2?6?$AA@ 3003fc7c     cg_event.obj
 0002:00001c8c       ??_C@_0O@LFE@EV_USE_ITEM1?6?$AA@ 3003fc8c     cg_event.obj
 0002:00001c9c       ??_C@_0O@BNPO@EV_USE_ITEM0?6?$AA@ 3003fc9c     cg_event.obj
 0002:00001cac       ??_C@_0BA@PFOI@EV_FIRE_WEAPON?6?$AA@ 3003fcac     cg_event.obj
 0002:00001cbc       ??_C@_0BC@JHHM@EV_CHANGE_WEAPON?6?$AA@ 3003fcbc     cg_event.obj
 0002:00001cd0       ??_C@_0L@EHFO@EV_NOAMMO?6?$AA@ 3003fcd0     cg_event.obj
 0002:00001cdc       ??_C@_0BH@CNCH@EV_GLOBAL_ITEM_PICKUP?6?$AA@ 3003fcdc     cg_event.obj
 0002:00001cf4       ??_C@_0BA@LJKF@EV_ITEM_PICKUP?6?$AA@ 3003fcf4     cg_event.obj
 0002:00001d04       ??_C@_09IIFC@?$CKgasp?4wav?$AA@ 3003fd04     cg_event.obj
 0002:00001d10       ??_C@_0BA@CPOA@EV_WATER_CLEAR?6?$AA@ 3003fd10     cg_event.obj
 0002:00001d20       ??_C@_0BA@CFGA@EV_WATER_UNDER?6?$AA@ 3003fd20     cg_event.obj
 0002:00001d30       ??_C@_0BA@MKDB@EV_WATER_LEAVE?6?$AA@ 3003fd30     cg_event.obj
 0002:00001d40       ??_C@_0BA@HOEJ@EV_WATER_TOUCH?6?$AA@ 3003fd40     cg_event.obj
 0002:00001d50       ??_C@_0L@GPKI@?$CKtaunt?4wav?$AA@ 3003fd50     cg_event.obj
 0002:00001d5c       ??_C@_09IPKD@EV_TAUNT?6?$AA@ 3003fd5c     cg_event.obj
 0002:00001d68       ??_C@_08IIFH@EV_JUMP?6?$AA@ 3003fd68     cg_event.obj
 0002:00001d74       ??_C@_0L@EIFI@?$CKjump1?4wav?$AA@ 3003fd74     cg_event.obj
 0002:00001d80       ??_C@_0N@NGHL@EV_JUMP_PAD?6?$AA@ 3003fd80     cg_event.obj
 0002:00001d90       __real@4@40048000000000000000 3003fd90     cg_event.obj
 0002:00001d94       ??_C@_08JOOK@EV_STEP?6?$AA@ 3003fd94     cg_event.obj
 0002:00001da0       ??_C@_0L@HOHM@?$CKfall1?4wav?$AA@ 3003fda0     cg_event.obj
 0002:00001dac       ??_C@_0N@HHME@EV_FALL_FAR?6?$AA@ 3003fdac     cg_event.obj
 0002:00001dbc       ??_C@_0BA@EHKG@EV_FALL_MEDIUM?6?$AA@ 3003fdbc     cg_event.obj
 0002:00001dcc       ??_C@_0P@HPFI@EV_FALL_SHORT?6?$AA@ 3003fdcc     cg_event.obj
 0002:00001ddc       ??_C@_08LKAO@EV_SWIM?6?$AA@ 3003fddc     cg_event.obj
 0002:00001de8       ??_C@_0N@OIMO@EV_FOOTWADE?6?$AA@ 3003fde8     cg_event.obj
 0002:00001df8       ??_C@_0P@HGDB@EV_FOOTSPLASH?6?$AA@ 3003fdf8     cg_event.obj
 0002:00001e08       ??_C@_0BD@OBHC@EV_FOOTSTEP_METAL?6?$AA@ 3003fe08     cg_event.obj
 0002:00001e1c       ??_C@_0N@PJNP@EV_FOOTSTEP?6?$AA@ 3003fe1c     cg_event.obj
 0002:00001e2c       ??_C@_0L@NDEP@ZEROEVENT?6?$AA@ 3003fe2c     cg_event.obj
 0002:00001e38       ??_C@_0BE@MLMA@ent?3?$CF3i?5?5event?3?$CF3i?5?$AA@ 3003fe38     cg_event.obj
 0002:00001e4c       ??_C@_09PFNP@?$CFs?5died?4?6?$AA@ 3003fe4c     cg_event.obj
 0002:00001e58       ??_C@_0M@JPCK@?$CFs?5?$CFs?5?$CFs?$CFs?6?$AA@ 3003fe58     cg_event.obj
 0002:00001e64       ??_C@_0O@BPF@was?5killed?5by?$AA@ 3003fe64     cg_event.obj
 0002:00001e74       ??_C@_09PFNJ@?8s?5attack?$AA@ 3003fe74     cg_event.obj
 0002:00001e80       ??_C@_0BL@OPJB@finally?5bled?5to?5death?5from?$AA@ 3003fe80     cg_event.obj
 0002:00001e9c       ??_C@_0BC@EAHL@?8s?5personal?5space?$AA@ 3003fe9c     cg_event.obj
 0002:00001eb0       ??_C@_0BA@BOPB@tried?5to?5invade?$AA@ 3003feb0     cg_event.obj
 0002:00001ec0       ??_C@_06BFBK@?8s?5BFG?$AA@ 3003fec0     cg_event.obj
 0002:00001ec8       ??_C@_0P@PJPG@was?5blasted?5by?$AA@ 3003fec8     cg_event.obj
 0002:00001ed8       ??_C@_0BE@LNLI@was?5electrocuted?5by?$AA@ 3003fed8     cg_event.obj
 0002:00001eec       ??_C@_0O@CAMJ@was?5railed?5by?$AA@ 3003feec     cg_event.obj
 0002:00001efc       ??_C@_0N@FLCB@?8s?5plasmagun?$AA@ 3003fefc     cg_event.obj
 0002:00001f0c       ??_C@_0O@BKII@was?5melted?5by?$AA@ 3003ff0c     cg_event.obj
 0002:00001f1c       ??_C@_0O@FKJL@almost?5dodged?$AA@ 3003ff1c     cg_event.obj
 0002:00001f2c       ??_C@_09LGPO@?8s?5rocket?$AA@ 3003ff2c     cg_event.obj
 0002:00001f38       ??_C@_0M@JEIL@?8s?5shrapnel?$AA@ 3003ff38     cg_event.obj
 0002:00001f44       ??_C@_0BA@LEDP@was?5shredded?5by?$AA@ 3003ff44     cg_event.obj
 0002:00001f54       ??_C@_0L@JJNB@?8s?5grenade?$AA@ 3003ff54     cg_event.obj
 0002:00001f60       ??_C@_03CNHG@ate?$AA@      3003ff60     cg_event.obj
 0002:00001f64       ??_C@_0BD@BGJE@was?5gunned?5down?5by?$AA@ 3003ff64     cg_event.obj
 0002:00001f78       ??_C@_0BF@PMCN@was?5machinegunned?5by?$AA@ 3003ff78     cg_event.obj
 0002:00001f90       ??_C@_0BA@CIJ@was?5pummeled?5by?$AA@ 3003ff90     cg_event.obj
 0002:00001fa0       ??_C@_0O@IGPI@was?5caught?5by?$AA@ 3003ffa0     cg_event.obj
 0002:00001fb0       ??_C@_06IPHI@noname?$AA@   3003ffb0     cg_event.obj
 0002:00001fb8       ??_C@_0P@MJDJ@You?5fragged?5?$CFs?$AA@ 3003ffb8     cg_event.obj
 0002:00001fc8       ??_C@_0CA@LJDA@You?5fragged?5?$CFs?6?$CFs?5place?5with?5?$CFi?$AA@ 3003ffc8     cg_event.obj
 0002:00001fe8       ??_C@_07GGCL@?$CFs?5?$CFs?4?6?$AA@ 3003ffe8     cg_event.obj
 0002:00001ff0       ??_C@_0P@GGKD@killed?5himself?$AA@ 3003fff0     cg_event.obj
 0002:00002000       ??_C@_0O@IICO@killed?5itself?$AA@ 30040000     cg_event.obj
 0002:00002010       ??_C@_0P@POKH@killed?5herself?$AA@ 30040010     cg_event.obj
 0002:00002020       ??_C@_0BP@OCJB@died?5of?5a?5sucking?5chest?5wound?4?$AA@ 30040020     cg_event.obj
 0002:00002040       ??_C@_0BP@NJLA@should?5have?5used?5a?5smaller?5gun?$AA@ 30040040     cg_event.obj
 0002:00002060       ??_C@_0P@JFBO@melted?5himself?$AA@ 30040060     cg_event.obj
 0002:00002070       ??_C@_0O@DFIK@melted?5itself?$AA@ 30040070     cg_event.obj
 0002:00002080       ??_C@_0P@NBK@melted?5herself?$AA@ 30040080     cg_event.obj
 0002:00002090       ??_C@_0BA@IPDB@blew?5himself?5up?$AA@ 30040090     cg_event.obj
 0002:000020a0       ??_C@_0P@HBOM@blew?5itself?5up?$AA@ 300400a0     cg_event.obj
 0002:000020b0       ??_C@_0BA@KPAE@blew?5herself?5up?$AA@ 300400b0     cg_event.obj
 0002:000020c0       ??_C@_0BL@HMJI@tripped?5on?5his?5own?5grenade?$AA@ 300400c0     cg_event.obj
 0002:000020dc       ??_C@_0BL@JILB@tripped?5on?5its?5own?5grenade?$AA@ 300400dc     cg_event.obj
 0002:000020f8       ??_C@_0BL@KODL@tripped?5on?5her?5own?5grenade?$AA@ 300400f8     cg_event.obj
 0002:00002114       ??_C@_0BO@LLHB@died?5of?5a?5sucking?5chest?5wound?$AA@ 30040114     cg_event.obj
 0002:00002134       ??_C@_0BH@BPGN@was?5in?5the?5wrong?5place?$AA@ 30040134     cg_event.obj
 0002:0000214c       ??_C@_0O@NKOE@saw?5the?5light?$AA@ 3004014c     cg_event.obj
 0002:0000215c       ??_C@_0BP@CFPL@does?5a?5back?5flip?5into?5the?5lava?$AA@ 3004015c     cg_event.obj
 0002:0000217c       ??_C@_06BOLJ@melted?$AA@   3004017c     cg_event.obj
 0002:00002184       ??_C@_0BB@PFDP@sank?5like?5a?5rock?$AA@ 30040184     cg_event.obj
 0002:00002198       ??_C@_0N@NNIF@was?5squished?$AA@ 30040198     cg_event.obj
 0002:000021a8       ??_C@_08LBFE@cratered?$AA@ 300401a8     cg_event.obj
 0002:000021b4       ??_C@_08LLKL@suicides?$AA@ 300401b4     cg_event.obj
 0002:000021c0       ??_C@_02KMNC@?$FO7?$AA@    300401c0     cg_event.obj
 0002:000021c4       ??_C@_0CB@KOEE@CG_Obituary?3?5target?5out?5of?5range@ 300401c4     cg_event.obj
 0002:000021e8       ??_C@_06CKFM@Use?5?$CFs?$AA@ 300401e8     cg_event.obj
 0002:000021f0       ??_C@_0P@HAHF@No?5item?5to?5use?$AA@ 300401f0     cg_event.obj
 0002:00002200       ??_C@_0BN@DNDF@sound?1player?1announce?1?$CFs?4wav?$AA@ 30040200     cg_info.obj
 0002:00002220       ??_C@_0BO@BKAG@models?1players?1?$CFs?1icon_?$CFs?4tga?$AA@ 30040220     cg_info.obj
 0002:00002240       ??_C@_07FMEP@default?$AA@  30040240     cg_info.obj
 0002:00002248       ??_C@_05LHJL@model?$AA@    30040248     cg_info.obj
 0002:00002250       ??_C@_0BA@JKMP@capturelimit?5?$CFi?$AA@ 30040250     cg_info.obj
 0002:00002260       ??_C@_0N@ELFE@capturelimit?$AA@ 30040260     cg_info.obj
 0002:00002270       ??_C@_0N@IHCP@fraglimit?5?$CFi?$AA@ 30040270     cg_info.obj
 0002:00002280       ??_C@_09DPJO@fraglimit?$AA@ 30040280     cg_info.obj
 0002:0000228c       ??_C@_0N@IEML@timelimit?5?$CFi?$AA@ 3004028c     cg_info.obj
 0002:0000229c       ??_C@_09GBNJ@timelimit?$AA@ 3004029c     cg_info.obj
 0002:000022a8       ??_C@_0BB@POJO@Unknown?5Gametype?$AA@ 300402a8     cg_info.obj
 0002:000022bc       ??_C@_0BB@EBBK@Capture?5The?5Flag?$AA@ 300402bc     cg_info.obj
 0002:000022d0       ??_C@_0L@MDJG@Tournament?$AA@ 300402d0     cg_info.obj
 0002:000022dc       ??_C@_0O@IEE@Single?5Player?$AA@ 300402dc     cg_info.obj
 0002:000022ec       ??_C@_0BD@EJEG@CHEATS?5ARE?5ENABLED?$AA@ 300402ec     cg_info.obj
 0002:00002300       ??_C@_09CPMK@sv_cheats?$AA@ 30040300     cg_info.obj
 0002:0000230c       ??_C@_0M@PCHP@Pure?5Server?$AA@ 3004030c     cg_info.obj
 0002:00002318       ??_C@_07OEHJ@sv_pure?$AA@  30040318     cg_info.obj
 0002:00002320       ??_C@_0M@IHPH@sv_hostname?$AA@ 30040320     cg_info.obj
 0002:0000232c       ??_C@_0L@HNAD@sv_running?$AA@ 3004032c     cg_info.obj
 0002:00002338       ??_C@_0BF@PPE@Awaiting?5snapshot?4?4?4?$AA@ 30040338     cg_info.obj
 0002:00002350       ??_C@_0O@NNNJ@Loading?4?4?4?5?$CFs?$AA@ 30040350     cg_info.obj
 0002:00002360       ??_C@_0BA@OBBJ@levelShotDetail?$AA@ 30040360     cg_info.obj
 0002:00002370       ??_C@_0BE@GNPF@menu?1art?1unknownmap?$AA@ 30040370     cg_info.obj
 0002:00002384       ??_C@_0BC@PKPD@levelshots?1?$CFs?4tga?$AA@ 30040384     cg_info.obj
 0002:00002398       ??_C@_07DOCO@mapname?$AA@  30040398     cg_info.obj
 0002:000023a0       ??_C@_0BP@IMDD@CG_FreeLocalEntity?3?5not?5active?$AA@ 300403a0     cg_localents.obj
 0002:000023c0       __real@4@c0008000000000000000 300403c0     cg_localents.obj
 0002:000023c8       __real@8@40038000000000000000 300403c8     cg_localents.obj
 0002:000023d0       __real@8@3ffcccccccccccccd000 300403d0     cg_localents.obj
 0002:000023d8       __real@8@3ff7f5c28f5c28f5c000 300403d8     cg_localents.obj
 0002:000023e0       ??_C@_0P@IAID@Bad?5leType?3?5?$CFi?$AA@ 300403e0     cg_localents.obj
 0002:000023f0       __real@4@c0018000000000000000 300403f0     cg_localents.obj
 0002:000023f8       __real@8@4004a800000000000000 300403f8     cg_localents.obj
 0002:00002400       __real@8@3ffda8f5c28f5c28f800 30040400     cg_localents.obj
 0002:00002408       ??_C@_0BJ@GGEM@gfx?12d?1numbers?1minus_32b?$AA@ 30040408     cg_main.obj
 0002:00002424       ??_C@_0BI@IIHO@gfx?12d?1numbers?1nine_32b?$AA@ 30040424     cg_main.obj
 0002:0000243c       ??_C@_0BJ@HKOM@gfx?12d?1numbers?1eight_32b?$AA@ 3004043c     cg_main.obj
 0002:00002458       ??_C@_0BJ@FIML@gfx?12d?1numbers?1seven_32b?$AA@ 30040458     cg_main.obj
 0002:00002474       ??_C@_0BH@CBJN@gfx?12d?1numbers?1six_32b?$AA@ 30040474     cg_main.obj
 0002:0000248c       ??_C@_0BI@DOAJ@gfx?12d?1numbers?1five_32b?$AA@ 3004048c     cg_main.obj
 0002:000024a4       ??_C@_0BI@FDL@gfx?12d?1numbers?1four_32b?$AA@ 300404a4     cg_main.obj
 0002:000024bc       ??_C@_0BJ@GFMA@gfx?12d?1numbers?1three_32b?$AA@ 300404bc     cg_main.obj
 0002:000024d8       ??_C@_0BH@BJ@gfx?12d?1numbers?1two_32b?$AA@ 300404d8     cg_main.obj
 0002:000024f0       ??_C@_0BH@MNJD@gfx?12d?1numbers?1one_32b?$AA@ 300404f0     cg_main.obj
 0002:00002508       ??_C@_0BI@EDF@gfx?12d?1numbers?1zero_32b?$AA@ 30040508     cg_main.obj
 0002:00002520       ??_C@_0BE@CFBM@g_syncronousClients?$AA@ 30040520     cg_main.obj
 0002:00002534       ??_C@_09NJEO@com_blood?$AA@ 30040534     cg_main.obj
 0002:00002540       ??_C@_09ENJF@cl_paused?$AA@ 30040540     cg_main.obj
 0002:0000254c       ??_C@_0BA@ELKM@com_buildScript?$AA@ 3004054c     cg_main.obj
 0002:0000255c       ??_C@_0L@DPIB@cl_autoaim?$AA@ 3004055c     cg_main.obj
 0002:00002568       ??_C@_02CKLK@32?$AA@       30040568     cg_main.obj
 0002:0000256c       ??_C@_0BE@KOOF@r_railSegmentLength?$AA@ 3004056c     cg_main.obj
 0002:00002580       ??_C@_02KNLD@16?$AA@       30040580     cg_main.obj
 0002:00002584       ??_C@_0M@JMJK@r_railWidth?$AA@ 30040584     cg_main.obj
 0002:00002590       ??_C@_0BH@LJNK@cg_sphericalExplosions?$AA@ 30040590     cg_main.obj
 0002:000025a8       ??_C@_0P@ICLM@cg_coolRailGun?$AA@ 300405a8     cg_main.obj
 0002:000025b8       ??_C@_0M@HPF@g_HeadScale?$AA@ 300405b8     cg_main.obj
 0002:000025c4       ??_C@_03DJMC@150?$AA@      300405c4     cg_main.obj
 0002:000025c8       ??_C@_0BA@CDBJ@cg_ScaleWeapons?$AA@ 300405c8     cg_main.obj
 0002:000025d8       ??_C@_0M@ELJM@cg_BobItems?$AA@ 300405d8     cg_main.obj
 0002:000025e4       ??_C@_08LFEE@cg_stats?$AA@ 300405e4     cg_main.obj
 0002:000025f0       ??_C@_0M@FNOC@teamoverlay?$AA@ 300405f0     cg_main.obj
 0002:000025fc       ??_C@_0BD@HGHB@cg_drawTeamOverlay?$AA@ 300405fc     cg_main.obj
 0002:00002610       ??_C@_0BA@HEHH@cg_deferPlayers?$AA@ 30040610     cg_main.obj
 0002:00002620       ??_C@_0BA@PHDH@cg_predictItems?$AA@ 30040620     cg_main.obj
 0002:00002630       ??_C@_0O@JDJH@cg_forceModel?$AA@ 30040630     cg_main.obj
 0002:00002640       ??_C@_0BC@MGOP@cg_teamChatHeight?$AA@ 30040640     cg_main.obj
 0002:00002654       ??_C@_04LHEB@3000?$AA@     30040654     cg_main.obj
 0002:0000265c       ??_C@_0BA@NLMO@cg_teamChatTime?$AA@ 3004065c     cg_main.obj
 0002:0000266c       ??_C@_0P@LBPA@cg_thirdPerson?$AA@ 3004066c     cg_main.obj
 0002:0000267c       ??_C@_0BE@BKEC@cg_thirdPersonAngle?$AA@ 3004067c     cg_main.obj
 0002:00002690       ??_C@_02BOMB@40?$AA@       30040690     cg_main.obj
 0002:00002694       ??_C@_0BE@GEFO@cg_thirdPersonRange?$AA@ 30040694     cg_main.obj
 0002:000026a8       ??_C@_0BA@LOGF@cg_tracerlength?$AA@ 300406a8     cg_main.obj
 0002:000026b8       ??_C@_0P@JDDG@cg_tracerwidth?$AA@ 300406b8     cg_main.obj
 0002:000026c8       ??_C@_0BA@JHJM@cg_tracerchance?$AA@ 300406c8     cg_main.obj
 0002:000026d8       ??_C@_0N@IIAN@cg_footsteps?$AA@ 300406d8     cg_main.obj
 0002:000026e8       ??_C@_0M@MOEE@cg_showmiss?$AA@ 300406e8     cg_main.obj
 0002:000026f4       ??_C@_0BB@BPFD@cg_noplayeranims?$AA@ 300406f4     cg_main.obj
 0002:00002708       ??_C@_0N@PIGE@cg_nopredict?$AA@ 30040708     cg_main.obj
 0002:00002718       ??_C@_0O@KAC@cg_errordecay?$AA@ 30040718     cg_main.obj
 0002:00002728       ??_C@_0P@NKCK@cg_debugevents?$AA@ 30040728     cg_main.obj
 0002:00002738       ??_C@_0BB@CONE@cg_debugposition?$AA@ 30040738     cg_main.obj
 0002:0000274c       ??_C@_0N@GCOC@cg_debuganim?$AA@ 3004074c     cg_main.obj
 0002:0000275c       ??_C@_0N@EFHB@cg_animspeed?$AA@ 3004075c     cg_main.obj
 0002:0000276c       ??_C@_03HAGP@0?43?$AA@     3004076c     cg_main.obj
 0002:00002770       ??_C@_0O@HJHK@cg_swingSpeed?$AA@ 30040770     cg_main.obj
 0002:00002780       ??_C@_0L@FDJB@cg_bobroll?$AA@ 30040780     cg_main.obj
 0002:0000278c       ??_C@_0M@JFLD@cg_bobpitch?$AA@ 3004078c     cg_main.obj
 0002:00002798       ??_C@_08BIFL@cg_bobup?$AA@ 30040798     cg_main.obj
 0002:000027a4       ??_C@_05HONO@0?4005?$AA@   300407a4     cg_main.obj
 0002:000027ac       ??_C@_0L@OHDH@cg_runroll?$AA@ 300407ac     cg_main.obj
 0002:000027b8       ??_C@_05CLDL@0?4002?$AA@   300407b8     cg_main.obj
 0002:000027c0       ??_C@_0M@CMAH@cg_runpitch?$AA@ 300407c0     cg_main.obj
 0002:000027cc       ??_C@_01ECJ@3?$AA@         300407cc     cg_main.obj
 0002:000027d0       ??_C@_0O@MAPC@cg_centertime?$AA@ 300407d0     cg_main.obj
 0002:000027e0       ??_C@_07BCIE@cg_gunZ?$AA@  300407e0     cg_main.obj
 0002:000027e8       ??_C@_07ONDN@cg_gunY?$AA@  300407e8     cg_main.obj
 0002:000027f0       ??_C@_07EHKK@cg_gunX?$AA@  300407f0     cg_main.obj
 0002:000027f8       ??_C@_03GPIO@400?$AA@      300407f8     cg_main.obj
 0002:000027fc       ??_C@_0BB@PGOB@cg_railTrailTime?$AA@ 300407fc     cg_main.obj
 0002:00002810       ??_C@_0N@JOJA@cg_lagometer?$AA@ 30040810     cg_main.obj
 0002:00002820       ??_C@_08PKCG@cg_marks?$AA@ 30040820     cg_main.obj
 0002:0000282c       ??_C@_0P@CMNJ@cg_simpleItems?$AA@ 3004082c     cg_main.obj
 0002:0000283c       ??_C@_04BFMI@1250?$AA@     3004083c     cg_main.obj
 0002:00002844       ??_C@_0N@OGMG@cg_brassTime?$AA@ 30040844     cg_main.obj
 0002:00002854       ??_C@_0O@BAFO@cg_crosshairY?$AA@ 30040854     cg_main.obj
 0002:00002864       ??_C@_0O@LKMJ@cg_crosshairX?$AA@ 30040864     cg_main.obj
 0002:00002874       ??_C@_0BD@DAFD@cg_crosshairHealth?$AA@ 30040874     cg_main.obj
 0002:00002888       ??_C@_02MDGC@24?$AA@       30040888     cg_main.obj
 0002:0000288c       ??_C@_0BB@OMED@cg_crosshairSize?$AA@ 3004088c     cg_main.obj
 0002:000028a0       ??_C@_0P@FGKI@cg_drawRewards?$AA@ 300408a0     cg_main.obj
 0002:000028b0       ??_C@_0BG@JAIH@cg_drawCrosshairNames?$AA@ 300408b0     cg_main.obj
 0002:000028c8       ??_C@_01FBMM@4?$AA@        300408c8     cg_main.obj
 0002:000028cc       ??_C@_0BB@BIJH@cg_drawCrosshair?$AA@ 300408cc     cg_main.obj
 0002:000028e0       ??_C@_0BA@GOGM@cg_drawAttacker?$AA@ 300408e0     cg_main.obj
 0002:000028f0       ??_C@_0BD@CH@cg_drawAmmoWarning?$AA@ 300408f0     cg_main.obj
 0002:00002904       ??_C@_0N@PODO@cg_drawIcons?$AA@ 30040904     cg_main.obj
 0002:00002914       ??_C@_0P@CEHN@cg_draw3dIcons?$AA@ 30040914     cg_main.obj
 0002:00002924       ??_C@_0BA@EDDP@cg_drawSnapshot?$AA@ 30040924     cg_main.obj
 0002:00002934       ??_C@_0L@PKAE@cg_drawFPS?$AA@ 30040934     cg_main.obj
 0002:00002940       ??_C@_0N@DNNE@cg_drawTimer?$AA@ 30040940     cg_main.obj
 0002:00002950       ??_C@_0O@FKIK@cg_drawStatus?$AA@ 30040950     cg_main.obj
 0002:00002960       ??_C@_09EBKA@cg_draw2D?$AA@ 30040960     cg_main.obj
 0002:0000296c       ??_C@_07KIDA@cg_gibs?$AA@  3004096c     cg_main.obj
 0002:00002974       ??_C@_0L@FKLD@cg_shadows?$AA@ 30040974     cg_main.obj
 0002:00002980       ??_C@_03CFIK@0?44?$AA@     30040980     cg_main.obj
 0002:00002984       ??_C@_0BE@GEEB@cg_stereoSeparation?$AA@ 30040984     cg_main.obj
 0002:00002998       ??_C@_03HFMC@100?$AA@      30040998     cg_main.obj
 0002:0000299c       ??_C@_02OHJF@90?$AA@       3004099c     cg_main.obj
 0002:000029a0       ??_C@_06PPLP@cg_fov?$AA@   300409a0     cg_main.obj
 0002:000029a8       ??_C@_04JOPH@22?45?$AA@    300409a8     cg_main.obj
 0002:000029b0       ??_C@_0L@DLEJ@cg_zoomfov?$AA@ 300409b0     cg_main.obj
 0002:000029bc       ??_C@_0L@JOKD@cg_drawGun?$AA@ 300409bc     cg_main.obj
 0002:000029c8       ??_C@_01FBAH@1?$AA@        300409c8     cg_main.obj
 0002:000029cc       ??_C@_0O@LDOP@cg_autoswitch?$AA@ 300409cc     cg_main.obj
 0002:000029dc       ??_C@_01PLJA@0?$AA@        300409dc     cg_main.obj
 0002:000029e0       ??_C@_09DOEH@cg_ignore?$AA@ 300409e0     cg_main.obj
 0002:000029ec       ??_C@_0BL@KEBB@vmMain?3?5unknown?5command?5?$CFi?$AA@ 300409ec     cg_main.obj
 0002:00002a08       ??_C@_02DILL@?$CFs?$AA@    30040a08     cg_main.obj
 0002:00002a0c       ??_C@_0BP@LEPA@CG_ConfigString?3?5bad?5index?3?5?$CFi?$AA@ 30040a0c     cg_main.obj
 0002:00002a2c       ??_C@_0DG@OFDD@Check?5out?5our?5website?5at?5http?3?1?1@ 30040a2c     cg_main.obj
 0002:00002a64       ??_C@_0CG@LPBB@Welcome?5to?5Q3A?5Viz?5v1?41?40?0?5by?5He@ 30040a64     cg_main.obj
 0002:00002a8c       ??_C@_06HADE@sounds?$AA@   30040a8c     cg_main.obj
 0002:00002a94       ??_C@_0O@JOGL@collision?5map?$AA@ 30040a94     cg_main.obj
 0002:00002aa4       ??_C@_0CD@MNBB@Client?1Server?5game?5mismatch?3?5?$CFs?1@ 30040aa4     cg_main.obj
 0002:00002ac8       ??_C@_09LPNC@Viz?51?43?45?$AA@ 30040ac8     cg_main.obj
 0002:00002ad8       __real@8@4007f000000000000000 30040ad8     cg_main.obj
 0002:00002ae0       __real@8@4008a000000000000000 30040ae0     cg_main.obj
 0002:00002ae8       ??_C@_0BI@GNCN@menu?1art?1font2_prop?4tga?$AA@ 30040ae8     cg_main.obj
 0002:00002b00       ??_C@_0BM@LJCL@menu?1art?1font1_prop_glo?4tga?$AA@ 30040b00     cg_main.obj
 0002:00002b1c       ??_C@_0BI@PNGL@menu?1art?1font1_prop?4tga?$AA@ 30040b1c     cg_main.obj
 0002:00002b34       ??_C@_05GMF@white?$AA@     30040b34     cg_main.obj
 0002:00002b3c       ??_C@_0BA@OLJD@gfx?12d?1bigchars?$AA@ 30040b3c     cg_main.obj
 0002:00002b4c       ??_C@_0CC@LDHC@sound?1weapons?1plasma?1plasmx1a?4wa@ 30040b4c     cg_main.obj
 0002:00002b70       ??_C@_0CC@DPBF@sound?1weapons?1rocket?1rocklx1a?4wa@ 30040b70     cg_main.obj
 0002:00002b94       ??_C@_0CD@DKPN@sound?1weapons?1railgun?1railgf1a?4w@ 30040b94     cg_main.obj
 0002:00002bb8       ??_C@_0CC@NBBC@sound?1weapons?1machinegun?1ric3?4wa@ 30040bb8     cg_main.obj
 0002:00002bdc       ??_C@_0CC@HBDH@sound?1weapons?1machinegun?1ric2?4wa@ 30040bdc     cg_main.obj
 0002:00002c00       ??_C@_0CC@JBFI@sound?1weapons?1machinegun?1ric1?4wa@ 30040c00     cg_main.obj
 0002:00002c24       ??_C@_0BI@PONI@sound?1items?1damage3?4wav?$AA@ 30040c24     cg_main.obj
 0002:00002c3c       ??_C@_0CD@LJPM@sound?1player?1footsteps?1clank?$CFi?4w@ 30040c3c     cg_main.obj
 0002:00002c60       ??_C@_0CE@MLNE@sound?1player?1footsteps?1splash?$CFi?4@ 30040c60     cg_main.obj
 0002:00002c84       ??_C@_0CE@MLH@sound?1player?1footsteps?1energy?$CFi?4@ 30040c84     cg_main.obj
 0002:00002ca8       ??_C@_0CC@DOOK@sound?1player?1footsteps?1mech?$CFi?4wa@ 30040ca8     cg_main.obj
 0002:00002ccc       ??_C@_0CD@CINL@sound?1player?1footsteps?1flesh?$CFi?4w@ 30040ccc     cg_main.obj
 0002:00002cf0       ??_C@_0CC@DPAJ@sound?1player?1footsteps?1boot?$CFi?4wa@ 30040cf0     cg_main.obj
 0002:00002d14       ??_C@_0CC@FHIL@sound?1player?1footsteps?1step?$CFi?4wa@ 30040d14     cg_main.obj
 0002:00002d38       ??_C@_0BI@NOB@sound?1world?1jumppad?4wav?$AA@ 30040d38     cg_main.obj
 0002:00002d50       ??_C@_0BJ@CEFN@sound?1player?1watr_un?4wav?$AA@ 30040d50     cg_main.obj
 0002:00002d6c       ??_C@_0BK@IONP@sound?1player?1watr_out?4wav?$AA@ 30040d6c     cg_main.obj
 0002:00002d88       ??_C@_0BJ@IFNO@sound?1player?1watr_in?4wav?$AA@ 30040d88     cg_main.obj
 0002:00002da4       ??_C@_0BM@NEMN@sound?1feedback?1lostlead?4wav?$AA@ 30040da4     cg_main.obj
 0002:00002dc0       ??_C@_0BM@OCDK@sound?1feedback?1tiedlead?4wav?$AA@ 30040dc0     cg_main.obj
 0002:00002ddc       ??_C@_0BN@PKAH@sound?1feedback?1takenlead?4wav?$AA@ 30040ddc     cg_main.obj
 0002:00002dfc       ??_C@_0BP@FFCB@sound?1feedback?1humiliation?4wav?$AA@ 30040dfc     cg_main.obj
 0002:00002e1c       ??_C@_0BK@OBGG@sound?1feedback?1denied?4wav?$AA@ 30040e1c     cg_main.obj
 0002:00002e38       ??_C@_0BN@PGHI@sound?1feedback?1excellent?4wav?$AA@ 30040e38     cg_main.obj
 0002:00002e58       ??_C@_0BO@EDAB@sound?1feedback?1impressive?4wav?$AA@ 30040e58     cg_main.obj
 0002:00002e78       ??_C@_0BH@NKIK@sound?1feedback?1hit?4wav?$AA@ 30040e78     cg_main.obj
 0002:00002e90       ??_C@_0BH@OPKF@sound?1player?1land1?4wav?$AA@ 30040e90     cg_main.obj
 0002:00002ea8       ??_C@_0BG@MMD@sound?1player?1talk?4wav?$AA@ 30040ea8     cg_main.obj
 0002:00002ec0       ??_C@_0BJ@LMIL@sound?1weapons?1noammo?4wav?$AA@ 30040ec0     cg_main.obj
 0002:00002edc       ??_C@_0BJ@MKPL@sound?1items?1respawn1?4wav?$AA@ 30040edc     cg_main.obj
 0002:00002ef8       ??_C@_0BI@JK@sound?1world?1teleout?4wav?$AA@ 30040ef8     cg_main.obj
 0002:00002f10       ??_C@_0BH@MACJ@sound?1world?1telein?4wav?$AA@ 30040f10     cg_main.obj
 0002:00002f28       ??_C@_0BJ@MPBB@sound?1player?1gibimp3?4wav?$AA@ 30040f28     cg_main.obj
 0002:00002f44       ??_C@_0BJ@GPDE@sound?1player?1gibimp2?4wav?$AA@ 30040f44     cg_main.obj
 0002:00002f60       ??_C@_0BJ@IPFL@sound?1player?1gibimp1?4wav?$AA@ 30040f60     cg_main.obj
 0002:00002f7c       ??_C@_0BK@GJHN@sound?1player?1gibsplt1?4wav?$AA@ 30040f7c     cg_main.obj
 0002:00002f98       ??_C@_0BM@HEPC@sound?1items?1use_nothing?4wav?$AA@ 30040f98     cg_main.obj
 0002:00002fb4       ??_C@_0BI@PGLK@sound?1items?1wearoff?4wav?$AA@ 30040fb4     cg_main.obj
 0002:00002fcc       ??_C@_0BJ@IJDF@sound?1weapons?1change?4wav?$AA@ 30040fcc     cg_main.obj
 0002:00002fe8       ??_C@_0CG@LCFH@sound?1weapons?1machinegun?1buletby@ 30040fe8     cg_main.obj
 0002:00003010       ??_C@_0CA@BJLL@sound?1feedback?1hit_teammate?4wav?$AA@ 30041010     cg_main.obj
 0002:00003030       ??_C@_0BN@BEJD@sound?1feedback?1teamstied?4wav?$AA@ 30041030     cg_main.obj
 0002:00003050       ??_C@_0BN@KLBA@sound?1feedback?1blueleads?4wav?$AA@ 30041050     cg_main.obj
 0002:00003070       ??_C@_0BM@PPAE@sound?1feedback?1redleads?4wav?$AA@ 30041070     cg_main.obj
 0002:0000308c       ??_C@_0BL@GDED@sound?1feedback?1prepare?4wav?$AA@ 3004108c     cg_main.obj
 0002:000030a8       ??_C@_0BJ@HPLO@sound?1feedback?1fight?4wav?$AA@ 300410a8     cg_main.obj
 0002:000030c4       ??_C@_0BH@FJHC@sound?1feedback?1one?4wav?$AA@ 300410c4     cg_main.obj
 0002:000030dc       ??_C@_0BH@JEPI@sound?1feedback?1two?4wav?$AA@ 300410dc     cg_main.obj
 0002:000030f4       ??_C@_0BJ@CGEK@sound?1feedback?1three?4wav?$AA@ 300410f4     cg_main.obj
 0002:00003110       ??_C@_0BL@EEJO@sound?1feedback?13_frags?4wav?$AA@ 30041110     cg_main.obj
 0002:0000312c       ??_C@_0BL@KOBB@sound?1feedback?12_frags?4wav?$AA@ 3004112c     cg_main.obj
 0002:00003148       ??_C@_0BK@LPJP@sound?1feedback?11_frag?4wav?$AA@ 30041148     cg_main.obj
 0002:00003164       ??_C@_0CA@CIFA@sound?1feedback?1sudden_death?4wav?$AA@ 30041164     cg_main.obj
 0002:00003184       ??_C@_0BM@JEGM@sound?1feedback?15_minute?4wav?$AA@ 30041184     cg_main.obj
 0002:000031a0       ??_C@_0BM@CDMG@sound?1feedback?11_minute?4wav?$AA@ 300411a0     cg_main.obj
 0002:000031bc       ??_C@_03JAAL@wav?$AA@      300411bc     cg_main.obj
 0002:000031c0       ??_C@_0CJ@CCML@PrecacheItem?3?5?$CFs?5has?5bad?5precach@ 300411c0     cg_main.obj
 0002:000031ec       ??_C@_03OGBA@?$CK?$CFi?$AA@ 300411ec     cg_main.obj
 0002:000031f0       ??_C@_09NBPF@bloodMark?$AA@ 300411f0     cg_main.obj
 0002:000031fc       ??_C@_04MCIG@wake?$AA@     300411fc     cg_main.obj
 0002:00003204       ??_C@_0L@MHIE@markShadow?$AA@ 30041204     cg_main.obj
 0002:00003210       ??_C@_0BG@FAEE@gfx?1damage?1plasma_mrk?$AA@ 30041210     cg_main.obj
 0002:00003228       ??_C@_0BH@IEIN@gfx?1damage?1hole_lg_mrk?$AA@ 30041228     cg_main.obj
 0002:00003240       ??_C@_0BI@MJNK@gfx?1damage?1burn_med_mrk?$AA@ 30041240     cg_main.obj
 0002:00003258       ??_C@_0BG@LFHE@gfx?1damage?1bullet_mrk?$AA@ 30041258     cg_main.obj
 0002:00003270       ??_C@_0P@FFMN@medal_gauntlet?$AA@ 30041270     cg_main.obj
 0002:00003280       ??_C@_0BA@MJGL@medal_excellent?$AA@ 30041280     cg_main.obj
 0002:00003290       ??_C@_0BB@KJCG@medal_impressive?$AA@ 30041290     cg_main.obj
 0002:000032a4       ??_C@_0P@DFMD@teleportEffect?$AA@ 300412a4     cg_main.obj
 0002:000032b4       ??_C@_0BG@DGHM@models?1misc?1telep?4md3?$AA@ 300412b4     cg_main.obj
 0002:000032cc       ??_C@_0BC@GAAO@models?1sphere?4md3?$AA@ 300412cc     cg_main.obj
 0002:000032e0       ??_C@_0BL@MAGG@models?1weaphits?1ring02?4md3?$AA@ 300412e0     cg_main.obj
 0002:000032fc       ??_C@_0BL@KMEP@models?1weaphits?1bullet?4md3?$AA@ 300412fc     cg_main.obj
 0002:00003318       ??_C@_0O@BKJO@railExplosion?$AA@ 30041318     cg_main.obj
 0002:00003328       ??_C@_0P@DMIO@bloodExplosion?$AA@ 30041328     cg_main.obj
 0002:00003338       ??_C@_0BB@GJFJ@sprites?1balloon3?$AA@ 30041338     cg_main.obj
 0002:0000334c       ??_C@_0BG@GELG@models?1gibs?1brain?4md3?$AA@ 3004134c     cg_main.obj
 0002:00003364       ??_C@_0BG@NJKJ@models?1gibs?1skull?4md3?$AA@ 30041364     cg_main.obj
 0002:0000337c       ??_C@_0BE@GONB@models?1gibs?1leg?4md3?$AA@ 3004137c     cg_main.obj
 0002:00003390       ??_C@_0BK@IPCD@models?1gibs?1intestine?4md3?$AA@ 30041390     cg_main.obj
 0002:000033ac       ??_C@_0BI@HDBE@models?1gibs?1forearm?4md3?$AA@ 300413ac     cg_main.obj
 0002:000033c4       ??_C@_0BF@JIAB@models?1gibs?1foot?4md3?$AA@ 300413c4     cg_main.obj
 0002:000033dc       ??_C@_0BF@NOPP@models?1gibs?1fist?4md3?$AA@ 300413dc     cg_main.obj
 0002:000033f4       ??_C@_0BG@NABO@models?1gibs?1chest?4md3?$AA@ 300413f4     cg_main.obj
 0002:0000340c       ??_C@_0BE@HNLN@models?1gibs?1arm?4md3?$AA@ 3004140c     cg_main.obj
 0002:00003420       ??_C@_0BI@MMIP@models?1gibs?1abdomen?4md3?$AA@ 30041420     cg_main.obj
 0002:00003438       ??_C@_0CD@DFOI@models?1weapons2?1shells?1s_shell?4m@ 30041438     cg_main.obj
 0002:0000345c       ??_C@_0CD@LGEK@models?1weapons2?1shells?1m_shell?4m@ 3004145c     cg_main.obj
 0002:00003480       ??_C@_0BE@MFJI@gfx?12d?1colorbar?4tga?$AA@ 30041480     cg_main.obj
 0002:00003494       ??_C@_0BC@FIIO@powerups?1blueflag?$AA@ 30041494     cg_main.obj
 0002:000034a8       ??_C@_0M@DEOK@sprites?1foe?$AA@ 300414a8     cg_main.obj
 0002:000034b4       ??_C@_0BB@IOJF@icons?1iconf_blu3?$AA@ 300414b4     cg_main.obj
 0002:000034c8       ??_C@_0BB@CEAC@icons?1iconf_blu2?$AA@ 300414c8     cg_main.obj
 0002:000034dc       ??_C@_0BB@GFBE@icons?1iconf_red3?$AA@ 300414dc     cg_main.obj
 0002:000034f0       ??_C@_0BB@MPID@icons?1iconf_red2?$AA@ 300414f0     cg_main.obj
 0002:00003504       ??_C@_0BC@ONDP@models?1wings?4skin?$AA@ 30041504     cg_main.obj
 0002:00003518       ??_C@_0BP@EDDC@models?1players?1hunter?1head?4md3?$AA@ 30041518     cg_main.obj
 0002:00003538       ??_C@_0P@NOLD@hasteSmokePuff?$AA@ 30041538     cg_main.obj
 0002:00003548       ??_C@_0P@KCNN@powerups?1regen?$AA@ 30041548     cg_main.obj
 0002:00003558       ??_C@_0BG@DGGP@powerups?1invisibility?$AA@ 30041558     cg_main.obj
 0002:00003570       ??_C@_0BG@PEBI@powerups?1battleWeapon?$AA@ 30041570     cg_main.obj
 0002:00003588       ??_C@_0BE@EPKD@powerups?1battleSuit?$AA@ 30041588     cg_main.obj
 0002:0000359c       ??_C@_0BE@IADB@powerups?1quadWeapon?$AA@ 3004159c     cg_main.obj
 0002:000035b0       ??_C@_0O@KEKI@powerups?1quad?$AA@ 300415b0     cg_main.obj
 0002:000035c0       ??_C@_0N@CIJO@icons?1noammo?$AA@ 300415c0     cg_main.obj
 0002:000035d0       ??_C@_0BA@EMNI@gfx?12d?1backtile?$AA@ 300415d0     cg_main.obj
 0002:000035e0       ??_C@_0BD@LP@gfx?12d?1crosshair?$CFc?$AA@ 300415e0     cg_main.obj
 0002:000035f4       ??_C@_0O@NNHH@gfx?12d?1select?$AA@ 300415f4     cg_main.obj
 0002:00003604       ??_C@_0BA@EFC@gfx?1misc?1tracer?$AA@ 30041604     cg_main.obj
 0002:00003614       ??_C@_0M@MHCB@waterBubble?$AA@ 30041614     cg_main.obj
 0002:00003620       ??_C@_0N@OGHP@disconnected?$AA@ 30041620     cg_main.obj
 0002:00003630       ??_C@_09FFBB@lagometer?$AA@ 30041630     cg_main.obj
 0002:0000363c       ??_C@_0L@KJM@bloodTrail?$AA@ 3004163c     cg_main.obj
 0002:00003648       ??_C@_0BA@GFOI@sprites?1plasma1?$AA@ 30041648     cg_main.obj
 0002:00003658       ??_C@_0BB@PFF@shotgunSmokePuff?$AA@ 30041658     cg_main.obj
 0002:0000366c       ??_C@_0BB@MPIG@smokePuffRagePro?$AA@ 3004166c     cg_main.obj
 0002:00003680       ??_C@_09ELFP@smokePuff?$AA@ 30041680     cg_main.obj
 0002:0000368c       ??_C@_0BC@LCPM@menu?1tab?1time?4tga?$AA@ 3004168c     cg_main.obj
 0002:000036a0       ??_C@_0BD@GFLC@menu?1tab?1score?4tga?$AA@ 300416a0     cg_main.obj
 0002:000036b4       ??_C@_0BC@GMOM@menu?1tab?1ping?4tga?$AA@ 300416b4     cg_main.obj
 0002:000036c8       ??_C@_0BC@JFJB@menu?1tab?1name?4tga?$AA@ 300416c8     cg_main.obj
 0002:000036dc       ??_C@_0BB@NIJN@gfx?12d?1defer?4tga?$AA@ 300416dc     cg_main.obj
 0002:000036f0       ??_C@_0P@EJBO@viewBloodBlend?$AA@ 300416f0     cg_main.obj
 0002:00003700       ??_C@_0BE@HPMM@menu?1art?1skill5?4tga?$AA@ 30041700     cg_main.obj
 0002:00003714       ??_C@_0BE@NPOJ@menu?1art?1skill4?4tga?$AA@ 30041714     cg_main.obj
 0002:00003728       ??_C@_0BE@LPBD@menu?1art?1skill3?4tga?$AA@ 30041728     cg_main.obj
 0002:0000373c       ??_C@_0BE@BPDG@menu?1art?1skill2?4tga?$AA@ 3004173c     cg_main.obj
 0002:00003750       ??_C@_0BE@PPFJ@menu?1art?1skill1?4tga?$AA@ 30041750     cg_main.obj
 0002:00003764       ??_C@_0L@KCHM@game?5media?$AA@ 30041764     cg_main.obj
 0002:00003770       __real@4@c003a000000000000000 30041770     cg_marks.obj
 0002:00003774       ??_C@_0CG@DAAF@CG_ImpactMark?5called?5with?5?$DM?$DN?50?5r@ 30041774     cg_marks.obj
 0002:000037a0       __real@8@4007e100000000000000 300417a0     cg_marks.obj
 0002:000037a8       __real@8@400abb80000000000000 300417a8     cg_marks.obj
 0002:000037b0       ??_C@_0L@PAPK@?$CKdrown?4wav?$AA@ 300417b0     cg_players.obj
 0002:000037bc       ??_C@_0O@IAAP@?$CKfalling1?4wav?$AA@ 300417bc     cg_players.obj
 0002:000037cc       ??_C@_0M@MNAN@?$CKdeath3?4wav?$AA@ 300417cc     cg_players.obj
 0002:000037d8       ??_C@_0M@GNCI@?$CKdeath2?4wav?$AA@ 300417d8     cg_players.obj
 0002:000037e4       ??_C@_0M@INEH@?$CKdeath1?4wav?$AA@ 300417e4     cg_players.obj
 0002:000037f0       ??_C@_0BJ@IDLH@Unknown?5custom?5sound?3?5?$CFs?$AA@ 300417f0     cg_players.obj
 0002:0000380c       ??_C@_0CH@JCI@Memory?5is?5low?4?5?5Using?5deferred?5m@ 3004180c     cg_players.obj
 0002:00003834       ??_C@_0CP@NBGK@model?3?5?$CFs?5skin?3?5?$CFs?5headmodel?3?5?$CFs@ 30041834     cg_players.obj
 0002:00003864       ??_C@_01PEAM@t?$AA@        30041864     cg_players.obj
 0002:00003868       ??_C@_01JME@l?$AA@         30041868     cg_players.obj
 0002:0000386c       ??_C@_01LLF@w?$AA@         3004186c     cg_players.obj
 0002:00003870       ??_C@_02MCDK@hc?$AA@       30041870     cg_players.obj
 0002:00003874       ??_C@_05MIHE@skill?$AA@    30041874     cg_players.obj
 0002:0000387c       ??_C@_02BFAP@c1?$AA@       3004187c     cg_players.obj
 0002:00003880       ??_C@_0BD@FEG@sound?1player?1?$CFs?1?$CFs?$AA@ 30041880     cg_players.obj
 0002:00003894       ??_C@_0CG@CIED@DEFAULT_MODEL?5?$CI?$CFs?$CJ?5failed?5to?5reg@ 30041894     cg_players.obj
 0002:000038bc       ??_C@_0DA@KOEK@DEFAULT_MODEL?5?1?5skin?5?$CI?$CFs?1?$CFs?$CJ?5fai@ 300418bc     cg_players.obj
 0002:000038ec       ??_C@_05JPCA@sarge?$AA@    300418ec     cg_players.obj
 0002:000038f4       ??_C@_0DB@DJJN@CG_RegisterClientModelname?$CI?5?$CFs?1?$CF@ 300418f4     cg_players.obj
 0002:00003928       ??_C@_0CJ@DNB@Registering?5model?3?5?$FL?$CFs?$FN?1?$FL?$CFs?$FN?5?$CL?$FL?$CF@ 30041928     cg_players.obj
 0002:00003954       ??_C@_0BO@GHGD@Failed?5to?5load?5icon?5file?3?5?$CFs?6?$AA@ 30041954     cg_players.obj
 0002:00003974       ??_C@_0CC@OHOC@Failed?5to?5load?5animation?5file?5?$CFs@ 30041974     cg_players.obj
 0002:00003998       ??_C@_0CA@ELJL@models?1players?1?$CFs?1animation?4cfg?$AA@ 30041998     cg_players.obj
 0002:000039b8       ??_C@_0CI@IBGK@Failed?5to?5load?5skin?5file?3?5?$CFs?1?$CFs?5@ 300419b8     cg_players.obj
 0002:000039e0       ??_C@_0BL@MPJF@models?1players?1?$CFs?1head?4md3?$AA@ 300419e0     cg_players.obj
 0002:000039fc       ??_C@_0BM@CCGI@models?1players?1?$CFs?1upper?4md3?$AA@ 300419fc     cg_players.obj
 0002:00003a18       ??_C@_0BO@ELEH@Failed?5to?5load?5model?5file?5?$CFs?6?$AA@ 30041a18     cg_players.obj
 0002:00003a38       ??_C@_0BM@CEFP@models?1players?1?$CFs?1lower?4md3?$AA@ 30041a38     cg_players.obj
 0002:00003a54       ??_C@_0CB@GMGP@Error?5parsing?5animation?5file?3?5?$CFs@ 30041a54     cg_players.obj
 0002:00003a78       ??_C@_0BK@LJDE@unknown?5token?5?8?$CFs?8?5is?5?$CFs?6?$AA@ 30041a78     cg_players.obj
 0002:00003a94       ??_C@_03CJDB@sex?$AA@      30041a94     cg_players.obj
 0002:00003a98       ??_C@_0L@EPMP@headoffset?$AA@ 30041a98     cg_players.obj
 0002:00003aa4       ??_C@_0BO@PCCE@Bad?5footsteps?5parm?5in?5?$CFs?3?5?$CFs?6?$AA@ 30041aa4     cg_players.obj
 0002:00003ac4       ??_C@_06GBBO@energy?$AA@   30041ac4     cg_players.obj
 0002:00003acc       ??_C@_04FOOO@mech?$AA@     30041acc     cg_players.obj
 0002:00003ad4       ??_C@_05NMDE@flesh?$AA@    30041ad4     cg_players.obj
 0002:00003adc       ??_C@_04CDC@boot?$AA@      30041adc     cg_players.obj
 0002:00003ae4       ??_C@_06KMLP@normal?$AA@   30041ae4     cg_players.obj
 0002:00003aec       ??_C@_09EDIM@footsteps?$AA@ 30041aec     cg_players.obj
 0002:00003af8       ??_C@_0BC@GFDL@File?5?$CFs?5too?5long?6?$AA@ 30041af8     cg_players.obj
 0002:00003b0c       ??_C@_0BP@GEHB@models?1players?1?$CFs?1head_?$CFs?4skin?$AA@ 30041b0c     cg_players.obj
 0002:00003b2c       ??_C@_0CA@LBBA@models?1players?1?$CFs?1upper_?$CFs?4skin?$AA@ 30041b2c     cg_players.obj
 0002:00003b4c       ??_C@_0CA@FIAK@models?1players?1?$CFs?1lower_?$CFs?4skin?$AA@ 30041b4c     cg_players.obj
 0002:00003b6c       ??_C@_08JGJE@tag_head?$AA@ 30041b6c     cg_players.obj
 0002:00003b78       __real@4@c001a000000000000000 30041b78     cg_players.obj
 0002:00003b7c       ??_C@_09ECJI@tag_torso?$AA@ 30041b7c     cg_players.obj
 0002:00003b88       __real@4@c004a000000000000000 30041b88     cg_players.obj
 0002:00003b8c       ??_C@_05KPPP@WTF?$CB?$DP?$AA@ 30041b8c     cg_players.obj
 0002:00003b94       ??_C@_0BP@MOFG@Bad?5clientNum?5on?5player?5entity?$AA@ 30041b94     cg_players.obj
 0002:00003bb4       ??_C@_0BF@OFAO@Clamp?5lf?9?$DOframeTime?6?$AA@ 30041bb4     cg_players.obj
 0002:00003bcc       ??_C@_09FILE@Anim?3?5?$CFi?6?$AA@ 30041bcc     cg_players.obj
 0002:00003bd8       ??_C@_0BJ@MCPI@Bad?5animation?5number?3?5?$CFi?$AA@ 30041bd8     cg_players.obj
 0002:00003bf8       __real@8@3ffaccccccccccccd000 30041bf8     cg_players.obj
 0002:00003c00       __real@4@c007b400000000000000 30041c00     cg_players.obj
 0002:00003c04       ??_C@_0BK@HHHI@Bad?5player?5movement?5angle?$AA@ 30041c04     cg_players.obj
 0002:00003c20       __real@4@4005b400000000000000 30041c20     cg_players.obj
 0002:00003c24       __real@4@4001c000000000000000 30041c24     cg_players.obj
 0002:00003c28       ??_C@_0BN@PDIA@?$CFi?5ResetPlayerEntity?5yaw?$DN?$CFi?6?$AA@ 30041c28     cg_players.obj
 0002:00003c48       __real@8@bfff8000000000000000 30041c48     cg_playerstate.obj
 0002:00003c50       __real@8@4006ff00000000000000 30041c50     cg_playerstate.obj
 0002:00003c58       __real@8@4004a000000000000000 30041c58     cg_playerstate.obj
 0002:00003c60       ??_C@_0N@HFCI@Bad?5reward_t?$AA@ 30041c60     cg_playerstate.obj
 0002:00003c70       ??_C@_0L@PNJD@not?5moved?6?$AA@ 30041c70     cg_predict.obj
 0002:00003c7c       ??_C@_0L@KNMH@?$FL?$CFi?5?3?5?$CFi?$FN?5?$AA@ 30041c7c     cg_predict.obj
 0002:00003c88       ??_C@_0BN@HHO@Double?5prediction?5decay?3?5?$CFf?6?$AA@ 30041c88     cg_predict.obj
 0002:00003ca8       ??_C@_0BF@EJKK@Prediction?5miss?3?5?$CFf?6?$AA@ 30041ca8     cg_predict.obj
 0002:00003cc0       ??_C@_0BE@LGAC@PredictionTeleport?6?$AA@ 30041cc0     cg_predict.obj
 0002:00003cd4       ??_C@_0CE@GAJH@exceeded?5PACKET_BACKUP?5on?5comman@ 30041cd4     cg_predict.obj
 0002:00003cf8       ??_C@_0BE@LFKI@Blue?5leads?5?$CFi?5to?5?$CFi?$AA@ 30041cf8     cg_scoreboard.obj
 0002:00003d0c       ??_C@_0BD@JNHP@Red?5leads?5?$CFi?5to?5?$CFi?$AA@ 30041d0c     cg_scoreboard.obj
 0002:00003d20       ??_C@_0BF@JNNA@Teams?5are?5tied?5at?5?$CFi?$AA@ 30041d20     cg_scoreboard.obj
 0002:00003d38       ??_C@_0BB@NFNC@?$CFs?5place?5with?5?$CFi?$AA@ 30041d38     cg_scoreboard.obj
 0002:00003d4c       ??_C@_0O@NJOP@Fragged?5by?5?$CFs?$AA@ 30041d4c     cg_scoreboard.obj
 0002:00003d5c       ??_C@_05HKPI@READY?$AA@    30041d5c     cg_scoreboard.obj
 0002:00003d64       ??_C@_0P@BDKN@?$CF5i?5?$CF4i?5?$CF4i?5?$CFs?$AA@ 30041d64     cg_scoreboard.obj
 0002:00003d74       ??_C@_0BC@BLFH@?5SPECT?5?$CF3i?5?$CF4i?5?$CFs?$AA@ 30041d74     cg_scoreboard.obj
 0002:00003d88       ??_C@_0BC@PMKJ@?5connecting?5?5?5?5?$CFs?$AA@ 30041d88     cg_scoreboard.obj
 0002:00003d9c       ??_C@_05CJED@?$CFi?1?$CFi?$AA@ 30041d9c     cg_scoreboard.obj
 0002:00003da4       ??_C@_0BH@EOKJ@Bad?5score?9?$DOclient?3?5?$CFi?6?$AA@ 30041da4     cg_scoreboard.obj
 0002:00003dbc       ??_C@_09OLDB@Blue?5Team?$AA@ 30041dbc     cg_scoreboard.obj
 0002:00003dc8       ??_C@_08PHPI@Red?5Team?$AA@ 30041dc8     cg_scoreboard.obj
 0002:00003dd4       ??_C@_0L@PJCP@Scoreboard?$AA@ 30041dd4     cg_scoreboard.obj
 0002:00003de0       ??_C@_0M@HBDC@maps?1?$CFs?4bsp?$AA@ 30041de0     cg_servercmds.obj
 0002:00003dec       ??_C@_0O@KKJL@sv_maxclients?$AA@ 30041dec     cg_servercmds.obj
 0002:00003dfc       ??_C@_09NNDG@teamflags?$AA@ 30041dfc     cg_servercmds.obj
 0002:00003e08       ??_C@_07NJLK@dmflags?$AA@  30041e08     cg_servercmds.obj
 0002:00003e10       ??_C@_0L@IEJM@g_gametype?$AA@ 30041e10     cg_servercmds.obj
 0002:00003e1c       ??_C@_0CB@PEKB@Unknown?5client?5game?5command?3?5?$CFs?6@ 30041e1c     cg_servercmds.obj
 0002:00003e40       ??_C@_0BA@OGON@clientLevelShot?$AA@ 30041e40     cg_servercmds.obj
 0002:00003e50       ??_C@_0M@PKCG@map_restart?$AA@ 30041e50     cg_servercmds.obj
 0002:00003e5c       ??_C@_05DLPD@tinfo?$AA@    30041e5c     cg_servercmds.obj
 0002:00003e64       ??_C@_06CLLB@scores?$AA@   30041e64     cg_servercmds.obj
 0002:00003e6c       ??_C@_05NEJE@tchat?$AA@    30041e6c     cg_servercmds.obj
 0002:00003e74       ??_C@_03HHKO@?$CFs?6?$AA@  30041e74     cg_servercmds.obj
 0002:00003e78       ??_C@_04FLKK@chat?$AA@     30041e78     cg_servercmds.obj
 0002:00003e80       ??_C@_05KCGF@print?$AA@    30041e80     cg_servercmds.obj
 0002:00003e88       ??_C@_02OFOB@cs?$AA@       30041e88     cg_servercmds.obj
 0002:00003e8c       ??_C@_02BKFI@cp?$AA@       30041e8c     cg_servercmds.obj
 0002:00003e90       ??_C@_06GEGH@FIGHT?$CB?$AA@ 30041e90     cg_servercmds.obj
 0002:00003e98       ??_C@_0P@IGKC@CG_MapRestart?6?$AA@ 30041e98     cg_servercmds.obj
 0002:00003ea8       ??_C@_0DI@CBJH@CG_ProcessSnapshots?3?5cg?4nextSnap@ 30041ea8     cg_snapshot.obj
 0002:00003ee0       ??_C@_0CF@EMJA@CG_ProcessSnapshots?3?5cg?4snap?5?$DN?$DN?5@ 30041ee0     cg_snapshot.obj
 0002:00003f08       ??_C@_0DA@DBCO@CG_ProcessSnapshots?3?5Server?5time@ 30041f08     cg_snapshot.obj
 0002:00003f38       ??_C@_0CO@GEJI@CG_ProcessSnapshots?3?5n?5?$DM?5cg?4late@ 30041f38     cg_snapshot.obj
 0002:00003f68       ??_C@_0CI@MEOD@CG_TransitionSnapshot?3?5NULL?5cg?4n@ 30041f68     cg_snapshot.obj
 0002:00003f90       ??_C@_0CE@LMCK@CG_TransitionSnapshot?3?5NULL?5cg?4s@ 30041f90     cg_snapshot.obj
 0002:00003fb4       ??_C@_0CP@GMAG@CG_ReadNextSnapshot?3?5way?5out?5of?5@ 30041fb4     cg_snapshot.obj
 0002:00003fe4       ??_C@_0BG@MBEM@Can?8t?5register?5model?6?$AA@ 30041fe4     cg_view.obj
 0002:00003ffc       ??_C@_09KDBC@frame?5?$CFi?6?$AA@ 30041ffc     cg_view.obj
 0002:00004008       ??_C@_08CDMB@skin?5?$CFi?6?$AA@ 30042008     cg_view.obj
 0002:00004014       ??_C@_0BD@BFGA@cg?4clientFrame?3?$CFi?6?$AA@ 30042014     cg_view.obj
 0002:00004028       __real@4@c0028000000000000000 30042028     cg_view.obj
 0002:0000402c       ??_C@_02HPJE@30?$AA@       3004202c     cg_view.obj
 0002:00004030       __real@8@c004e52ee0d31e0fc000 30042030     cg_view.obj
 0002:00004038       __real@8@40048000000000000000 30042038     cg_view.obj
 0002:00004040       __real@4@40088000000000000000 30042040     cg_view.obj
 0002:00004044       __real@4@4007e100000000000000 30042044     cg_view.obj
 0002:00004048       __real@4@40069600000000000000 30042048     cg_view.obj
 0002:0000404c       __real@4@4007c800000000000000 3004204c     cg_view.obj
 0002:00004050       __real@8@40059600000000000000 30042050     cg_view.obj
 0002:00004058       __real@4@4006a000000000000000 30042058     cg_view.obj
 0002:00004060       __real@8@4004f880000000000000 30042060     cg_weapons.obj
 0002:00004068       ??_C@_0CB@BDCJ@Error?3?5zero?5r_railSegmentLength?6@ 30042068     cg_weapons.obj
 0002:0000408c       __real@4@c001c000000000000000 3004208c     cg_weapons.obj
 0002:00004090       __real@4@4003d000000000000000 30042090     cg_weapons.obj
 0002:00004094       ??_C@_0BI@ONPH@models?1weaphits?1bfg?4md3?$AA@ 30042094     cg_weapons.obj
 0002:000040ac       ??_C@_0N@EBOG@bfgExplosion?$AA@ 300420ac     cg_weapons.obj
 0002:000040bc       ??_C@_0BP@NFJJ@sound?1weapons?1bfg?1bfg_fire?4wav?$AA@ 300420bc     cg_weapons.obj
 0002:000040dc       ??_C@_0BO@HMHF@sound?1weapons?1bfg?1bfg_hum?4wav?$AA@ 300420dc     cg_weapons.obj
 0002:000040fc       ??_C@_08DAFP@railCore?$AA@ 300420fc     cg_weapons.obj
 0002:00004108       ??_C@_08MPEO@railDisc?$AA@ 30042108     cg_weapons.obj
 0002:00004114       ??_C@_0CB@HGGM@sound?1weapons?1railgun?1rg_hum?4wav@ 30042114     cg_weapons.obj
 0002:00004138       ??_C@_0BA@NFMO@plasmaExplosion?$AA@ 30042138     cg_weapons.obj
 0002:00004148       ??_C@_0CC@JIFL@sound?1weapons?1plasma?1hyprbf1a?4wa@ 30042148     cg_weapons.obj
 0002:0000416c       ??_C@_0CA@NOMN@sound?1weapons?1plasma?1lasfly?4wav?$AA@ 3004216c     cg_weapons.obj
 0002:0000418c       ??_C@_0BB@OGAO@grenadeExplosion?$AA@ 3004218c     cg_weapons.obj
 0002:000041a0       ??_C@_0CD@LLBD@sound?1weapons?1grenade?1grenlf1a?4w@ 300421a0     cg_weapons.obj
 0002:000041c4       ??_C@_0BJ@OLCP@models?1ammo?1grenade1?4md3?$AA@ 300421c4     cg_weapons.obj
 0002:000041e0       ??_C@_0BA@LLML@rocketExplosion?$AA@ 300421e0     cg_weapons.obj
 0002:000041f0       ??_C@_0CC@EFJP@sound?1weapons?1rocket?1rocklf1a?4wa@ 300421f0     cg_weapons.obj
 0002:00004214       ??_C@_0CB@BJPM@sound?1weapons?1rocket?1rockfly?4wav@ 30042214     cg_weapons.obj
 0002:00004238       ??_C@_0CD@ILHF@sound?1weapons?1shotgun?1sshotf1b?4w@ 30042238     cg_weapons.obj
 0002:0000425c       ??_C@_0BA@OKAK@bulletExplosion?$AA@ 3004225c     cg_weapons.obj
 0002:0000426c       ??_C@_0CG@NLKL@sound?1weapons?1machinegun?1machgf4@ 3004226c     cg_weapons.obj
 0002:00004294       ??_C@_0CG@DDML@sound?1weapons?1machinegun?1machgf3@ 30042294     cg_weapons.obj
 0002:000042bc       ??_C@_0CG@KGGL@sound?1weapons?1machinegun?1machgf2@ 300422bc     cg_weapons.obj
 0002:000042e4       ??_C@_0CG@BIIL@sound?1weapons?1machinegun?1machgf1@ 300422e4     cg_weapons.obj
 0002:0000430c       ??_C@_0BO@CMJ@models?1ammo?1rocket?1rocket?4md3?$AA@ 3004230c     cg_weapons.obj
 0002:0000432c       ??_C@_0CE@NIOG@sound?1weapons?1lightning?1lg_hit3?4@ 3004232c     cg_weapons.obj
 0002:00004350       ??_C@_0CE@HIMD@sound?1weapons?1lightning?1lg_hit2?4@ 30042350     cg_weapons.obj
 0002:00004374       ??_C@_0CD@IMBG@sound?1weapons?1lightning?1lg_hit?4w@ 30042374     cg_weapons.obj
 0002:00004398       ??_C@_0BM@JNJK@models?1weaphits?1crackle?4md3?$AA@ 30042398     cg_weapons.obj
 0002:000043b4       ??_C@_0O@LKNG@lightningBolt?$AA@ 300423b4     cg_weapons.obj
 0002:000043c4       ??_C@_0CE@JPGL@sound?1weapons?1lightning?1lg_fire?4@ 300423c4     cg_weapons.obj
 0002:000043e8       ??_C@_0CD@IOMP@sound?1weapons?1lightning?1lg_hum?4w@ 300423e8     cg_weapons.obj
 0002:0000440c       ??_C@_0BP@PNMO@sound?1weapons?1melee?1fsthum?4wav?$AA@ 3004240c     cg_weapons.obj
 0002:0000442c       ??_C@_0CA@KDLC@sound?1weapons?1melee?1fstatck?4wav?$AA@ 3004242c     cg_weapons.obj
 0002:0000444c       ??_C@_0BP@NNHN@sound?1weapons?1melee?1fstrun?4wav?$AA@ 3004244c     cg_weapons.obj
 0002:0000446c       ??_C@_0CJ@HMHN@models?1weapons2?1shotgun?1shotgun_@ 3004246c     cg_weapons.obj
 0002:00004498       ??_C@_09EPBB@_hand?4md3?$AA@ 30042498     cg_weapons.obj
 0002:000044a4       ??_C@_0M@LLAK@_barrel?4md3?$AA@ 300424a4     cg_weapons.obj
 0002:000044b0       ??_C@_0L@LKFC@_flash?4md3?$AA@ 300424b0     cg_weapons.obj
 0002:000044bc       ??_C@_0BI@GDKJ@Couldn?8t?5find?5weapon?5?$CFi?$AA@ 300424bc     cg_weapons.obj
 0002:000044d8       __real@8@3ffdccccccccccccd000 300424d8     cg_weapons.obj
 0002:000044e0       __real@8@4004c800000000000000 300424e0     cg_weapons.obj
 0002:000044e8       __real@8@c004c800000000000000 300424e8     cg_weapons.obj
 0002:000044f0       __real@8@c004a000000000000000 300424f0     cg_weapons.obj
 0002:000044f8       __real@8@4002a000000000000000 300424f8     cg_weapons.obj
 0002:00004500       ??_C@_09ONMF@tag_flash?$AA@ 30042500     cg_weapons.obj
 0002:0000450c       ??_C@_0L@FMME@tag_weapon?$AA@ 3004250c     cg_weapons.obj
 0002:00004518       __real@8@40068000000000000000 30042518     cg_weapons.obj
 0002:00004520       __real@4@4009bb80000000000000 30042520     cg_weapons.obj
 0002:00004524       __real@4@4008c000000000000000 30042524     cg_weapons.obj
 0002:00004528       __real@4@4002e000000000000000 30042528     cg_weapons.obj
 0002:00004530       __real@8@3ffee666666666666800 30042530     cg_weapons.obj
 0002:00004538       __real@8@bffcccccccccccccd000 30042538     cg_weapons.obj
 0002:00004540       __real@8@40079600000000000000 30042540     cg_weapons.obj
 0002:00004548       ??_C@_09HADH@Dropped?3?5?$AA@ 30042548     cg_weapons.obj
 0002:00004554       ??_C@_0CN@IAOL@CG_FireWeapon?3?5ent?9?$DOweapon?5?$DO?$DN?5WP@ 30042554     cg_weapons.obj
 0002:00004588       __real@8@4008c800000000000000 30042588     cg_weapons.obj
 0002:00004590       __real@4@4004c800000000000000 30042590     cg_weapons.obj
 0002:00004594       __real@4@400f8000000000000000 30042594     q_math.obj
 0002:00004598       __real@4@3ffe8000000000000000 30042598     q_math.obj
 0002:0000459c       __real@4@c006b400000000000000 3004259c     q_math.obj
 0002:000045a0       __real@8@4006b60b60b60b60b800 300425a0     q_math.obj
 0002:000045a8       __real@4@bfff8000000000000000 300425a8     q_math.obj
 0002:000045b0       __real@8@3ff98efa351294e9c800 300425b0     q_math.obj
 0002:000045b8       ??_C@_0BF@JENF@MatchToken?3?5?$CFs?5?$CB?$DN?5?$CFs?$AA@ 300425b8     q_shared.obj
 0002:000045d0       ??_C@_01KMMP@?$CJ?$AA@     300425d0     q_shared.obj
 0002:000045d4       ??_C@_01GFI@?$CI?$AA@      300425d4     q_shared.obj
 0002:000045d8       ??_C@_0BJ@GDCK@Q_strncpyz?3?5destsize?5?$DM?51?$AA@ 300425d8     q_shared.obj
 0002:000045f4       ??_C@_0BF@OBLI@Q_strncpyz?3?5NULL?5src?$AA@ 300425f4     q_shared.obj
 0002:0000460c       ??_C@_0BN@PKJG@Q_strcat?3?5already?5overflowed?$AA@ 3004260c     q_shared.obj
 0002:0000462c       ??_C@_0CD@KCEE@Com_sprintf?3?5overflow?5of?5?$CFi?5in?5?$CF@ 3004262c     q_shared.obj
 0002:00004650       ??_C@_0CC@NDC@Com_sprintf?3?5overflowed?5bigbuffe@ 30042650     q_shared.obj
 0002:00004674       ??_C@_0CG@FAFH@Info_ValueForKey?3?5oversize?5infos@ 30042674     q_shared.obj
 0002:0000469c       ??_C@_0CE@CNEE@Info_RemoveKey?3?5oversize?5infostr@ 3004269c     q_shared.obj
 0002:000046c0       ??_C@_0BN@DPCF@Info?5string?5length?5exceeded?6?$AA@ 300426c0     q_shared.obj
 0002:000046e0       ??_C@_06GNBE@?2?$CFs?2?$CFs?$AA@ 300426e0     q_shared.obj
 0002:000046e8       ??_C@_0CD@NLGB@Can?8t?5use?5keys?5or?5values?5with?5a?5@ 300426e8     q_shared.obj
 0002:0000470c       ??_C@_0CL@GPCB@Can?8t?5use?5keys?5or?5values?5with?5a?5@ 3004270c     q_shared.obj
 0002:00004738       ??_C@_0CD@MJE@Can?8t?5use?5keys?5or?5values?5with?5a?5@ 30042738     q_shared.obj
 0002:0000475c       ??_C@_0CJ@GBHP@Info_SetValueForKey?3?5oversize?5in@ 3004275c     q_shared.obj
 0002:00004788       ??_C@_0P@LNLA@format?5?$CB?$DN?5NULL?$AA@ 30042788     LIBCMTD:vsprintf.obj
 0002:00004798       ??_C@_0L@HE@vsprintf?4c?$AA@ 30042798     LIBCMTD:vsprintf.obj
 0002:000047a4       ??_C@_0P@OOIN@string?5?$CB?$DN?5NULL?$AA@ 300427a4     LIBCMTD:vsprintf.obj
 0002:000047c8       __DEFAULT_CW_in_mem        300427c8     LIBCMTD:common.obj
 0002:000047ca       __pi_by_2_to_61            300427ca     LIBCMTD:common.obj
 0002:00004804       ??_C@_0BK@JEGK@IsProcessorFeaturePresent?$AA@ 30042804     LIBCMTD:testfdiv.obj
 0002:00004820       ??_C@_08OBID@KERNEL32?$AA@ 30042820     LIBCMTD:testfdiv.obj
 0002:0000482c       ??_C@_05OFLO@e?$CL000?$AA@ 3004282c     LIBCMTD:cvt.obj
 0002:00004834       ??_C@_03GAFO@_yn?$AA@      30042834     LIBCMTD:fpexcept.obj
 0002:00004838       ??_C@_03GNLD@_y1?$AA@      30042838     LIBCMTD:fpexcept.obj
 0002:0000483c       ??_C@_03MHCE@_y0?$AA@      3004283c     LIBCMTD:fpexcept.obj
 0002:00004840       ??_C@_05PAK@frexp?$AA@     30042840     LIBCMTD:fpexcept.obj
 0002:00004848       ??_C@_04JKCH@fmod?$AA@     30042848     LIBCMTD:fpexcept.obj
 0002:00004850       ??_C@_06GGHF@_hypot?$AA@   30042850     LIBCMTD:fpexcept.obj
 0002:00004858       ??_C@_05JNMC@_cabs?$AA@    30042858     LIBCMTD:fpexcept.obj
 0002:00004860       ??_C@_05MEKH@ldexp?$AA@    30042860     LIBCMTD:fpexcept.obj
 0002:00004868       ??_C@_04KAOJ@modf?$AA@     30042868     LIBCMTD:fpexcept.obj
 0002:00004870       ??_C@_04EHAJ@fabs?$AA@     30042870     LIBCMTD:fpexcept.obj
 0002:00004878       ??_C@_05MFBN@floor?$AA@    30042878     LIBCMTD:fpexcept.obj
 0002:00004880       ??_C@_04JJMP@ceil?$AA@     30042880     LIBCMTD:fpexcept.obj
 0002:00004888       ??_C@_03JLPI@tan?$AA@      30042888     LIBCMTD:fpexcept.obj
 0002:0000488c       ??_C@_03DLFL@cos?$AA@      3004288c     LIBCMTD:fpexcept.obj
 0002:00004890       ??_C@_03JAMN@sin?$AA@      30042890     LIBCMTD:fpexcept.obj
 0002:00004894       ??_C@_04LMBE@sqrt?$AA@     30042894     LIBCMTD:fpexcept.obj
 0002:0000489c       ??_C@_05BFPO@atan2?$AA@    3004289c     LIBCMTD:fpexcept.obj
 0002:000048a4       ??_C@_04EAGN@atan?$AA@     300428a4     LIBCMTD:fpexcept.obj
 0002:000048ac       ??_C@_04OAMO@acos?$AA@     300428ac     LIBCMTD:fpexcept.obj
 0002:000048b4       ??_C@_04ELFI@asin?$AA@     300428b4     LIBCMTD:fpexcept.obj
 0002:000048bc       ??_C@_04LFAD@tanh?$AA@     300428bc     LIBCMTD:fpexcept.obj
 0002:000048c4       ??_C@_04PFKD@cosh?$AA@     300428c4     LIBCMTD:fpexcept.obj
 0002:000048cc       ??_C@_04NPAI@sinh?$AA@     300428cc     LIBCMTD:fpexcept.obj
 0002:000048d4       ??_C@_05IJHH@log10?$AA@    300428d4     LIBCMTD:fpexcept.obj
 0002:000048dc       ??_C@_03BGKD@log?$AA@      300428dc     LIBCMTD:fpexcept.obj
 0002:000048e0       ??_C@_03EGFG@pow?$AA@      300428e0     LIBCMTD:fpexcept.obj
 0002:000048e4       ??_C@_03CDGJ@exp?$AA@      300428e4     LIBCMTD:fpexcept.obj
 0002:000048e8       ??_C@_0DP@IHIN@?$CI?$CCinconsistent?5IOB?5fields?$CC?0?5stre@ 300428e8     LIBCMTD:_flsbuf.obj
 0002:00004928       ??_C@_09LGEI@_flsbuf?4c?$AA@ 30042928     LIBCMTD:_flsbuf.obj
 0002:00004934       ??_C@_0M@KJPK@str?5?$CB?$DN?5NULL?$AA@ 30042934     LIBCMTD:_flsbuf.obj
 0002:00004940       ___lookuptable             30042940     LIBCMTD:output.obj
 0002:0000499c       ??_C@_1O@POHA@?$AA?$CI?$AAn?$AAu?$AAl?$AAl?$AA?$CJ?$AA?$AA@ 3004299c     LIBCMTD:output.obj
 0002:000049ac       ??_C@_06ONKE@?$CInull?$CJ?$AA@ 300429ac     LIBCMTD:output.obj
 0002:000049b4       ??_C@_08MIHI@output?4c?$AA@ 300429b4     LIBCMTD:output.obj
 0002:000049c0       ??_C@_0P@PIHB@ch?5?$CB?$DN?5_T?$CI?8?20?8?$CJ?$AA@ 300429c0     LIBCMTD:output.obj
 0002:000049d0       ??_C@_0BB@BLL@Assertion?5Failed?$AA@ 300429d0     LIBCMTD:dbgrpt.obj
 0002:000049e4       ??_C@_05CKBG@Error?$AA@    300429e4     LIBCMTD:dbgrpt.obj
 0002:000049ec       ??_C@_07JCGI@Warning?$AA@  300429ec     LIBCMTD:dbgrpt.obj
 0002:000049f4       ??_C@_0M@ODEP@?$CFs?$CI?$CFd?$CJ?5?3?5?$CFs?$AA@ 300429f4     LIBCMTD:dbgrpt.obj
 0002:00004a00       ??_C@_01BJG@?6?$AA@        30042a00     LIBCMTD:dbgrpt.obj
 0002:00004a04       ??_C@_01FEHD@?$AN?$AA@     30042a04     LIBCMTD:dbgrpt.obj
 0002:00004a08       ??_C@_0BC@OIMC@Assertion?5failed?$CB?$AA@ 30042a08     LIBCMTD:dbgrpt.obj
 0002:00004a1c       ??_C@_0BD@BEAK@Assertion?5failed?3?5?$AA@ 30042a1c     LIBCMTD:dbgrpt.obj
 0002:00004a30       ??_C@_0CL@LCCP@_CrtDbgReport?3?5String?5too?5long?5o@ 30042a30     LIBCMTD:dbgrpt.obj
 0002:00004a5c       ??_C@_0DC@EMDK@Second?5Chance?5Assertion?5Failed?3?5@ 30042a5c     LIBCMTD:dbgrpt.obj
 0002:00004a90       ??_C@_09NJAK@wsprintfA?$AA@ 30042a90     LIBCMTD:dbgrpt.obj
 0002:00004a9c       ??_C@_0L@HKL@user32?4dll?$AA@ 30042a9c     LIBCMTD:dbgrpt.obj
 0002:00004aa8       ??_C@_0CD@GCMD@Microsoft?5Visual?5C?$CL?$CL?5Debug?5Libra@ 30042aa8     LIBCMTD:dbgrpt.obj
 0002:00004acc       ??_C@_0FD@EBDD@Debug?5?$CFs?$CB?6?6Program?3?5?$CFs?$CFs?$CFs?$CFs?$CFs?$CFs@ 30042acc     LIBCMTD:dbgrpt.obj
 0002:00004b20       ??_C@_09DCKN@?6Module?3?5?$AA@ 30042b20     LIBCMTD:dbgrpt.obj
 0002:00004b2c       ??_C@_07HJII@?6File?3?5?$AA@ 30042b2c     LIBCMTD:dbgrpt.obj
 0002:00004b34       ??_C@_07LFGN@?6Line?3?5?$AA@ 30042b34     LIBCMTD:dbgrpt.obj
 0002:00004b3c       ??_C@_02JJJH@?6?6?$AA@     30042b3c     LIBCMTD:dbgrpt.obj
 0002:00004b40       ??_C@_0N@NOAB@Expression?3?5?$AA@ 30042b40     LIBCMTD:dbgrpt.obj
 0002:00004b50       ??_C@_0HD@BHFH@?6?6For?5information?5on?5how?5your?5pr@ 30042b50     LIBCMTD:dbgrpt.obj
 0002:00004bc4       ??_C@_03NAME@?4?4?4?$AA@   30042bc4     LIBCMTD:dbgrpt.obj
 0002:00004bc8       ??_C@_0BH@NNCD@?$DMprogram?5name?5unknown?$DO?$AA@ 30042bc8     LIBCMTD:dbgrpt.obj
 0002:00004be0       ??_C@_08GFHP@dbgrpt?4c?$AA@ 30042be0     LIBCMTD:dbgrpt.obj
 0002:00004bec       ??_C@_0BG@FBEA@szUserMessage?5?$CB?$DN?5NULL?$AA@ 30042bec     LIBCMTD:dbgrpt.obj
 0002:00004c40       ??_C@_07PDLA@mlock?4c?$AA@ 30042c40     LIBCMTD:mlock.obj
 0002:00004c48       ??_C@_07PCLE@LC_TIME?$AA@  30042c48     LIBCMTD:setlocal.obj
 0002:00004c50       ??_C@_0L@NKG@LC_NUMERIC?$AA@ 30042c50     LIBCMTD:setlocal.obj
 0002:00004c5c       ??_C@_0M@CBIH@LC_MONETARY?$AA@ 30042c5c     LIBCMTD:setlocal.obj
 0002:00004c68       ??_C@_08LFGE@LC_CTYPE?$AA@ 30042c68     LIBCMTD:setlocal.obj
 0002:00004c74       ??_C@_0L@CFLC@LC_COLLATE?$AA@ 30042c74     LIBCMTD:setlocal.obj
 0002:00004c80       ??_C@_06GCPK@LC_ALL?$AA@   30042c80     LIBCMTD:setlocal.obj
 0002:00004c88       ??_C@_01FAJB@?$DL?$AA@     30042c88     LIBCMTD:setlocal.obj
 0002:00004c8c       ??_C@_02BGDO@?$DN?$DL?$AA@ 30042c8c     LIBCMTD:setlocal.obj
 0002:00004c90       ??_C@_0L@MOEE@setlocal?4c?$AA@ 30042c90     LIBCMTD:setlocal.obj
 0002:00004c9c       ??_C@_01KPOD@?$DN?$AA@     30042c9c     LIBCMTD:setlocal.obj
 0002:00004ca0       ??_C@_03DBOJ@_?4?0?$AA@    30042ca0     LIBCMTD:setlocal.obj
 0002:00004ca4       ??_C@_01PJCK@?4?$AA@       30042ca4     LIBCMTD:setlocal.obj
 0002:00004ca8       ??_C@_01NON@_?$AA@         30042ca8     LIBCMTD:setlocal.obj
 0002:00004cac       ??_C@_01A@?$AA?$AA@        30042cac     LIBCMTD:a_map.obj
 0002:00004cb0       ??_C@_13A@?$AA?$AA?$AA?$AA@ 30042cb0     LIBCMTD:a_map.obj
 0002:00004cd0       ??_C@_0L@ENLJ@tidtable?4c?$AA@ 30042cd0     LIBCMTD:tidtable.obj
 0002:00004cdc       ??_C@_08KFDJ@ioinit?4c?$AA@ 30042cdc     LIBCMTD:ioinit.obj
 0002:00004ce8       ??_C@_06DPMO@Client?$AA@   30042ce8     LIBCMTD:dbgheap.obj
 0002:00004cf0       ??_C@_06BAFM@Ignore?$AA@   30042cf0     LIBCMTD:dbgheap.obj
 0002:00004cf8       ??_C@_03DICE@CRT?$AA@      30042cf8     LIBCMTD:dbgheap.obj
 0002:00004cfc       ??_C@_06BILL@Normal?$AA@   30042cfc     LIBCMTD:dbgheap.obj
 0002:00004d04       ??_C@_04NEN@Free?$AA@      30042d04     LIBCMTD:dbgheap.obj
 0002:00004d0c       ??_C@_0DC@CGID@Error?3?5memory?5allocation?3?5bad?5me@ 30042d0c     LIBCMTD:dbgheap.obj
 0002:00004d40       ??_C@_0CE@FMIA@Invalid?5allocation?5size?3?5?$CFu?5byte@ 30042d40     LIBCMTD:dbgheap.obj
 0002:00004d64       ??_C@_0CB@CPBI@Client?5hook?5allocation?5failure?4?6@ 30042d64     LIBCMTD:dbgheap.obj
 0002:00004d88       ??_C@_0DF@DKHF@Client?5hook?5allocation?5failure?5a@ 30042d88     LIBCMTD:dbgheap.obj
 0002:00004dc0       ??_C@_09IMJC@dbgheap?4c?$AA@ 30042dc0     LIBCMTD:dbgheap.obj
 0002:00004dcc       ??_C@_0BC@EPKL@_CrtCheckMemory?$CI?$CJ?$AA@ 30042dcc     LIBCMTD:dbgheap.obj
 0002:00004de0       ??_C@_0BK@JDHA@_pFirstBlock?5?$DN?$DN?5pOldBlock?$AA@ 30042de0     LIBCMTD:dbgheap.obj
 0002:00004dfc       ??_C@_0BJ@NMEF@_pLastBlock?5?$DN?$DN?5pOldBlock?$AA@ 30042dfc     LIBCMTD:dbgheap.obj
 0002:00004e18       ??_C@_0DC@BOCN@fRealloc?5?$HM?$HM?5?$CI?$CBfRealloc?5?$CG?$CG?5pNewBl@ 30042e18     LIBCMTD:dbgheap.obj
 0002:00004e4c       ??_C@_0DK@DKOM@_BLOCK_TYPE?$CIpOldBlock?9?$DOnBlockUse@ 30042e4c     LIBCMTD:dbgheap.obj
 0002:00004e88       ??_C@_0EF@EDKM@pOldBlock?9?$DOnLine?5?$DN?$DN?5IGNORE_LINE?5@ 30042e88     LIBCMTD:dbgheap.obj
 0002:00004ed0       ??_C@_0CC@GPMO@_CrtIsValidHeapPointer?$CIpUserData@ 30042ed0     LIBCMTD:dbgheap.obj
 0002:00004ef4       ??_C@_0CN@FHGE@Allocation?5too?5large?5or?5negative@ 30042ef4     LIBCMTD:dbgheap.obj
 0002:00004f24       ??_C@_0CE@EAMN@Client?5hook?5re?9allocation?5failur@ 30042f24     LIBCMTD:dbgheap.obj
 0002:00004f48       ??_C@_0DI@KKMM@Client?5hook?5re?9allocation?5failur@ 30042f48     LIBCMTD:dbgheap.obj
 0002:00004f80       ??_C@_0BG@JCEC@_pFirstBlock?5?$DN?$DN?5pHead?$AA@ 30042f80     LIBCMTD:dbgheap.obj
 0002:00004f98       ??_C@_0BF@NLNN@_pLastBlock?5?$DN?$DN?5pHead?$AA@ 30042f98     LIBCMTD:dbgheap.obj
 0002:00004fb0       ??_C@_0BO@PLHH@pHead?9?$DOnBlockUse?5?$DN?$DN?5nBlockUse?$AA@ 30042fb0     LIBCMTD:dbgheap.obj
 0002:00004fd0       ??_C@_0DN@KKIO@pHead?9?$DOnLine?5?$DN?$DN?5IGNORE_LINE?5?$CG?$CG?5p@ 30042fd0     LIBCMTD:dbgheap.obj
 0002:00005010       ??_C@_0CK@OJNB@DAMAGE?3?5after?5?$CFhs?5block?5?$CI?$CD?$CFd?$CJ?5at@ 30043010     LIBCMTD:dbgheap.obj
 0002:0000503c       ??_C@_0CL@IJIL@DAMAGE?3?5before?5?$CFhs?5block?5?$CI?$CD?$CFd?$CJ?5a@ 3004303c     LIBCMTD:dbgheap.obj
 0002:00005068       ??_C@_0CH@PHOC@_BLOCK_TYPE_IS_VALID?$CIpHead?9?$DOnBlo@ 30043068     LIBCMTD:dbgheap.obj
 0002:00005090       ??_C@_0BL@MBNA@Client?5hook?5free?5failure?4?6?$AA@ 30043090     LIBCMTD:dbgheap.obj
 0002:000050ac       ??_C@_0DK@EKKL@memory?5check?5error?5at?50x?$CF08X?5?$DN?50@ 300430ac     LIBCMTD:dbgheap.obj
 0002:000050e8       ??_C@_0CJ@GCII@?$CFhs?5located?5at?50x?$CF08X?5is?5?$CFu?5byte@ 300430e8     LIBCMTD:dbgheap.obj
 0002:00005114       ??_C@_0CA@EJPI@?$CFhs?5allocated?5at?5file?5?$CFhs?$CI?$CFd?$CJ?4?6?$AA@ 30043114     LIBCMTD:dbgheap.obj
 0002:00005134       ??_C@_0CJ@LHHG@DAMAGE?3?5on?5top?5of?5Free?5block?5at?5@ 30043134     LIBCMTD:dbgheap.obj
 0002:00005160       ??_C@_07GJHM@DAMAGED?$AA@  30043160     LIBCMTD:dbgheap.obj
 0002:00005168       ??_C@_0CL@ODIE@_heapchk?5fails?5with?5unknown?5retu@ 30043168     LIBCMTD:dbgheap.obj
 0002:00005194       ??_C@_0CC@EHNC@_heapchk?5fails?5with?5_HEAPBADPTR?4@ 30043194     LIBCMTD:dbgheap.obj
 0002:000051b8       ??_C@_0CC@JNDP@_heapchk?5fails?5with?5_HEAPBADEND?4@ 300431b8     LIBCMTD:dbgheap.obj
 0002:000051dc       ??_C@_0CD@DNMG@_heapchk?5fails?5with?5_HEAPBADNODE@ 300431dc     LIBCMTD:dbgheap.obj
 0002:00005200       ??_C@_0CE@JMCB@_heapchk?5fails?5with?5_HEAPBADBEGI@ 30043200     LIBCMTD:dbgheap.obj
 0002:00005224       ??_C@_0CD@MEMI@Bad?5memory?5block?5found?5at?50x?$CF08X@ 30043224     LIBCMTD:dbgheap.obj
 0002:00005248       ??_C@_0CI@GMAO@_CrtMemCheckPoint?3?5NULL?5state?5po@ 30043248     LIBCMTD:dbgheap.obj
 0002:00005270       ??_C@_0CI@MNAE@_CrtMemDifference?3?5NULL?5state?5po@ 30043270     LIBCMTD:dbgheap.obj
 0002:00005298       ??_C@_0BH@PKIJ@Object?5dump?5complete?4?6?$AA@ 30043298     LIBCMTD:dbgheap.obj
 0002:000052b0       ??_C@_0DB@DBPF@crt?5block?5at?50x?$CF08X?0?5subtype?5?$CFx?0@ 300432b0     LIBCMTD:dbgheap.obj
 0002:000052e4       ??_C@_0CI@JLM@normal?5block?5at?50x?$CF08X?0?5?$CFu?5bytes@ 300432e4     LIBCMTD:dbgheap.obj
 0002:0000530c       ??_C@_0DE@PFEA@client?5block?5at?50x?$CF08X?0?5subtype?5@ 3004330c     LIBCMTD:dbgheap.obj
 0002:00005340       ??_C@_06MBCE@?$HL?$CFld?$HN?5?$AA@ 30043340     LIBCMTD:dbgheap.obj
 0002:00005348       ??_C@_0L@BLDJ@?$CFhs?$CI?$CFd?$CJ?5?3?5?$AA@ 30043348     LIBCMTD:dbgheap.obj
 0002:00005354       ??_C@_0BE@FEMA@?$CDFile?5Error?$CD?$CI?$CFd?$CJ?5?3?5?$AA@ 30043354     LIBCMTD:dbgheap.obj
 0002:00005368       ??_C@_0BE@FPPM@Dumping?5objects?5?9?$DO?6?$AA@ 30043368     LIBCMTD:dbgheap.obj
 0002:0000537c       ??_C@_0BA@POLM@?5Data?3?5?$DM?$CFs?$DO?5?$CFs?6?$AA@ 3004337c     LIBCMTD:dbgheap.obj
 0002:0000538c       ??_C@_05JLAO@?$CF?42X?5?$AA@ 3004338c     LIBCMTD:dbgheap.obj
 0002:00005394       ??_C@_0BI@KONA@Detected?5memory?5leaks?$CB?6?$AA@ 30043394     LIBCMTD:dbgheap.obj
 0002:000053ac       ??_C@_0BP@LCCN@Total?5allocations?3?5?$CFld?5bytes?4?6?$AA@ 300433ac     LIBCMTD:dbgheap.obj
 0002:000053cc       ??_C@_0CB@COID@Largest?5number?5used?3?5?$CFld?5bytes?4?6@ 300433cc     LIBCMTD:dbgheap.obj
 0002:000053f0       ??_C@_0BO@MEJD@?$CFld?5bytes?5in?5?$CFld?5?$CFhs?5Blocks?4?6?$AA@ 300433f0     LIBCMTD:dbgheap.obj
 0002:00005410       ??_C@_09IGKD@stdenvp?4c?$AA@ 30043410     LIBCMTD:stdenvp.obj
 0002:0000541c       ??_C@_09MPMN@stdargv?4c?$AA@ 3004341c     LIBCMTD:stdargv.obj
 0002:00005428       ??_C@_07BNNE@a_env?4c?$AA@ 30043428     LIBCMTD:a_env.obj
 0002:00005430       ??_C@_0P@GGKG@runtime?5error?5?$AA@ 30043430     LIBCMTD:crt0msg.obj
 0002:00005440       ??_C@_02PIMC@?$AN?6?$AA@   30043440     LIBCMTD:crt0msg.obj
 0002:00005444       ??_C@_0O@DELO@TLOSS?5error?$AN?6?$AA@ 30043444     LIBCMTD:crt0msg.obj
 0002:00005454       ??_C@_0N@OMLL@SING?5error?$AN?6?$AA@ 30043454     LIBCMTD:crt0msg.obj
 0002:00005464       ??_C@_0P@OJAK@DOMAIN?5error?$AN?6?$AA@ 30043464     LIBCMTD:crt0msg.obj
 0002:00005474       ??_C@_0CF@EANP@R6028?$AN?6?9?5unable?5to?5initialize?5he@ 30043474     LIBCMTD:crt0msg.obj
 0002:0000549c       ??_C@_0DF@ECGN@R6027?$AN?6?9?5not?5enough?5space?5for?5lo@ 3004349c     LIBCMTD:crt0msg.obj
 0002:000054d4       ??_C@_0DF@FKAC@R6026?$AN?6?9?5not?5enough?5space?5for?5st@ 300434d4     LIBCMTD:crt0msg.obj
 0002:0000550c       ??_C@_0CG@DPMN@R6025?$AN?6?9?5pure?5virtual?5function?5c@ 3004350c     LIBCMTD:crt0msg.obj
 0002:00005534       ??_C@_0DF@CKIP@R6024?$AN?6?9?5not?5enough?5space?5for?5_o@ 30043534     LIBCMTD:crt0msg.obj
 0002:0000556c       ??_C@_0CJ@GGOE@R6019?$AN?6?9?5unable?5to?5open?5console?5@ 3004356c     LIBCMTD:crt0msg.obj
 0002:00005598       ??_C@_0CB@LBOB@R6018?$AN?6?9?5unexpected?5heap?5error?$AN?6@ 30043598     LIBCMTD:crt0msg.obj
 0002:000055bc       ??_C@_0CN@FPEG@R6017?$AN?6?9?5unexpected?5multithread?5@ 300435bc     LIBCMTD:crt0msg.obj
 0002:000055ec       ??_C@_0CM@OBIC@R6016?$AN?6?9?5not?5enough?5space?5for?5th@ 300435ec     LIBCMTD:crt0msg.obj
 0002:00005618       ??_C@_0CB@HPAL@?$AN?6abnormal?5program?5termination?$AN?6@ 30043618     LIBCMTD:crt0msg.obj
 0002:0000563c       ??_C@_0CM@JOOB@R6009?$AN?6?9?5not?5enough?5space?5for?5en@ 3004363c     LIBCMTD:crt0msg.obj
 0002:00005668       ??_C@_0CK@OIBL@R6008?$AN?6?9?5not?5enough?5space?5for?5ar@ 30043668     LIBCMTD:crt0msg.obj
 0002:00005694       ??_C@_0CF@LKPB@R6002?$AN?6?9?5floating?5point?5not?5load@ 30043694     LIBCMTD:crt0msg.obj
 0002:000056bc       ??_C@_0CF@JPDF@Microsoft?5Visual?5C?$CL?$CL?5Runtime?5Lib@ 300436bc     LIBCMTD:crt0msg.obj
 0002:000056e4       ??_C@_0BK@DEOK@Runtime?5Error?$CB?6?6Program?3?5?$AA@ 300436e4     LIBCMTD:crt0msg.obj
 0002:0000570c       ??_C@_09EMDO@_getbuf?4c?$AA@ 3004370c     LIBCMTD:_getbuf.obj
 0002:00005718       ??_C@_07HPAH@_file?4c?$AA@ 30043718     LIBCMTD:_file.obj
 0002:00005720       ??_C@_09NEAG@sprintf?4c?$AA@ 30043720     LIBCMTD:snprintf.obj
 0002:0000572c       ??_C@_08CNMA@winsig?4c?$AA@ 3004372c     LIBCMTD:winsig.obj
 0002:00005738       ??_C@_0BD@NJFP@GetLastActivePopup?$AA@ 30043738     LIBCMTD:crtmbox.obj
 0002:0000574c       ??_C@_0BA@GILI@GetActiveWindow?$AA@ 3004374c     LIBCMTD:crtmbox.obj
 0002:0000575c       ??_C@_0M@PKCK@MessageBoxA?$AA@ 3004375c     LIBCMTD:crtmbox.obj
 0002:00005768       ??_C@_0L@EEGJ@inittime?4c?$AA@ 30043768     LIBCMTD:inittime.obj
 0002:00005774       ??_C@_09IMJJ@initnum?4c?$AA@ 30043774     LIBCMTD:initnum.obj
 0002:00005780       ??_C@_09KPNI@initmon?4c?$AA@ 30043780     LIBCMTD:initmon.obj
 0002:0000578c       ??_C@_0L@COIL@initctyp?4c?$AA@ 3004378c     LIBCMTD:initctyp.obj
 0002:00005798       ??_C@_08OBJD@Paraguay?$AA@ 30043798     LIBCMTD:getqloc.obj
 0002:000057a4       ??_C@_07GLKH@Uruguay?$AA@  300437a4     LIBCMTD:getqloc.obj
 0002:000057ac       ??_C@_05FPFC@Chile?$AA@    300437ac     LIBCMTD:getqloc.obj
 0002:000057b4       ??_C@_07IIGF@Ecuador?$AA@  300437b4     LIBCMTD:getqloc.obj
 0002:000057bc       ??_C@_09PKAL@Argentina?$AA@ 300437bc     LIBCMTD:getqloc.obj
 0002:000057c8       ??_C@_04LKAH@Peru?$AA@     300437c8     LIBCMTD:getqloc.obj
 0002:000057d0       ??_C@_08NEEM@Colombia?$AA@ 300437d0     LIBCMTD:getqloc.obj
 0002:000057dc       ??_C@_09ODEB@Venezuela?$AA@ 300437dc     LIBCMTD:getqloc.obj
 0002:000057e8       ??_C@_0BD@CLEL@Dominican?5Republic?$AA@ 300437e8     LIBCMTD:getqloc.obj
 0002:000057fc       ??_C@_0N@MDGL@South?5Africa?$AA@ 300437fc     LIBCMTD:getqloc.obj
 0002:0000580c       ??_C@_06NKBG@Panama?$AA@   3004380c     LIBCMTD:getqloc.obj
 0002:00005814       ??_C@_0L@BMHO@Luxembourg?$AA@ 30043814     LIBCMTD:getqloc.obj
 0002:00005820       ??_C@_0L@IMDK@Costa?5Rica?$AA@ 30043820     LIBCMTD:getqloc.obj
 0002:0000582c       ??_C@_0M@BLJF@Switzerland?$AA@ 3004382c     LIBCMTD:getqloc.obj
 0002:00005838       ??_C@_09KBOL@Guatemala?$AA@ 30043838     LIBCMTD:getqloc.obj
 0002:00005844       ??_C@_06JNAK@Canada?$AA@   30043844     LIBCMTD:getqloc.obj
 0002:0000584c       ??_C@_0BG@OLLP@Spanish?5?9?5Modern?5Sort?$AA@ 3004384c     LIBCMTD:getqloc.obj
 0002:00005864       ??_C@_09IDKE@Australia?$AA@ 30043864     LIBCMTD:getqloc.obj
 0002:00005870       ??_C@_07JJJJ@English?$AA@  30043870     LIBCMTD:getqloc.obj
 0002:00005878       ??_C@_07NMDO@Austria?$AA@  30043878     LIBCMTD:getqloc.obj
 0002:00005880       ??_C@_06DEFE@German?$AA@   30043880     LIBCMTD:getqloc.obj
 0002:00005888       ??_C@_07JAIH@Belgium?$AA@  30043888     LIBCMTD:getqloc.obj
 0002:00005890       ??_C@_06BNLJ@Mexico?$AA@   30043890     LIBCMTD:getqloc.obj
 0002:00005898       ??_C@_07JHAG@Spanish?$AA@  30043898     LIBCMTD:getqloc.obj
 0002:000058a0       ??_C@_06DADE@Basque?$AA@   300438a0     LIBCMTD:getqloc.obj
 0002:000058a8       ??_C@_06ENFP@Sweden?$AA@   300438a8     LIBCMTD:getqloc.obj
 0002:000058b0       ??_C@_07JPMH@Swedish?$AA@  300438b0     LIBCMTD:getqloc.obj
 0002:000058b8       ??_C@_07IEKF@Iceland?$AA@  300438b8     LIBCMTD:getqloc.obj
 0002:000058c0       ??_C@_09KNEA@Icelandic?$AA@ 300438c0     LIBCMTD:getqloc.obj
 0002:000058cc       ??_C@_06IJOD@France?$AA@   300438cc     LIBCMTD:getqloc.obj
 0002:000058d4       ??_C@_06EINI@French?$AA@   300438d4     LIBCMTD:getqloc.obj
 0002:000058dc       ??_C@_07FOOE@Finland?$AA@  300438dc     LIBCMTD:getqloc.obj
 0002:000058e4       ??_C@_07OJOM@Finnish?$AA@  300438e4     LIBCMTD:getqloc.obj
 0002:000058ec       ??_C@_05FFAC@Spain?$AA@    300438ec     LIBCMTD:getqloc.obj
 0002:000058f4       ??_C@_0BL@BIHM@Spanish?5?9?5Traditional?5Sort?$AA@ 300438f4     LIBCMTD:getqloc.obj
 0002:00005910       ??_C@_0O@GLHB@united?9states?$AA@ 30043910     LIBCMTD:getqloc.obj
 0002:00005920       ??_C@_0P@IIKK@united?9kingdom?$AA@ 30043920     LIBCMTD:getqloc.obj
 0002:00005930       ??_C@_0BC@FHBO@trinidad?5?$CG?5tobago?$AA@ 30043930     LIBCMTD:getqloc.obj
 0002:00005944       ??_C@_0M@BDFM@south?9korea?$AA@ 30043944     LIBCMTD:getqloc.obj
 0002:00005950       ??_C@_0N@CKFA@south?9africa?$AA@ 30043950     LIBCMTD:getqloc.obj
 0002:00005960       ??_C@_0M@HNHN@south?5korea?$AA@ 30043960     LIBCMTD:getqloc.obj
 0002:0000596c       ??_C@_0N@MKDO@south?5africa?$AA@ 3004396c     LIBCMTD:getqloc.obj
 0002:0000597c       ??_C@_06KFFJ@slovak?$AA@   3004397c     LIBCMTD:getqloc.obj
 0002:00005984       ??_C@_0M@NMAC@puerto?9rico?$AA@ 30043984     LIBCMTD:getqloc.obj
 0002:00005990       ??_C@_08EJOH@pr?9china?$AA@ 30043990     LIBCMTD:getqloc.obj
 0002:0000599c       ??_C@_08CHMG@pr?5china?$AA@ 3004399c     LIBCMTD:getqloc.obj
 0002:000059a8       ??_C@_02OCJK@nz?$AA@       300439a8     LIBCMTD:getqloc.obj
 0002:000059ac       ??_C@_0M@MMKA@new?9zealand?$AA@ 300439ac     LIBCMTD:getqloc.obj
 0002:000059b8       ??_C@_09MGEH@hong?9kong?$AA@ 300439b8     LIBCMTD:getqloc.obj
 0002:000059c4       ??_C@_07CCAK@holland?$AA@  300439c4     LIBCMTD:getqloc.obj
 0002:000059cc       ??_C@_0O@MEPL@great?5britain?$AA@ 300439cc     LIBCMTD:getqloc.obj
 0002:000059dc       ??_C@_07LGIB@england?$AA@  300439dc     LIBCMTD:getqloc.obj
 0002:000059e4       ??_C@_05BMOA@czech?$AA@    300439e4     LIBCMTD:getqloc.obj
 0002:000059ec       ??_C@_05NMPB@china?$AA@    300439ec     LIBCMTD:getqloc.obj
 0002:000059f4       ??_C@_07GN@britain?$AA@    300439f4     LIBCMTD:getqloc.obj
 0002:000059fc       ??_C@_07DLAK@america?$AA@  300439fc     LIBCMTD:getqloc.obj
 0002:00005a04       ??_C@_03IPEP@usa?$AA@      30043a04     LIBCMTD:getqloc.obj
 0002:00005a08       ??_C@_02PILH@us?$AA@       30043a08     LIBCMTD:getqloc.obj
 0002:00005a0c       ??_C@_02FHP@uk?$AA@        30043a0c     LIBCMTD:getqloc.obj
 0002:00005a10       ??_C@_05DEAI@swiss?$AA@    30043a10     LIBCMTD:getqloc.obj
 0002:00005a18       ??_C@_0BA@LIAF@swedish?9finland?$AA@ 30043a18     LIBCMTD:getqloc.obj
 0002:00005a28       ??_C@_0BC@FMEG@spanish?9venezuela?$AA@ 30043a28     LIBCMTD:getqloc.obj
 0002:00005a3c       ??_C@_0BA@BNMG@spanish?9uruguay?$AA@ 30043a3c     LIBCMTD:getqloc.obj
 0002:00005a4c       ??_C@_0BE@BKDJ@spanish?9puerto?5rico?$AA@ 30043a4c     LIBCMTD:getqloc.obj
 0002:00005a60       ??_C@_0N@JIBL@spanish?9peru?$AA@ 30043a60     LIBCMTD:getqloc.obj
 0002:00005a70       ??_C@_0BB@OGOF@spanish?9paraguay?$AA@ 30043a70     LIBCMTD:getqloc.obj
 0002:00005a84       ??_C@_0P@LLFA@spanish?9panama?$AA@ 30043a84     LIBCMTD:getqloc.obj
 0002:00005a94       ??_C@_0BC@BBJM@spanish?9nicaragua?$AA@ 30043a94     LIBCMTD:getqloc.obj
 0002:00005aa8       ??_C@_0P@NJBN@spanish?9modern?$AA@ 30043aa8     LIBCMTD:getqloc.obj
 0002:00005ab8       ??_C@_0BA@NHDN@spanish?9mexican?$AA@ 30043ab8     LIBCMTD:getqloc.obj
 0002:00005ac8       ??_C@_0BB@JHOJ@spanish?9honduras?$AA@ 30043ac8     LIBCMTD:getqloc.obj
 0002:00005adc       ??_C@_0BC@BOOM@spanish?9guatemala?$AA@ 30043adc     LIBCMTD:getqloc.obj
 0002:00005af0       ??_C@_0BE@EELI@spanish?9el?5salvador?$AA@ 30043af0     LIBCMTD:getqloc.obj
 0002:00005b04       ??_C@_0BA@POAE@spanish?9ecuador?$AA@ 30043b04     LIBCMTD:getqloc.obj
 0002:00005b14       ??_C@_0BL@LDKN@spanish?9dominican?5republic?$AA@ 30043b14     LIBCMTD:getqloc.obj
 0002:00005b30       ??_C@_0BD@HPMH@spanish?9costa?5rica?$AA@ 30043b30     LIBCMTD:getqloc.obj
 0002:00005b44       ??_C@_0BB@NDDK@spanish?9colombia?$AA@ 30043b44     LIBCMTD:getqloc.obj
 0002:00005b58       ??_C@_0O@BJHA@spanish?9chile?$AA@ 30043b58     LIBCMTD:getqloc.obj
 0002:00005b68       ??_C@_0BA@OBNG@spanish?9bolivia?$AA@ 30043b68     LIBCMTD:getqloc.obj
 0002:00005b78       ??_C@_0BC@EFAM@spanish?9argentina?$AA@ 30043b78     LIBCMTD:getqloc.obj
 0002:00005b8c       ??_C@_0BF@KMMM@portuguese?9brazilian?$AA@ 30043b8c     LIBCMTD:getqloc.obj
 0002:00005ba4       ??_C@_0BC@BAAE@norwegian?9nynorsk?$AA@ 30043ba4     LIBCMTD:getqloc.obj
 0002:00005bb8       ??_C@_0BB@PBHK@norwegian?9bokmal?$AA@ 30043bb8     LIBCMTD:getqloc.obj
 0002:00005bcc       ??_C@_09EHKL@norwegian?$AA@ 30043bcc     LIBCMTD:getqloc.obj
 0002:00005bd8       ??_C@_0O@BEAN@italian?9swiss?$AA@ 30043bd8     LIBCMTD:getqloc.obj
 0002:00005be8       ??_C@_0O@OIFK@irish?9english?$AA@ 30043be8     LIBCMTD:getqloc.obj
 0002:00005bf8       ??_C@_0N@NBPL@german?9swiss?$AA@ 30043bf8     LIBCMTD:getqloc.obj
 0002:00005c08       ??_C@_0BC@ICFJ@german?9luxembourg?$AA@ 30043c08     LIBCMTD:getqloc.obj
 0002:00005c1c       ??_C@_0BE@GGPC@german?9lichtenstein?$AA@ 30043c1c     LIBCMTD:getqloc.obj
 0002:00005c30       ??_C@_0BA@MKDC@german?9austrian?$AA@ 30043c30     LIBCMTD:getqloc.obj
 0002:00005c40       ??_C@_0N@ODNB@french?9swiss?$AA@ 30043c40     LIBCMTD:getqloc.obj
 0002:00005c50       ??_C@_0BC@MGCM@french?9luxembourg?$AA@ 30043c50     LIBCMTD:getqloc.obj
 0002:00005c64       ??_C@_0BA@NABK@french?9canadian?$AA@ 30043c64     LIBCMTD:getqloc.obj
 0002:00005c74       ??_C@_0P@CJNO@french?9belgian?$AA@ 30043c74     LIBCMTD:getqloc.obj
 0002:00005c84       ??_C@_0M@LJOL@english?9usa?$AA@ 30043c84     LIBCMTD:getqloc.obj
 0002:00005c90       ??_C@_0L@FMNC@english?9us?$AA@ 30043c90     LIBCMTD:getqloc.obj
 0002:00005c9c       ??_C@_0L@KBBK@english?9uk?$AA@ 30043c9c     LIBCMTD:getqloc.obj
 0002:00005ca8       ??_C@_0BK@NDDE@english?9trinidad?5y?5tobago?$AA@ 30043ca8     LIBCMTD:getqloc.obj
 0002:00005cc4       ??_C@_0BF@LKML@english?9south?5africa?$AA@ 30043cc4     LIBCMTD:getqloc.obj
 0002:00005cdc       ??_C@_0L@EGPP@english?9nz?$AA@ 30043cdc     LIBCMTD:getqloc.obj
 0002:00005ce8       ??_C@_0BA@HLH@english?9jamaica?$AA@ 30043ce8     LIBCMTD:getqloc.obj
 0002:00005cf8       ??_C@_0M@PMJI@english?9ire?$AA@ 30043cf8     LIBCMTD:getqloc.obj
 0002:00005d04       ??_C@_0BC@HINE@english?9caribbean?$AA@ 30043d04     LIBCMTD:getqloc.obj
 0002:00005d18       ??_C@_0M@DCFH@english?9can?$AA@ 30043d18     LIBCMTD:getqloc.obj
 0002:00005d24       ??_C@_0P@DGHK@english?9belize?$AA@ 30043d24     LIBCMTD:getqloc.obj
 0002:00005d34       ??_C@_0M@FLHK@english?9aus?$AA@ 30043d34     LIBCMTD:getqloc.obj
 0002:00005d40       ??_C@_0BB@HNCK@english?9american?$AA@ 30043d40     LIBCMTD:getqloc.obj
 0002:00005d54       ??_C@_0O@PAMI@dutch?9belgian?$AA@ 30043d54     LIBCMTD:getqloc.obj
 0002:00005d64       ??_C@_0BE@FPEJ@chinese?9traditional?$AA@ 30043d64     LIBCMTD:getqloc.obj
 0002:00005d78       ??_C@_0BC@CHFL@chinese?9singapore?$AA@ 30043d78     LIBCMTD:getqloc.obj
 0002:00005d8c       ??_C@_0BD@DCMH@chinese?9simplified?$AA@ 30043d8c     LIBCMTD:getqloc.obj
 0002:00005da0       ??_C@_0BB@JMOE@chinese?9hongkong?$AA@ 30043da0     LIBCMTD:getqloc.obj
 0002:00005db4       ??_C@_07NGFN@chinese?$AA@  30043db4     LIBCMTD:getqloc.obj
 0002:00005dbc       ??_C@_03PCOI@chi?$AA@      30043dbc     LIBCMTD:getqloc.obj
 0002:00005dc0       ??_C@_03FIHP@chh?$AA@      30043dc0     LIBCMTD:getqloc.obj
 0002:00005dc4       ??_C@_08HFLO@canadian?$AA@ 30043dc4     LIBCMTD:getqloc.obj
 0002:00005dd0       ??_C@_07INIJ@belgian?$AA@  30043dd0     LIBCMTD:getqloc.obj
 0002:00005dd8       ??_C@_0L@LCCA@australian?$AA@ 30043dd8     LIBCMTD:getqloc.obj
 0002:00005de4       ??_C@_0BB@BJIO@american?9english?$AA@ 30043de4     LIBCMTD:getqloc.obj
 0002:00005df8       ??_C@_0BB@DAGO@american?5english?$AA@ 30043df8     LIBCMTD:getqloc.obj
 0002:00005e0c       ??_C@_08HENB@american?$AA@ 30043e0c     LIBCMTD:getqloc.obj
 0002:00005e18       ??_C@_03DGJE@OCP?$AA@      30043e18     LIBCMTD:getqloc.obj
 0002:00005e1c       ??_C@_03EKFG@ACP?$AA@      30043e1c     LIBCMTD:getqloc.obj
 0002:00005e20       ??_C@_06PAPI@1?$CDQNAN?$AA@ 30043e20     LIBCMTD:x10fout.obj
 0002:00005e28       ??_C@_05BGNL@1?$CDINF?$AA@ 30043e28     LIBCMTD:x10fout.obj
 0002:00005e30       ??_C@_05EDPF@1?$CDIND?$AA@ 30043e30     LIBCMTD:x10fout.obj
 0002:00005e38       ??_C@_06LKFM@1?$CDSNAN?$AA@ 30043e38     LIBCMTD:x10fout.obj
 0002:00005e40       ??_C@_09LNLM@osfinfo?4c?$AA@ 30043e40     LIBCMTD:osfinfo.obj
 0002:00005e4c       ??_C@_07CJME@H?3mm?3ss?$AA@ 30043e4c     LIBCMTD:strftime.obj
 0002:00005e54       ??_C@_0BE@MHI@dddd?0?5MMMM?5dd?0?5yyyy?$AA@ 30043e54     LIBCMTD:strftime.obj
 0002:00005e68       ??_C@_06HCAD@M?1d?1yy?$AA@ 30043e68     LIBCMTD:strftime.obj
 0002:00005e70       ??_C@_02DBLP@PM?$AA@       30043e70     LIBCMTD:strftime.obj
 0002:00005e74       ??_C@_02ENLM@AM?$AA@       30043e74     LIBCMTD:strftime.obj
 0002:00005e78       ??_C@_08LIDF@December?$AA@ 30043e78     LIBCMTD:strftime.obj
 0002:00005e84       ??_C@_08NJLI@November?$AA@ 30043e84     LIBCMTD:strftime.obj
 0002:00005e90       ??_C@_07IAMM@October?$AA@  30043e90     LIBCMTD:strftime.obj
 0002:00005e98       ??_C@_09MKGD@September?$AA@ 30043e98     LIBCMTD:strftime.obj
 0002:00005ea4       ??_C@_06PADP@August?$AA@   30043ea4     LIBCMTD:strftime.obj
 0002:00005eac       ??_C@_04PIJO@July?$AA@     30043eac     LIBCMTD:strftime.obj
 0002:00005eb4       ??_C@_04ICFP@June?$AA@     30043eb4     LIBCMTD:strftime.obj
 0002:00005ebc       ??_C@_05JFGC@April?$AA@    30043ebc     LIBCMTD:strftime.obj
 0002:00005ec4       ??_C@_05FGPD@March?$AA@    30043ec4     LIBCMTD:strftime.obj
 0002:00005ecc       ??_C@_08PGBA@February?$AA@ 30043ecc     LIBCMTD:strftime.obj
 0002:00005ed8       ??_C@_07BPKJ@January?$AA@  30043ed8     LIBCMTD:strftime.obj
 0002:00005ee0       ??_C@_03PGJO@Dec?$AA@      30043ee0     LIBCMTD:strftime.obj
 0002:00005ee4       ??_C@_03PDLM@Nov?$AA@      30043ee4     LIBCMTD:strftime.obj
 0002:00005ee8       ??_C@_03BLHK@Oct?$AA@      30043ee8     LIBCMTD:strftime.obj
 0002:00005eec       ??_C@_03DPFM@Sep?$AA@      30043eec     LIBCMTD:strftime.obj
 0002:00005ef0       ??_C@_03CMCH@Aug?$AA@      30043ef0     LIBCMTD:strftime.obj
 0002:00005ef4       ??_C@_03OBKI@Jul?$AA@      30043ef4     LIBCMTD:strftime.obj
 0002:00005ef8       ??_C@_03LEIG@Jun?$AA@      30043ef8     LIBCMTD:strftime.obj
 0002:00005efc       ??_C@_03MGHB@May?$AA@      30043efc     LIBCMTD:strftime.obj
 0002:00005f00       ??_C@_03MJJM@Apr?$AA@      30043f00     LIBCMTD:strftime.obj
 0002:00005f04       ??_C@_03GNHA@Mar?$AA@      30043f04     LIBCMTD:strftime.obj
 0002:00005f08       ??_C@_03PICE@Feb?$AA@      30043f08     LIBCMTD:strftime.obj
 0002:00005f0c       ??_C@_03IEIF@Jan?$AA@      30043f0c     LIBCMTD:strftime.obj
 0002:00005f10       ??_C@_08FAKH@Saturday?$AA@ 30043f10     LIBCMTD:strftime.obj
 0002:00005f1c       ??_C@_06ONCK@Friday?$AA@   30043f1c     LIBCMTD:strftime.obj
 0002:00005f24       ??_C@_08CCFO@Thursday?$AA@ 30043f24     LIBCMTD:strftime.obj
 0002:00005f30       ??_C@_09PBIN@Wednesday?$AA@ 30043f30     LIBCMTD:strftime.obj
 0002:00005f3c       ??_C@_07BMBC@Tuesday?$AA@  30043f3c     LIBCMTD:strftime.obj
 0002:00005f44       ??_C@_06CHLK@Monday?$AA@   30043f44     LIBCMTD:strftime.obj
 0002:00005f4c       ??_C@_06OOEM@Sunday?$AA@   30043f4c     LIBCMTD:strftime.obj
 0002:00005f54       ??_C@_03MPKK@Sat?$AA@      30043f54     LIBCMTD:strftime.obj
 0002:00005f58       ??_C@_03FINJ@Fri?$AA@      30043f58     LIBCMTD:strftime.obj
 0002:00005f5c       ??_C@_03HIKC@Thu?$AA@      30043f5c     LIBCMTD:strftime.obj
 0002:00005f60       ??_C@_03HECK@Wed?$AA@      30043f60     LIBCMTD:strftime.obj
 0002:00005f64       ??_C@_03ECCP@Tue?$AA@      30043f64     LIBCMTD:strftime.obj
 0002:00005f68       ??_C@_03PIEP@Mon?$AA@      30043f68     LIBCMTD:strftime.obj
 0002:00005f6c       ??_C@_03FHEP@Sun?$AA@      30043f6c     LIBCMTD:strftime.obj
 0002:00005f70       ??_C@_03MKGK@a?1p?$AA@     30043f70     LIBCMTD:strftime.obj
 0002:00005f74       ??_C@_05BDJK@am?1pm?$AA@   30043f74     LIBCMTD:strftime.obj
 0002:00005f7c       ??_C@_0L@HKCB@inithelp?4c?$AA@ 30043f7c     LIBCMTD:inithelp.obj
 0002:00005fa0       ??_C@_08PHBD@fclose?4c?$AA@ 30043fa0     LIBCMTD:fclose.obj
 0002:00005fac       ??_C@_0P@FHEA@stream?5?$CB?$DN?5NULL?$AA@ 30043fac     LIBCMTD:fclose.obj
 0002:00005fbc       ___dnames                  30043fbc     LIBCMTD:timeset.obj
 0002:00005fd4       ___mnames                  30043fd4     LIBCMTD:timeset.obj
 0002:00005ffc       ??_C@_07DEKI@tzset?4c?$AA@ 30043ffc     LIBCMTD:tzset.obj
 0002:00006004       ??_C@_02JHIA@TZ?$AA@       30044004     LIBCMTD:tzset.obj
 0002:00006024       ??_C@_0L@JIE@_freebuf?4c?$AA@ 30044024     LIBCMTD:_freebuf.obj
 0002:00006030       ??_C@_0L@EJNO@wtombenv?4c?$AA@ 30044030     LIBCMTD:wtombenv.obj
 0002:0000603c       ??_C@_07FOIK@a_cmp?4c?$AA@ 3004403c     LIBCMTD:a_cmp.obj
 0002:00006044       ??_C@_0DN@PPKB@cchCount1?$DN?$DN0?5?$CG?$CG?5cchCount2?$DN?$DN1?5?$HM?$HM?5@ 30044044     LIBCMTD:a_cmp.obj
 0002:000060a0       ??_C@_08FEIK@setenv?4c?$AA@ 300440a0     LIBCMTD:setenv.obj
 0003:00000000       ___xc_a                    30045000     LIBCMTD:crt0init.obj
 0003:00000004       ___xc_z                    30045004     LIBCMTD:crt0init.obj
 0003:00000008       ___xi_a                    30045008     LIBCMTD:crt0init.obj
 0003:00000014       ___xi_z                    30045014     LIBCMTD:crt0init.obj
 0003:00000018       ___xp_a                    30045018     LIBCMTD:crt0init.obj
 0003:00000020       ___xp_z                    30045020     LIBCMTD:crt0init.obj
 0003:00000024       ___xt_a                    30045024     LIBCMTD:crt0init.obj
 0003:00000028       ___xt_z                    30045028     LIBCMTD:crt0init.obj
 0003:00000030       _bg_itemlist               30045030     bg_misc.obj
 0003:000008b8       _bg_numItems               300458b8     bg_misc.obj
 0003:000008bc       _pm_stopspeed              300458bc     bg_pmove.obj
 0003:000008c0       _pm_duckScale              300458c0     bg_pmove.obj
 0003:000008c4       _pm_swimScale              300458c4     bg_pmove.obj
 0003:000008c8       _pm_wadeScale              300458c8     bg_pmove.obj
 0003:000008cc       _pm_accelerate             300458cc     bg_pmove.obj
 0003:000008d0       _pm_airaccelerate          300458d0     bg_pmove.obj
 0003:000008d4       _pm_wateraccelerate        300458d4     bg_pmove.obj
 0003:000008d8       _pm_flyaccelerate          300458d8     bg_pmove.obj
 0003:000008dc       _pm_friction               300458dc     bg_pmove.obj
 0003:000008e0       _pm_waterfriction          300458e0     bg_pmove.obj
 0003:000008e4       _pm_flightfriction         300458e4     bg_pmove.obj
 0003:00000988       _drawTeamOverlayModificationCount 30045988     cg_draw.obj
 0003:00001168       _cvarTable                 30046168     cg_main.obj
 0003:00001618       _cvarTableSize             30046618     cg_main.obj
 0003:00001648       _cg_customSoundNames       30046648     cg_players.obj
 0003:00001704       _axisDefault               30046704     q_math.obj
 0003:00001728       _colorBlack                30046728     q_math.obj
 0003:00001738       _colorRed                  30046738     q_math.obj
 0003:00001748       _colorGreen                30046748     q_math.obj
 0003:00001758       _colorBlue                 30046758     q_math.obj
 0003:00001768       _colorYellow               30046768     q_math.obj
 0003:00001778       _colorMagenta              30046778     q_math.obj
 0003:00001788       _colorCyan                 30046788     q_math.obj
 0003:00001798       _colorWhite                30046798     q_math.obj
 0003:000017a8       _colorLtGrey               300467a8     q_math.obj
 0003:000017b8       _colorMdGrey               300467b8     q_math.obj
 0003:000017c8       _colorDkGrey               300467c8     q_math.obj
 0003:000017d8       _g_color_table             300467d8     q_math.obj
 0003:00001858       _bytedirs                  30046858     q_math.obj
 0003:00002004       __fltused                  30047004     LIBCMTD:fpinit.obj
 0003:00002008       __ldused                   30047008     LIBCMTD:fpinit.obj
 0003:0000200c       __FPinit                   3004700c     LIBCMTD:fpinit.obj
 0003:00002010       __FPmtinit                 30047010     LIBCMTD:fpinit.obj
 0003:00002014       __FPmtterm                 30047014     LIBCMTD:fpinit.obj
 0003:00002030       __aexit_rtn                30047030     LIBCMTD:dllcrt0.obj
 0003:00002040       __indefinite               30047040     LIBCMTD:87disp.obj
 0003:0000204a       __piby2                    3004704a     LIBCMTD:87disp.obj
 0003:00002070       __cfltcvt_tab              30047070     LIBCMTD:cmiscdat.obj
 0003:00002088       __pctype                   30047088     LIBCMTD:ctype.obj
 0003:0000208c       __pwctype                  3004708c     LIBCMTD:ctype.obj
 0003:00002090       __ctype                    30047090     LIBCMTD:ctype.obj
 0003:00002294       ___mb_cur_max              30047294     LIBCMTD:nlsdata1.obj
 0003:00002298       ___decimal_point           30047298     LIBCMTD:nlsdata1.obj
 0003:0000229c       ___decimal_point_length    3004729c     LIBCMTD:nlsdata1.obj
 0003:00002378       __d_inf                    30047378     LIBCMTD:util.obj
 0003:00002380       __d_ind                    30047380     LIBCMTD:util.obj
 0003:00002388       __d_max                    30047388     LIBCMTD:util.obj
 0003:00002390       __d_min                    30047390     LIBCMTD:util.obj
 0003:00002398       __d_mzero                  30047398     LIBCMTD:util.obj
 0003:000023b8       ___nullstring              300473b8     LIBCMTD:output.obj
 0003:000023bc       ___wnullstring             300473bc     LIBCMTD:output.obj
 0003:000023c0       __crtAssertBusy            300473c0     LIBCMTD:dbgrpt.obj
 0003:000023c4       __CrtDbgMode               300473c4     LIBCMTD:dbgrpt.obj
 0003:000023d0       __CrtDbgFile               300473d0     LIBCMTD:dbgrpt.obj
 0003:000023f0       __OP_ATAN2jmptab           300473f0     LIBCMTD:87triga.obj
 0003:00002440       __locktable                30047440     LIBCMTD:mlock.obj
 0003:00002610       ___lc_category             30047610     LIBCMTD:setlocal.obj
 0003:00002658       ___tlsindex                30047658     LIBCMTD:tidtable.obj
 0003:00002660       ___badioinfo               30047660     LIBCMTD:ioinit.obj
 0003:00002684       __crtDbgFlag               30047684     LIBCMTD:dbgheap.obj
 0003:0000268c       __crtBreakAlloc            3004768c     LIBCMTD:dbgheap.obj
 0003:000026a8       __amblksiz                 300476a8     LIBCMTD:heapinit.obj
 0003:000028d8       __matherr_flag             300478d8     LIBCMTD:matherr.obj
 0003:000028e0       __iob                      300478e0     LIBCMTD:_file.obj
 0003:00002b60       ___rgLocInfo               30047b60     LIBCMTD:getqloc.obj
 0003:00003004       ___rglangidNotDefault      30048004     LIBCMTD:getqloc.obj
 0003:00003018       ___rg_country              30048018     LIBCMTD:getqloc.obj
 0003:000030d0       ___rg_language             300480d0     LIBCMTD:getqloc.obj
 0003:000032d8       __NLG_Destination          300482d8     LIBCMTD:exsup.obj
 0003:000032e8       __XcptActTab               300482e8     LIBCMTD:winxfltr.obj
 0003:00003360       __First_FPE_Indx           30048360     LIBCMTD:winxfltr.obj
 0003:00003364       __Num_FPE                  30048364     LIBCMTD:winxfltr.obj
 0003:00003368       __XcptActTabSize           30048368     LIBCMTD:winxfltr.obj
 0003:0000336c       __XcptActTabCount          3004836c     LIBCMTD:winxfltr.obj
 0003:00003370       __pfnAllocHook             30048370     LIBCMTD:dbghook.obj
 0003:00003374       ___sbh_threshold           30048374     LIBCMTD:sbheap.obj
 0003:00003470       ___lc_time_curr            30048470     LIBCMTD:strftime.obj
 0003:00003478       ___lc_time_c               30048478     LIBCMTD:strftime.obj
 0003:00003528       ___lconv_static_decimal    30048528     LIBCMTD:lconv.obj
 0003:00003530       ___lconv_c                 30048530     LIBCMTD:lconv.obj
 0003:00003560       ___lconv                   30048560     LIBCMTD:lconv.obj
 0003:00003570       __timezone                 30048570     LIBCMTD:timeset.obj
 0003:00003574       __daylight                 30048574     LIBCMTD:timeset.obj
 0003:00003578       __dstbias                  30048578     LIBCMTD:timeset.obj
 0003:000035fc       __tzname                   300485fc     LIBCMTD:timeset.obj
 0003:00003628       __pow10pos                 30048628     LIBCMTD:constpow.obj
 0003:00003788       __pow10neg                 30048788     LIBCMTD:constpow.obj
 0003:000038e4       __lpdays                   300488e4     LIBCMTD:days.obj
 0003:00003918       __days                     30048918     LIBCMTD:days.obj
 0003:00003954       _c_pmove                   30048954     bg_pmove.obj
 0003:00004794       _vec3_origin               30049794     q_math.obj
 0003:00014dc4       ___fastflag                30059dc4     LIBCMTD:fpinit.obj
 0003:00014dc8       __adjust_fdiv              30059dc8     LIBCMTD:fpinit.obj
 0003:00014dd0       __aenvptr                  30059dd0     LIBCMTD:dllcrt0.obj
 0003:00014dd4       __wenvptr                  30059dd4     LIBCMTD:dllcrt0.obj
 0003:00014dd8       ___error_mode              30059dd8     LIBCMTD:dllcrt0.obj
 0003:00014ddc       ___app_type                30059ddc     LIBCMTD:dllcrt0.obj
 0003:00014e54       ___lc_handle               30059e54     LIBCMTD:nlsdata2.obj
 0003:00014e6c       ___lc_codepage             30059e6c     LIBCMTD:nlsdata2.obj
 0003:00014e70       ___lc_collate_cp           30059e70     LIBCMTD:nlsdata2.obj
 0003:00014e78       __umaskval                 30059e78     LIBCMTD:crt0dat.obj
 0003:00014e7c       __osver                    30059e7c     LIBCMTD:crt0dat.obj
 0003:00014e80       __winver                   30059e80     LIBCMTD:crt0dat.obj
 0003:00014e84       __winmajor                 30059e84     LIBCMTD:crt0dat.obj
 0003:00014e88       __winminor                 30059e88     LIBCMTD:crt0dat.obj
 0003:00014e8c       ___argc                    30059e8c     LIBCMTD:crt0dat.obj
 0003:00014e90       ___argv                    30059e90     LIBCMTD:crt0dat.obj
 0003:00014e94       ___wargv                   30059e94     LIBCMTD:crt0dat.obj
 0003:00014e98       __environ                  30059e98     LIBCMTD:crt0dat.obj
 0003:00014e9c       ___initenv                 30059e9c     LIBCMTD:crt0dat.obj
 0003:00014ea0       __wenviron                 30059ea0     LIBCMTD:crt0dat.obj
 0003:00014ea4       ___winitenv                30059ea4     LIBCMTD:crt0dat.obj
 0003:00014ea8       __pgmptr                   30059ea8     LIBCMTD:crt0dat.obj
 0003:00014eac       __wpgmptr                  30059eac     LIBCMTD:crt0dat.obj
 0003:00014eb0       __exitflag                 30059eb0     LIBCMTD:crt0dat.obj
 0003:00014eb4       __C_Termination_Done       30059eb4     LIBCMTD:crt0dat.obj
 0003:00014eb8       __C_Exit_Done              30059eb8     LIBCMTD:crt0dat.obj
 0003:00014fdc       __adbgmsg                  30059fdc     LIBCMTD:crt0msg.obj
 0003:00014fe4       __cflush                   30059fe4     LIBCMTD:_file.obj
 0003:00015008       ___lc_time_intl            3005a008     LIBCMTD:inittime.obj
 0003:00015024       ___lc_id                   3005a024     LIBCMTD:nlsdata3.obj
 0003:0001506c       __newmode                  3005a06c     LIBCMTD:_newmode.obj
 0003:00015070       ?_pnhHeap@@3P6AHI@ZA       3005a070     LIBCMTD:handler.obj
 0003:00015080       ___lconv_static_null       3005a080     LIBCMTD:lconv.obj
 0003:00015150       _cg_freeMarkPolys          3005a150     <common>
 0003:00015160       _cg_activeMarkPolys        3005a160     <common>
 0003:00015280       _cg_markPolys              3005a280     <common>
 0003:00027280       _cg_BigHeadScale           3006c280     <common>
 0003:000273a0       _cg_railLength             3006c3a0     <common>
 0003:000274c0       _cg_BobItems               3006c4c0     <common>
 0003:000275e0       _cg_deferPlayers           3006c5e0     <common>
 0003:00027700       _cg_crosshairSize          3006c700     <common>
 0003:00027820       _cg_teamChatTime           3006c820     <common>
 0003:00027940       _cg_simpleItems            3006c940     <common>
 0003:00027a60       _cgs                       3006ca60     <common>
 0003:00051780       _cg_drawTeamOverlay        30096780     <common>
 0003:000518a0       _cg_predictItems           300968a0     <common>
 0003:000519c0       _cg_showmiss               300969c0     <common>
 0003:00051ae0       _cg_tracerChance           30096ae0     <common>
 0003:00051c00       _cg_drawFPS                30096c00     <common>
 0003:00051d20       _cg_viewsize               30096d20     <common>
 0003:00051e40       _cg_railWidth              30096e40     <common>
 0003:00051f60       _cg_drawCrosshair          30096f60     <common>
 0003:00052080       _cg_crosshairHealth        30097080     <common>
 0003:000521a0       _cl_autoaim                300971a0     <common>
 0003:000522c0       _cg_gun_x                  300972c0     <common>
 0003:000523e0       _cg_gun_y                  300973e0     <common>
 0003:00052500       _cg_errorDecay             30097500     <common>
 0003:00052620       _cg_crosshairX             30097620     <common>
 0003:00052740       _cg_drawAttacker           30097740     <common>
 0003:00052860       _cg_autoswitch             30097860     <common>
 0003:00052980       _cg_tracerLength           30097980     <common>
 0003:00052aa0       _cg_gun_z                  30097aa0     <common>
 0003:00052bc0       _cg_stats                  30097bc0     <common>
 0003:00052ce0       _cg_zoomFov                30097ce0     <common>
 0003:00052e00       _cg_forceModel             30097e00     <common>
 0003:00052f20       _cg_animSpeed              30097f20     <common>
 0003:00053040       _cg_debugEvents            30098040     <common>
 0003:00053160       _cg_thirdPerson            30098160     <common>
 0003:00053280       _cg_swingSpeed             30098280     <common>
 0003:000533a0       _cg_addMarks               300983a0     <common>
 0003:000534c0       _cg_blood                  300984c0     <common>
 0003:000535e0       _cg_teamChatHeight         300985e0     <common>
 0003:00053700       _cg_bobup                  30098700     <common>
 0003:00053820       _cg_drawAmmoWarning        30098820     <common>
 0003:00053940       _cg_paused                 30098940     <common>
 0003:00053a60       _cg_draw3dIcons            30098a60     <common>
 0003:00053b80       _cg_thirdPersonAngle       30098b80     <common>
 0003:00053ca0       _cg_drawGun                30098ca0     <common>
 0003:00053dc0       _cg_stereoSeparation       30098dc0     <common>
 0003:00053ee0       _cg_debugAnim              30098ee0     <common>
 0003:00054000       _cg_runpitch               30099000     <common>
 0003:00054120       _cg                        30099120     <common>
 0003:0006f7a0       _cg_teamOverlayUserinfo    300b47a0     <common>
 0003:0006f8c0       _cg_drawCrosshairNames     300b48c0     <common>
 0003:0006f9e0       _cg_syncronousClients      300b49e0     <common>
 0003:0006fb00       _cg_railTrailTime          300b4b00     <common>
 0003:0006fc20       _cg_tracerWidth            300b4c20     <common>
 0003:0006fd40       _cg_items                  300b4d40     <common>
 0003:00071540       _cg_drawTimer              300b6540     <common>
 0003:00071660       _cg_noPlayerAnims          300b6660     <common>
 0003:00071780       _cg_ScaleWeapons           300b6780     <common>
 0003:000718a0       _cg_weapons                300b68a0     <common>
 0003:000720e0       _cg_debugPosition          300b70e0     <common>
 0003:00072200       _cg_draw2D                 300b7200     <common>
 0003:00072320       _cg_bobpitch               300b7320     <common>
 0003:00072440       _cg_fov                    300b7440     <common>
 0003:00072560       _cg_buildScript            300b7560     <common>
 0003:00072680       _cg_drawSnapshot           300b7680     <common>
 0003:000727a0       _cg_centertime             300b77a0     <common>
 0003:000728c0       _cg_thirdPersonRange       300b78c0     <common>
 0003:000729e0       _cg_gibs                   300b79e0     <common>
 0003:00072b00       _cg_crosshairY             300b7b00     <common>
 0003:00072c20       _cg_drawIcons              300b7c20     <common>
 0003:00072d40       _cg_drawStatus             300b7d40     <common>
 0003:00072e60       _cg_CoolRailGun            300b7e60     <common>
 0003:00072f80       _cg_gun_frame              300b7f80     <common>
 0003:000730a0       _cg_ignore                 300b80a0     <common>
 0003:000731c0       _cg_runroll                300b81c0     <common>
 0003:000732e0       _cg_drawRewards            300b82e0     <common>
 0003:00073400       _cg_bobroll                300b8400     <common>
 0003:00073520       _cg_nopredict              300b8520     <common>
 0003:00073640       _cg_shadows                300b8640     <common>
 0003:00073760       _cg_footsteps              300b8760     <common>
 0003:00073880       _cg_entities               300b8880     <common>
 0003:0011d880       _cg_brassTime              30162880     <common>
 0003:0011d9a0       _cg_lagometer              301629a0     <common>
 0003:0011dac0       _cg_SphericalExplosions    30162ac0     <common>
 0003:0011dbe0       _cg_activeLocalEntities    30162be0     <common>
 0003:0011dd00       _cg_freeLocalEntities      30162d00     <common>
 0003:0011dd20       _cg_localEntities          30162d20     <common>
 0003:00141d20       _sortedTeamPlayers         30186d20     <common>
 0003:00141d40       _lagometer                 30186d40     <common>
 0003:00142348       _numSortedTeamPlayers      30187348     <common>
 0003:00142360       _pml                       30187360     <common>
 0003:001423ec       _pm                        301873ec     <common>
 0003:001423f0       ___alternate_form          301873f0     <common>
 0003:001423f4       ___no_lead_zeros           301873f4     <common>
 0003:001423f8       ___mbcodepage              301873f8     <common>
 0003:00142400       ___mbulinfo                30187400     <common>
 0003:0014240c       ___ismbcodepage            3018740c     <common>
 0003:00142420       __mbcasemap                30187420     <common>
 0003:00142520       __mbctype                  30187520     <common>
 0003:00142624       ___mblcid                  30187624     <common>
 0003:00142628       ___sbh_sizeHeaderList      30187628     <common>
 0003:0014262c       ___sbh_indGroupDefer       3018762c     <common>
 0003:00142630       ___sbh_pHeaderScan         30187630     <common>
 0003:00142634       ___sbh_pHeaderDefer        30187634     <common>
 0003:00142638       ___sbh_cntHeaderList       30187638     <common>
 0003:0014263c       ___sbh_pHeaderList         3018763c     <common>
 0003:00142640       ___piob                    30187640     <common>
 0003:00142660       __bufin                    30187660     <common>
 0003:00143660       __nstream                  30188660     <common>
 0003:00143664       __crtheap                  30188664     <common>
 0003:00143668       __pfnDumpClient            30188668     <common>
 0003:00143680       ___pioinfo                 30188680     <common>
 0003:00143780       __nhandle                  30188780     <common>
 0003:00143784       ___env_initialized         30188784     <common>
 0003:00143788       ___mbctype_initialized     30188788     <common>
 0003:0014378c       ___onexitend               3018878c     <common>
 0003:00143790       ___onexitbegin             30188790     <common>
 0003:00143794       ___setlc_active            30188794     <common>
 0003:00143798       ___unguarded_readlc_active 30188798     <common>
 0003:0014379c       __pfnReportHook            3018879c     <common>
 0003:001437a0       __acmdln                   301887a0     <common>
 0003:001437a4       __pRawDllMain              301887a4     <common>
 0004:00000000       __IMPORT_DESCRIPTOR_KERNEL32 30189000     kernel32:KERNEL32.dll
 0004:00000014       __NULL_IMPORT_DESCRIPTOR   30189014     kernel32:KERNEL32.dll
 0004:00000154       __imp__IsBadWritePtr@8     30189154     kernel32:KERNEL32.dll
 0004:00000158       __imp__InterlockedIncrement@4 30189158     kernel32:KERNEL32.dll
 0004:0000015c       __imp__GetCommandLineA@0   3018915c     kernel32:KERNEL32.dll
 0004:00000160       __imp__GetVersion@0        30189160     kernel32:KERNEL32.dll
 0004:00000164       __imp__GetProcAddress@8    30189164     kernel32:KERNEL32.dll
 0004:00000168       __imp__GetModuleHandleA@4  30189168     kernel32:KERNEL32.dll
 0004:0000016c       __imp__RaiseException@16   3018916c     kernel32:KERNEL32.dll
 0004:00000170       __imp__DebugBreak@0        30189170     kernel32:KERNEL32.dll
 0004:00000174       __imp__GetStdHandle@4      30189174     kernel32:KERNEL32.dll
 0004:00000178       __imp__WriteFile@20        30189178     kernel32:KERNEL32.dll
 0004:0000017c       __imp__OutputDebugStringA@4 3018917c     kernel32:KERNEL32.dll
 0004:00000180       __imp__LoadLibraryA@4      30189180     kernel32:KERNEL32.dll
 0004:00000184       __imp__GetModuleFileNameA@12 30189184     kernel32:KERNEL32.dll
 0004:00000188       __imp__InitializeCriticalSection@4 30189188     kernel32:KERNEL32.dll
 0004:0000018c       __imp__DeleteCriticalSection@4 3018918c     kernel32:KERNEL32.dll
 0004:00000190       __imp__EnterCriticalSection@4 30189190     kernel32:KERNEL32.dll
 0004:00000194       __imp__LeaveCriticalSection@4 30189194     kernel32:KERNEL32.dll
 0004:00000198       __imp__ExitProcess@4       30189198     kernel32:KERNEL32.dll
 0004:0000019c       __imp__FatalAppExitA@8     3018919c     kernel32:KERNEL32.dll
 0004:000001a0       __imp__Sleep@4             301891a0     kernel32:KERNEL32.dll
 0004:000001a4       __imp__WideCharToMultiByte@32 301891a4     kernel32:KERNEL32.dll
 0004:000001a8       __imp__MultiByteToWideChar@24 301891a8     kernel32:KERNEL32.dll
 0004:000001ac       __imp__LCMapStringA@24     301891ac     kernel32:KERNEL32.dll
 0004:000001b0       __imp__LCMapStringW@24     301891b0     kernel32:KERNEL32.dll
 0004:000001b4       __imp__TerminateProcess@8  301891b4     kernel32:KERNEL32.dll
 0004:000001b8       __imp__GetCurrentProcess@0 301891b8     kernel32:KERNEL32.dll
 0004:000001bc       __imp__GetCurrentThreadId@0 301891bc     kernel32:KERNEL32.dll
 0004:000001c0       __imp__TlsSetValue@8       301891c0     kernel32:KERNEL32.dll
 0004:000001c4       __imp__TlsAlloc@0          301891c4     kernel32:KERNEL32.dll
 0004:000001c8       __imp__TlsFree@4           301891c8     kernel32:KERNEL32.dll
 0004:000001cc       __imp__SetLastError@4      301891cc     kernel32:KERNEL32.dll
 0004:000001d0       __imp__TlsGetValue@4       301891d0     kernel32:KERNEL32.dll
 0004:000001d4       __imp__GetLastError@0      301891d4     kernel32:KERNEL32.dll
 0004:000001d8       __imp__GetCurrentThread@0  301891d8     kernel32:KERNEL32.dll
 0004:000001dc       __imp__SetHandleCount@4    301891dc     kernel32:KERNEL32.dll
 0004:000001e0       __imp__GetFileType@4       301891e0     kernel32:KERNEL32.dll
 0004:000001e4       __imp__GetStartupInfoA@4   301891e4     kernel32:KERNEL32.dll
 0004:000001e8       __imp__InterlockedDecrement@4 301891e8     kernel32:KERNEL32.dll
 0004:000001ec       __imp__IsBadReadPtr@8      301891ec     kernel32:KERNEL32.dll
 0004:000001f0       __imp__HeapValidate@12     301891f0     kernel32:KERNEL32.dll
 0004:000001f4       __imp__FreeEnvironmentStringsA@4 301891f4     kernel32:KERNEL32.dll
 0004:000001f8       __imp__FreeEnvironmentStringsW@4 301891f8     kernel32:KERNEL32.dll
 0004:000001fc       __imp__GetEnvironmentStrings@0 301891fc     kernel32:KERNEL32.dll
 0004:00000200       __imp__GetEnvironmentStringsW@0 30189200     kernel32:KERNEL32.dll
 0004:00000204       __imp__HeapDestroy@4       30189204     kernel32:KERNEL32.dll
 0004:00000208       __imp__HeapCreate@12       30189208     kernel32:KERNEL32.dll
 0004:0000020c       __imp__HeapFree@12         3018920c     kernel32:KERNEL32.dll
 0004:00000210       __imp__VirtualFree@12      30189210     kernel32:KERNEL32.dll
 0004:00000214       __imp__GetStringTypeA@20   30189214     kernel32:KERNEL32.dll
 0004:00000218       __imp__GetStringTypeW@16   30189218     kernel32:KERNEL32.dll
 0004:0000021c       __imp__SetFilePointer@16   3018921c     kernel32:KERNEL32.dll
 0004:00000220       __imp__SetConsoleCtrlHandler@8 30189220     kernel32:KERNEL32.dll
 0004:00000224       __imp__GetCPInfo@8         30189224     kernel32:KERNEL32.dll
 0004:00000228       __imp__IsValidLocale@8     30189228     kernel32:KERNEL32.dll
 0004:0000022c       __imp__IsValidCodePage@4   3018922c     kernel32:KERNEL32.dll
 0004:00000230       __imp__GetLocaleInfoA@16   30189230     kernel32:KERNEL32.dll
 0004:00000234       __imp__EnumSystemLocalesA@8 30189234     kernel32:KERNEL32.dll
 0004:00000238       __imp__GetUserDefaultLCID@0 30189238     kernel32:KERNEL32.dll
 0004:0000023c       __imp__GetVersionExA@4     3018923c     kernel32:KERNEL32.dll
 0004:00000240       __imp__RtlUnwind@16        30189240     kernel32:KERNEL32.dll
 0004:00000244       __imp__UnhandledExceptionFilter@4 30189244     kernel32:KERNEL32.dll
 0004:00000248       __imp__HeapAlloc@12        30189248     kernel32:KERNEL32.dll
 0004:0000024c       __imp__HeapReAlloc@16      3018924c     kernel32:KERNEL32.dll
 0004:00000250       __imp__VirtualAlloc@16     30189250     kernel32:KERNEL32.dll
 0004:00000254       __imp__GetACP@0            30189254     kernel32:KERNEL32.dll
 0004:00000258       __imp__GetOEMCP@0          30189258     kernel32:KERNEL32.dll
 0004:0000025c       __imp__SetStdHandle@8      3018925c     kernel32:KERNEL32.dll
 0004:00000260       __imp__FlushFileBuffers@4  30189260     kernel32:KERNEL32.dll
 0004:00000264       __imp__GetTimeZoneInformation@4 30189264     kernel32:KERNEL32.dll
 0004:00000268       __imp__GetLocaleInfoW@16   30189268     kernel32:KERNEL32.dll
 0004:0000026c       __imp__CloseHandle@4       3018926c     kernel32:KERNEL32.dll
 0004:00000270       __imp__CompareStringA@24   30189270     kernel32:KERNEL32.dll
 0004:00000274       __imp__CompareStringW@24   30189274     kernel32:KERNEL32.dll
 0004:00000278       __imp__SetEnvironmentVariableA@8 30189278     kernel32:KERNEL32.dll
 0004:0000027c       \177KERNEL32_NULL_THUNK_DATA 3018927c     kernel32:KERNEL32.dll

 entry point at        0001:00027010

 Static symbols

 0001:00025060       _SkipWhitespace            30026060 f   q_shared.obj
 0001:0001f900       _CG_MachineGunEjectBrass   30020900 f   cg_weapons.obj
 0001:0001fc50       _CG_ShotgunEjectBrass      30020c50 f   cg_weapons.obj
 0001:00020020       _CG_RocketTrail            30021020 f   cg_weapons.obj
 0001:000201b0       _CG_GrenadeTrail           300211b0 f   cg_weapons.obj
 0001:00020a80       _CG_LightningBolt          30021a80 f   cg_weapons.obj
 0001:00020d50       _CG_SpawnRailTrail         30021d50 f   cg_weapons.obj
 0001:00020dc0       _CG_MachinegunSpinAngle    30021dc0 f   cg_weapons.obj
 0001:00020eb0       _CG_AddWeaponWithPowerups  30021eb0 f   cg_weapons.obj
 0001:00021270       _CG_MapTorsoToWeaponFrame  30022270 f   cg_weapons.obj
 0001:00021320       _CG_CalculateWeaponPosition 30022320 f   cg_weapons.obj
 0001:00021820       _CG_WeaponSelectable       30022820 f   cg_weapons.obj
 0001:00022320       _CG_ShotgunPattern         30023320 f   cg_weapons.obj
 0001:00022470       _CG_ShotgunPellet          30023470 f   cg_weapons.obj
 0001:0001d910       _CG_AddTestModel           3001e910 f   cg_view.obj
 0001:0001da80       _CG_DamageBlendBlob        3001ea80 f   cg_view.obj
 0001:0001dc30       _CG_CalcViewValues         3001ec30 f   cg_view.obj
 0001:0001de80       _CG_CalcVrect              3001ee80 f   cg_view.obj
 0001:0001df70       _CG_OffsetThirdPersonView  3001ef70 f   cg_view.obj
 0001:0001e2b0       _CG_OffsetFirstPersonView  3001f2b0 f   cg_view.obj
 0001:0001e700       _CG_StepOffset             3001f700 f   cg_view.obj
 0001:0001e750       _CG_CalcFov                3001f750 f   cg_view.obj
 0001:0001e990       _CG_PowerupTimerSounds     3001f990 f   cg_view.obj
 0001:0001c360       _CG_ResetEntity            3001d360 f   cg_snapshot.obj
 0001:0001c560       _CG_TransitionSnapshot     3001d560 f   cg_snapshot.obj
 0001:0001c740       _CG_TransitionEntity       3001d740 f   cg_snapshot.obj
 0001:0001c7b0       _CG_SetNextSnap            3001d7b0 f   cg_snapshot.obj
 0001:0001c930       _CG_ReadNextSnapshot       3001d930 f   cg_snapshot.obj
 0001:0001b7c0       _CG_ServerCommand          3001c7c0 f   cg_servercmds.obj
 0001:0001b9b0       _CG_ParseScores            3001c9b0 f   cg_servercmds.obj
 0001:0001bbb0       _CG_ParseTeamInfo          3001cbb0 f   cg_servercmds.obj
 0001:0001bd00       _CG_ConfigStringModified   3001cd00 f   cg_servercmds.obj
 0001:0001bf30       _CG_ParseWarmup            3001cf30 f   cg_servercmds.obj
 0001:0001bfa0       _CG_AddToTeamChat          3001cfa0 f   cg_servercmds.obj
 0001:0001c1e0       _CG_MapRestart             3001d1e0 f   cg_servercmds.obj
 0001:0001ab90       _CG_DrawClientScore        3001bb90 f   cg_scoreboard.obj
 0001:0001b170       _CG_TeamScoreboard         3001c170 f   cg_scoreboard.obj
 0001:0001b520       _CG_CenterGiantLine        3001c520 f   cg_scoreboard.obj
 0001:000198a0       _CG_ClipMoveToEntities     3001a8a0 f   cg_predict.obj
 0001:0001a0a0       _CG_InterpolatePlayerState 3001b0a0 f   cg_predict.obj
 0001:0001a250       _CG_TouchTriggerPrediction 3001b250 f   cg_predict.obj
 0001:0001a400       _CG_TouchItem              3001b400 f   cg_predict.obj
 0001:00014a60       _CG_ColorFromString        30015a60 f   cg_players.obj
 0001:00014b10       _CG_LoadClientInfo         30015b10 f   cg_players.obj
 0001:00014d80       _CG_RegisterClientModelname 30015d80 f   cg_players.obj
 0001:00014f60       _CG_ParseAnimationFile     30015f60 f   cg_players.obj
 0001:00015460       _CG_RegisterClientSkin     30016460 f   cg_players.obj
 0001:00015530       _CG_CopyClientInfoModel    30016530 f   cg_players.obj
 0001:00015660       _CG_ScanForExistingClientInfo 30016660 f   cg_players.obj
 0001:00015720       _CG_SetDeferredClientInfo  30016720 f   cg_players.obj
 0001:00016680       _CG_PlayerAnimation        30017680 f   cg_players.obj
 0001:000167e0       _CG_RunLerpFrame           300177e0 f   cg_players.obj
 0001:000169f0       _CG_SetLerpFrameAnimation  300179f0 f   cg_players.obj
 0001:00016a90       _CG_PlayerAngles           30017a90 f   cg_players.obj
 0001:00016da0       _CG_SwingAngles            30017da0 f   cg_players.obj
 0001:00016f70       _CG_AddPainTwitch          30017f70 f   cg_players.obj
 0001:00016ff0       _CG_PlayerPowerups         30017ff0 f   cg_players.obj
 0001:00017150       _CG_HasteTrail             30018150 f   cg_players.obj
 0001:00017250       _CG_TrailItem              30018250 f   cg_players.obj
 0001:00017360       _CG_PlayerSprites          30018360 f   cg_players.obj
 0001:000174c0       _CG_PlayerFloatSprite      300184c0 f   cg_players.obj
 0001:00017590       _CG_PlayerShadow           30018590 f   cg_players.obj
 0001:000176e0       _CG_PlayerSplash           300186e0 f   cg_players.obj
 0001:00018b10       _CG_ClearLerpFrame         30019b10 f   cg_players.obj
 0001:00012bb0       _CG_RegisterSounds         30013bb0 f   cg_main.obj
 0001:000131f0       _CG_RegisterItemSounds     300141f0 f   cg_main.obj
 0001:00013300       _CG_RegisterGraphics       30014300 f   cg_main.obj
 0001:00013b20       _CG_RegisterClients        30014b20 f   cg_main.obj
 0001:00011dd0       _CG_AddMoveScaleFade       30012dd0 f   cg_localents.obj
 0001:00011ed0       _CG_AddScaleFade           30012ed0 f   cg_localents.obj
 0001:00011fb0       _CG_AddFallScaleFade       30012fb0 f   cg_localents.obj
 0001:000120b0       _CG_AddExplosion           300130b0 f   cg_localents.obj
 0001:000122f0       _CG_AddFalling             300132f0 f   cg_localents.obj
 0001:00012380       _CG_AddSpriteExplosion     30013380 f   cg_localents.obj
 0001:000112b0       _CG_DrawLoadingIcons       300122b0 f   cg_info.obj
 0001:000104d0       _CG_Obituary               300114d0 f   cg_event.obj
 0001:00010a30       _CG_UseItem                30011a30 f   cg_event.obj
 0001:00010b10       _CG_ItemPickup             30011b10 f   cg_event.obj
 0001:0000d5c0       _CG_CalcEntityLerpPositions 3000e5c0 f   cg_ents.obj
 0001:0000d670       _CG_InterpolateEntityPosition 3000e670 f   cg_ents.obj
 0001:0000d7b0       _CG_AddCEntity             3000e7b0 f   cg_ents.obj
 0001:0000d8d0       _CG_EntityEffects          3000e8d0 f   cg_ents.obj
 0001:0000d9b0       _CG_General                3000e9b0 f   cg_ents.obj
 0001:0000dac0       _CG_Speaker                3000eac0 f   cg_ents.obj
 0001:0000db80       _CG_Item                   3000eb80 f   cg_ents.obj
 0001:0000e380       _CG_Missile                3000f380 f   cg_ents.obj
 0001:0000e6f0       _CG_Grapple                3000f6f0 f   cg_ents.obj
 0001:0000e860       _CG_Mover                  3000f860 f   cg_ents.obj
 0001:0000e9a0       _CG_Portal                 3000f9a0 f   cg_ents.obj
 0001:0000ab50       _CG_TileClearBox           3000bb50 f   cg_drawtools.obj
 0001:0000af20       _UI_DrawBannerString2      3000bf20 f   cg_drawtools.obj
 0001:0000b390       _UI_DrawProportionalString2 3000c390 f   cg_drawtools.obj
 0001:000069d0       _CG_Draw3DModel            300079d0 f   cg_draw.obj
 0001:00007080       _CG_Draw2D                 30008080 f   cg_draw.obj
 0001:00007360       _CG_DrawStatusBar          30008360 f   cg_draw.obj
 0001:00007710       _CG_DrawField              30008710 f   cg_draw.obj
 0001:00007910       _CG_DrawStatusBarHead      30008910 f   cg_draw.obj
 0001:00007c60       _CG_DrawStatusBarFlag      30008c60 f   cg_draw.obj
 0001:00007c90       _CG_DrawUpperRight         30008c90 f   cg_draw.obj
 0001:00007d30       _CG_DrawAttacker           30008d30 f   cg_draw.obj
 0001:00007e80       _CG_DrawSnapshot           30008e80 f   cg_draw.obj
 0001:00007f10       _CG_DrawFPS                30008f10 f   cg_draw.obj
 0001:00008020       _CG_DrawTimer              30009020 f   cg_draw.obj
 0001:000080f0       _CG_DrawTeamOverlay        300090f0 f   cg_draw.obj
 0001:00008600       _CG_DrawLowerRight         30009600 f   cg_draw.obj
 0001:00008660       _CG_DrawScores             30009660 f   cg_draw.obj
 0001:00008cd0       _CG_DrawPowerups           30009cd0 f   cg_draw.obj
 0001:00009090       _CG_DrawLowerLeft          3000a090 f   cg_draw.obj
 0001:000090f0       _CG_DrawPickupItem         3000a0f0 f   cg_draw.obj
 0001:000091d0       _CG_DrawTeamInfo           3000a1d0 f   cg_draw.obj
 0001:00009400       _CG_DrawHoldableItem       3000a400 f   cg_draw.obj
 0001:00009460       _CG_DrawReward             3000a460 f   cg_draw.obj
 0001:00009530       _CG_DrawLagometer          3000a530 f   cg_draw.obj
 0001:000098e0       _CG_DrawDisconnect         3000a8e0 f   cg_draw.obj
 0001:000099b0       _CG_DrawCenterString       3000a9b0 f   cg_draw.obj
 0001:00009b50       _CG_DrawCrosshair          3000ab50 f   cg_draw.obj
 0001:00009cd0       _CG_DrawCrosshairNames     3000acd0 f   cg_draw.obj
 0001:00009db0       _CG_ScanForCrosshairEntity 3000adb0 f   cg_draw.obj
 0001:00009ea0       _CG_DrawSpectator          3000aea0 f   cg_draw.obj
 0001:00009f20       _CG_DrawVote               3000af20 f   cg_draw.obj
 0001:00009fd0       _CG_DrawIntermission       3000afd0 f   cg_draw.obj
 0001:0000a000       _CG_DrawFollow             3000b000 f   cg_draw.obj
 0001:0000a0d0       _CG_DrawAmmoWarning        3000b0d0 f   cg_draw.obj
 0001:0000a150       _CG_DrawWarmup             3000b150 f   cg_draw.obj
 0001:000064c0       _CG_SizeUp_f               300074c0 f   cg_consolecmds.obj
 0001:00006500       _CG_SizeDown_f             30007500 f   cg_consolecmds.obj
 0001:00006540       _CG_Viewpos_f              30007540 f   cg_consolecmds.obj
 0001:00006590       _CG_ScoresDown_f           30007590 f   cg_consolecmds.obj
 0001:00006600       _CG_ScoresUp_f             30007600 f   cg_consolecmds.obj
 0001:00006630       _CG_TellTarget_f           30007630 f   cg_consolecmds.obj
 0001:000066a0       _CG_TellAttacker_f         300076a0 f   cg_consolecmds.obj
 0001:000021a0       _PM_WaterJumpMove          300031a0 f   bg_pmove.obj
 0001:00002230       _PM_WaterMove              30003230 f   bg_pmove.obj
 0001:00002470       _PM_Friction               30003470 f   bg_pmove.obj
 0001:00002620       _PM_Accelerate             30003620 f   bg_pmove.obj
 0001:000026f0       _PM_CmdScale               300036f0 f   bg_pmove.obj
 0001:000027e0       _PM_CheckWaterJump         300037e0 f   bg_pmove.obj
 0001:00002980       _PM_FlyMove                30003980 f   bg_pmove.obj
 0001:00002a90       _PM_AirMove                30003a90 f   bg_pmove.obj
 0001:00002bf0       _PM_SetMovementDir         30003bf0 f   bg_pmove.obj
 0001:00002dd0       _PM_GrappleMove            30003dd0 f   bg_pmove.obj
 0001:00002f30       _PM_CrawlMove              30003f30 f   bg_pmove.obj
 0001:00003310       _PM_CheckJump              30004310 f   bg_pmove.obj
 0001:00003450       _PM_ForceLegsAnim          30004450 f   bg_pmove.obj
 0001:00003480       _PM_StartLegsAnim          30004480 f   bg_pmove.obj
 0001:000034e0       _PM_WalkMove               300044e0 f   bg_pmove.obj
 0001:000038a0       _PM_DeadMove               300048a0 f   bg_pmove.obj
 0001:00003980       _PM_NoclipMove             30004980 f   bg_pmove.obj
 0001:00003c00       _PM_GroundTrace            30004c00 f   bg_pmove.obj
 0001:00003f80       _PM_CrashLand              30004f80 f   bg_pmove.obj
 0001:000041f0       _PM_FootstepForSurface     300051f0 f   bg_pmove.obj
 0001:00004230       _PM_CorrectAllSolid        30005230 f   bg_pmove.obj
 0001:00004290       _PM_GroundTraceMissed      30005290 f   bg_pmove.obj
 0001:000043f0       _PM_GroundWallTrace        300053f0 f   bg_pmove.obj
 0001:000046b0       _PM_SetWaterLevel          300056b0 f   bg_pmove.obj
 0001:00004830       _PM_CheckDuck              30005830 f   bg_pmove.obj
 0001:00004a20       _PM_Footsteps              30005a20 f   bg_pmove.obj
 0001:00004d90       _PM_ContinueLegsAnim       30005d90 f   bg_pmove.obj
 0001:00004dd0       _PM_WaterEvents            30005dd0 f   bg_pmove.obj
 0001:00004e70       _PM_TorsoAnimation         30005e70 f   bg_pmove.obj
 0001:00004ec0       _PM_ContinueTorsoAnim      30005ec0 f   bg_pmove.obj
 0001:00004f00       _PM_StartTorsoAnim         30005f00 f   bg_pmove.obj
 0001:00004f50       _PM_Weapon                 30005f50 f   bg_pmove.obj
 0001:000054d0       _PM_BeginWeaponChange      300064d0 f   bg_pmove.obj
 0001:00005560       _PM_FinishWeaponChange     30006560 f   bg_pmove.obj
 0001:00005600       _PM_Animate                30006600 f   bg_pmove.obj
 0001:00005660       _PM_DropTimers             30006660 f   bg_pmove.obj
 0001:00000540       _swapfunc                  30001540 f   bg_lib.obj
 0001:00000600       _med3                      30001600 f   bg_lib.obj
 0001:0003bee0       _findenv                   3003cee0 f   LIBCMTD:setenv.obj
 0001:0003bf60       _copy_environ              3003cf60 f   LIBCMTD:setenv.obj
 0001:0003bbb0       _strncnt                   3003cbb0 f   LIBCMTD:a_cmp.obj
 0001:0003a7b0       __tzset_lk                 3003b7b0 f   LIBCMTD:tzset.obj
 0001:0003ab90       __isindst_lk               3003bb90 f   LIBCMTD:tzset.obj
 0001:0003ae90       _cvtdate                   3003be90 f   LIBCMTD:tzset.obj
 0001:00039f2c       lupe                       3003af2c f   LIBCMTD:strnicmp.obj
 0001:00039f44       skip1                      3003af44 f   LIBCMTD:strnicmp.obj
 0001:00039f4e       skip2                      3003af4e f   LIBCMTD:strnicmp.obj
 0001:00039f55       eject                      3003af55 f   LIBCMTD:strnicmp.obj
 0001:00039f5f       differ                     3003af5f f   LIBCMTD:strnicmp.obj
 0001:00039f71       notclocale                 3003af71 f   LIBCMTD:strnicmp.obj
 0001:00039f85       do_lock                    3003af85 f   LIBCMTD:strnicmp.obj
 0001:00039f9e       end_lock                   3003af9e f   LIBCMTD:strnicmp.obj
 0001:00039fa4       lupe2                      3003afa4 f   LIBCMTD:strnicmp.obj
 0001:00039fcf       eject2                     3003afcf f   LIBCMTD:strnicmp.obj
 0001:00039fd5       differ2                    3003afd5 f   LIBCMTD:strnicmp.obj
 0001:00039fde       toend2                     3003afde f   LIBCMTD:strnicmp.obj
 0001:00039fec       do_unlock                  3003afec f   LIBCMTD:strnicmp.obj
 0001:00039ffa       end_unlock                 3003affa f   LIBCMTD:strnicmp.obj
 0001:00039ffa       toend                      3003affa f   LIBCMTD:strnicmp.obj
 0001:00039e4c       chk_null                   3003ae4c f   LIBCMTD:stricmp.obj
 0001:00039e7e       done                       3003ae7e f   LIBCMTD:stricmp.obj
 0001:00039e83       notclocale                 3003ae83 f   LIBCMTD:stricmp.obj
 0001:00039e97       do_lock                    3003ae97 f   LIBCMTD:stricmp.obj
 0001:00039eac       end_lock                   3003aeac f   LIBCMTD:stricmp.obj
 0001:00039eb4       chk_null2                  3003aeb4 f   LIBCMTD:stricmp.obj
 0001:00039edf       done2                      3003aedf f   LIBCMTD:stricmp.obj
 0001:00039eef       do_unlock                  3003aeef f   LIBCMTD:stricmp.obj
 0001:00039ef9       end_unlock                 3003aef9 f   LIBCMTD:stricmp.obj
 0001:00039efb       doret                      3003aefb f   LIBCMTD:stricmp.obj
 0001:00038c30       __expandtime               30039c30 f   LIBCMTD:strftime.obj
 0001:00039250       __store_str                3003a250 f   LIBCMTD:strftime.obj
 0001:000392a0       __store_num                3003a2a0 f   LIBCMTD:strftime.obj
 0001:00039350       __store_number             3003a350 f   LIBCMTD:strftime.obj
 0001:00039400       __store_winword            3003a400 f   LIBCMTD:strftime.obj
 0001:00038370       _flsall                    30039370 f   LIBCMTD:fflush.obj
 0001:000362f0       _getSystemCP               300372f0 f   LIBCMTD:mbctype.obj
 0001:00036350       _CPtoLCID                  30037350 f   LIBCMTD:mbctype.obj
 0001:000363d0       _setSBCS                   300373d0 f   LIBCMTD:mbctype.obj
 0001:00036450       _setSBUpLow                30037450 f   LIBCMTD:mbctype.obj
 0001:00033c90       _xcptlookup                30034c90 f   LIBCMTD:winxfltr.obj
 0001:00033910       _gu_return                 30034910 f   LIBCMTD:exsup.obj
 0001:00033918       __unwind_handler           30034918 f   LIBCMTD:exsup.obj
 0001:00032d60       _TranslateName             30033d60 f   LIBCMTD:getqloc.obj
 0001:00032df0       _GetLcidFromLangCountry    30033df0 f   LIBCMTD:getqloc.obj
 0001:00032eb0       _LangCountryEnumProc@4     30033eb0 f   LIBCMTD:getqloc.obj
 0001:000331e0       _GetLcidFromLanguage       300341e0 f   LIBCMTD:getqloc.obj
 0001:00033260       _LanguageEnumProc@4        30034260 f   LIBCMTD:getqloc.obj
 0001:00033380       _GetLcidFromCountry        30034380 f   LIBCMTD:getqloc.obj
 0001:000333d0       _CountryEnumProc@4         300343d0 f   LIBCMTD:getqloc.obj
 0001:00033480       _GetLcidFromDefault        30034480 f   LIBCMTD:getqloc.obj
 0001:000334b0       _ProcessCodePage           300344b0 f   LIBCMTD:getqloc.obj
 0001:00033550       _TestDefaultCountry        30034550 f   LIBCMTD:getqloc.obj
 0001:000335a0       _TestDefaultLanguage       300345a0 f   LIBCMTD:getqloc.obj
 0001:00033630       _IsThisWindowsNT           30034630 f   LIBCMTD:getqloc.obj
 0001:00033680       _crtGetLocaleInfoA@16      30034680 f   LIBCMTD:getqloc.obj
 0001:00033810       _LcidFromHexString         30034810 f   LIBCMTD:getqloc.obj
 0001:00033890       _GetPrimaryLen             30034890 f   LIBCMTD:getqloc.obj
 0001:00032b34       listnext                   30033b34 f   LIBCMTD:strpbrk.obj
 0001:00032b41       listdone                   30033b41 f   LIBCMTD:strpbrk.obj
 0001:00032b44       dstnext                    30033b44 f   LIBCMTD:strpbrk.obj
 0001:00032b54       dstdone                    30033b54 f   LIBCMTD:strpbrk.obj
 0001:00032afa       okay                       30033afa f   LIBCMTD:strncmp.obj
 0001:00032b0d       firstbig                   30033b0d f   LIBCMTD:strncmp.obj
 0001:00032b0f       lastbig                    30033b0f f   LIBCMTD:strncmp.obj
 0001:00032b11       toend                      30033b11 f   LIBCMTD:strncmp.obj
 0001:00032ab4       listnext                   30033ab4 f   LIBCMTD:strcspn.obj
 0001:00032ac1       listdone                   30033ac1 f   LIBCMTD:strcspn.obj
 0001:00032ac8       dstnext                    30033ac8 f   LIBCMTD:strcspn.obj
 0001:00032ad6       dstdone                    30033ad6 f   LIBCMTD:strcspn.obj
 0001:000323c0       __get_lc_lconv             300333c0 f   LIBCMTD:initmon.obj
 0001:000325d0       _fix_grouping              300335d0 f   LIBCMTD:initmon.obj
 0001:00032650       __free_lc_lconv            30033650 f   LIBCMTD:initmon.obj
 0001:00032210       _fix_grouping              30033210 f   LIBCMTD:initnum.obj
 0001:000316c0       __get_lc_time              300326c0 f   LIBCMTD:inittime.obj
 0001:00031c50       __free_lc_time             30032c50 f   LIBCMTD:inittime.obj
 0001:000311c0       _ctrlevent_capture@4       300321c0 f   LIBCMTD:winsig.obj
 0001:000314a0       _siglookup                 300324a0 f   LIBCMTD:winsig.obj
 0001:00030af0       _xtoa                      30031af0 f   LIBCMTD:xtoa.obj
 0001:00030c70       _x64toa@20                 30031c70 f   LIBCMTD:xtoa.obj
 0001:00030a41       L1                         30031a41 f   LIBCMTD:ullrem.obj
 0001:00030a4f       L3                         30031a4f f   LIBCMTD:ullrem.obj
 0001:00030a7a       L4                         30031a7a f   LIBCMTD:ullrem.obj
 0001:00030a82       L5                         30031a82 f   LIBCMTD:ullrem.obj
 0001:00030a91       L2                         30031a91 f   LIBCMTD:ullrem.obj
 0001:000309d2       L1                         300319d2 f   LIBCMTD:ulldiv.obj
 0001:000309e0       L3                         300319e0 f   LIBCMTD:ulldiv.obj
 0001:00030a0e       L4                         30031a0e f   LIBCMTD:ulldiv.obj
 0001:00030a0f       L5                         30031a0f f   LIBCMTD:ulldiv.obj
 0001:00030a13       L2                         30031a13 f   LIBCMTD:ulldiv.obj
 0001:0002eff0       __abstract_cw              3002fff0 f   LIBCMTD:ieee87.obj
 0001:0002f170       __hw_cw                    30030170 f   LIBCMTD:ieee87.obj
 0001:0002f2d0       __abstract_sw              300302d0 f   LIBCMTD:ieee87.obj
 0001:0002e3b0       _parse_cmdline             3002f3b0 f   LIBCMTD:stdargv.obj
 0001:0002c6e0       _realloc_help              3002d6e0 f   LIBCMTD:dbgheap.obj
 0001:0002d320       _CheckBytes                3002e320 f   LIBCMTD:dbgheap.obj
 0001:0002df10       __printMemBlockData        3002ef10 f   LIBCMTD:dbgheap.obj
 0001:0002ba30       _doexit                    3002ca30 f   LIBCMTD:crt0dat.obj
 0001:0002bb40       __initterm                 3002cb40 f   LIBCMTD:crt0dat.obj
 0001:0002b920       _strncnt                   3002c920 f   LIBCMTD:a_map.obj
 0001:0002afb0       __setlocale_set_cat        3002bfb0 f   LIBCMTD:setlocal.obj
 0001:0002b150       __setlocale_get_all        3002c150 f   LIBCMTD:setlocal.obj
 0001:0002a6fc       fFATN2                     3002b6fc f   LIBCMTD:87triga.obj
 0001:0002a772       _rtforatnby0               3002b772 f   LIBCMTD:87triga.obj
 0001:0002a755       _rtforatn20                3002b755 f   LIBCMTD:87triga.obj
 0001:0002a3d0       _CrtMessageWindow          3002b3d0 f   LIBCMTD:dbgrpt.obj
 0001:00029dc0       _write_char                3002adc0 f   LIBCMTD:output.obj
 0001:00029e40       _write_multi_char          3002ae40 f   LIBCMTD:output.obj
 0001:00029e80       _write_string              3002ae80 f   LIBCMTD:output.obj
 0001:00029ed0       _get_int_arg               3002aed0 f   LIBCMTD:output.obj
 0001:00029ef0       _get_int64_arg             3002aef0 f   LIBCMTD:output.obj
 0001:00029f10       _get_short_arg             3002af10 f   LIBCMTD:output.obj
 0001:000289a0       __get_fname                300299a0 f   LIBCMTD:fpexcept.obj
 0001:00027de9       hard                       30028de9 f   LIBCMTD:llmul.obj
 0001:00027870       __cftoe2                   30028870 f   LIBCMTD:cvt.obj
 0001:00027a50       __cftof2                   30028a50 f   LIBCMTD:cvt.obj
 0001:00027ce0       __shift                    30028ce0 f   LIBCMTD:cvt.obj
 0001:00026a34       src_misaligned             30027a34 f   LIBCMTD:strncpy.obj
 0001:00026a50       tail_loop_start            30027a50 f   LIBCMTD:strncpy.obj
 0001:00026a55       copy_tail_loop             30027a55 f   LIBCMTD:strncpy.obj
 0001:00026a62       fill_tail_end1             30027a62 f   LIBCMTD:strncpy.obj
 0001:00026a6a       align_dest                 30027a6a f   LIBCMTD:strncpy.obj
 0001:00026a72       dest_align_loop            30027a72 f   LIBCMTD:strncpy.obj
 0001:00026a84       dest_align_loop_end        30027a84 f   LIBCMTD:strncpy.obj
 0001:00026a8b       finish_loop                30027a8b f   LIBCMTD:strncpy.obj
 0001:00026a8e       fill_tail_zero_bytes       30027a8e f   LIBCMTD:strncpy.obj
 0001:00026a93       finish                     30027a93 f   LIBCMTD:strncpy.obj
 0001:00026a99       main_loop                  30027a99 f   LIBCMTD:strncpy.obj
 0001:00026aa1       main_loop_entrance         30027aa1 f   LIBCMTD:strncpy.obj
 0001:00026ad7       byte_2                     30027ad7 f   LIBCMTD:strncpy.obj
 0001:00026ae1       byte_1                     30027ae1 f   LIBCMTD:strncpy.obj
 0001:00026aeb       byte_0                     30027aeb f   LIBCMTD:strncpy.obj
 0001:00026aef       fill_with_EOS_dwords       30027aef f   LIBCMTD:strncpy.obj
 0001:00026af7       fill_dwords_with_EOS       30027af7 f   LIBCMTD:strncpy.obj
 0001:00026af9       fill_with_EOS_loop         30027af9 f   LIBCMTD:strncpy.obj
 0001:00026b01       fill_tail                  30027b01 f   LIBCMTD:strncpy.obj
 0001:00026b06       fill_tail_end              30027b06 f   LIBCMTD:strncpy.obj
 0001:000269c0       _$$$00001                  300279c0 f   LIBCMTD:chkstk.obj
 0001:000269cc       probepages                 300279cc f   LIBCMTD:chkstk.obj
 0001:000269e0       lastpage                   300279e0 f   LIBCMTD:chkstk.obj
 0001:000264f0       LeadUp1                    300274f0 f   LIBCMTD:memcpy.obj
 0001:0002651c       LeadUp2                    3002751c f   LIBCMTD:memcpy.obj
 0001:00026540       LeadUp3                    30027540 f   LIBCMTD:memcpy.obj
 0001:000265bf       UnwindUp0                  300275bf f   LIBCMTD:memcpy.obj
 0001:000265ac       UnwindUp1                  300275ac f   LIBCMTD:memcpy.obj
 0001:000265a4       UnwindUp2                  300275a4 f   LIBCMTD:memcpy.obj
 0001:0002659c       UnwindUp3                  3002759c f   LIBCMTD:memcpy.obj
 0001:00026594       UnwindUp4                  30027594 f   LIBCMTD:memcpy.obj
 0001:0002658c       UnwindUp5                  3002758c f   LIBCMTD:memcpy.obj
 0001:00026584       UnwindUp6                  30027584 f   LIBCMTD:memcpy.obj
 0001:0002657c       UnwindUp7                  3002757c f   LIBCMTD:memcpy.obj
 0001:000265d8       TrailUp0                   300275d8 f   LIBCMTD:memcpy.obj
 0001:000265e0       TrailUp1                   300275e0 f   LIBCMTD:memcpy.obj
 0001:000265ec       TrailUp2                   300275ec f   LIBCMTD:memcpy.obj
 0001:00026600       TrailUp3                   30027600 f   LIBCMTD:memcpy.obj
 0001:00026678       LeadDown1                  30027678 f   LIBCMTD:memcpy.obj
 0001:00026698       LeadDown2                  30027698 f   LIBCMTD:memcpy.obj
 0001:000266c0       LeadDown3                  300276c0 f   LIBCMTD:memcpy.obj
 0001:00026714       UnwindDown7                30027714 f   LIBCMTD:memcpy.obj
 0001:0002671c       UnwindDown6                3002771c f   LIBCMTD:memcpy.obj
 0001:00026724       UnwindDown5                30027724 f   LIBCMTD:memcpy.obj
 0001:0002672c       UnwindDown4                3002772c f   LIBCMTD:memcpy.obj
 0001:00026734       UnwindDown3                30027734 f   LIBCMTD:memcpy.obj
 0001:0002673c       UnwindDown2                3002773c f   LIBCMTD:memcpy.obj
 0001:00026744       UnwindDown1                30027744 f   LIBCMTD:memcpy.obj
 0001:00026757       UnwindDown0                30027757 f   LIBCMTD:memcpy.obj
 0001:00026770       TrailDown0                 30027770 f   LIBCMTD:memcpy.obj
 0001:00026778       TrailDown1                 30027778 f   LIBCMTD:memcpy.obj
 0001:00026788       TrailDown2                 30027788 f   LIBCMTD:memcpy.obj
 0001:0002679c       TrailDown3                 3002779c f   LIBCMTD:memcpy.obj
 0001:000264a0       CopyUp                     300274a0 f   LIBCMTD:memcpy.obj
 0001:000264bc       CopyLeadUp                 300274bc f   LIBCMTD:memcpy.obj
 0001:000264d4       ByteCopyUp                 300274d4 f   LIBCMTD:memcpy.obj
 0001:000264dc       CopyUnwindUp               300274dc f   LIBCMTD:memcpy.obj
 0001:00026618       CopyDown                   30027618 f   LIBCMTD:memcpy.obj
 0001:00026640       CopyUnwindDown             30027640 f   LIBCMTD:memcpy.obj
 0001:0002664c       CopyLeadDown               3002764c f   LIBCMTD:memcpy.obj
 0001:00026664       ByteCopyDown               30027664 f   LIBCMTD:memcpy.obj
 0001:00026103       adjust_loop                30027103 f   LIBCMTD:memset.obj
 0001:00026109       dwords                     30027109 f   LIBCMTD:memset.obj
 0001:00026123       main_loop_tail             30027123 f   LIBCMTD:memset.obj
 0001:00026127       tail                       30027127 f   LIBCMTD:memset.obj
 0001:0002612d       finish                     3002712d f   LIBCMTD:memset.obj
 0001:00026133       toend                      30027133 f   LIBCMTD:memset.obj

FIXUPS: 278a5 fffff9a5 85 69 33 8c 34 fffffd4c 12 18 16 10 1c 31 10 fffffde3
FIXUPS: 2700c a ffffff41 12 2a 10 1b 2a 10 fffffeaf 12 2a 10 1b 2a 10 1092
FIXUPS: 27fdf 5 15 75 1e 1e 1d 68 9 fffffc11 1c 13 6d a7 fffffcdd 1c 13
FIXUPS: 27c05 a7 fffffd4a a fffffee6 2a 45 4a fffffe32 2b 28 16 1d 29 11a6
FIXUPS: 28a3c 94 35 68 12 34 33 48 3c 36 1c 1a 18 17 fffff8c5 ffffff54
FIXUPS: 284ec fffffefe 5e 7 fffffa9c 5e 9 17 a 5 5 5 3d 7 f 1022 c 3e e
FIXUPS: 29060 182 1d8 1ac 2b 33 1b6 f4 27 36 44 c 10 16 c 32 d fffff41d
FIXUPS: 285ee 28 19f 20 3a 2f 1a 48 60 ff 217d 30 75 32 22 26 170 55 53
FIXUPS: 29e30 108 10 3e 54 4d 28 fffffaab 1c3 17 fffff167 a 14 52 a 14
FIXUPS: 28ef3 2c c 3a e 11 2f 2495 11 1d 21 14 26 19d 18 19 19 a ffffeac4
FIXUPS: 2a1ba 24 cb 67 133 18 21 34 30 a8 e2 142 ba 31 1e 2a 1b 11d 25
FIXUPS: 2ab5e fa2 13 a 34 a fffffc51 3d 5e 133 38 fffffd96 1f 7 10 fffff8cb
FIXUPS: 2b154 2a 18 38 16 2b 14 2e 18 18 7a 63 34 47 1e d 2f bd6 47 1b
FIXUPS: 2c0ab 50 31 4c 4e 1a 25 2a 9b 19 1b 26 2e 1b 14 19 19 11 67 27
FIXUPS: 2c492 2a 45 2e 33 4a 25 2b fffff4a4 f95 77 12 13 19 b 31 10 fffffb6f
FIXUPS: 2c73d f6 fffff3ac 43 8c 48 51 19 2f 2d 39 21 5a 38 47 17 31 11
FIXUPS: 2bf62 22 10 43 26 300d 34 39 16 7c 2a 28 ffffdcdd 13 e8 29a fffff9a8
FIXUPS: 2cb9f 2e 37 81 2a 21 62 1a 1a 1a 1a 1a 1d e fffffbae 12 1d 20 1e
FIXUPS: 2ca1a 1ce4 67 47 7e 17 1c 4c 15 4d 5a 11 5c 1b ec 33 49 10e 1a
FIXUPS: 2ed1e 20 31 28 4f 3a 31 18 45 18 f 1a 88 69 fffff0a3 2b 1c 2c 1c
FIXUPS: 2e128 c 1f 62 51 1f 45 c 5a 1f 93 57 8 51 2b 28 28 28 16 94 2b
FIXUPS: 2e5dc 2b 39 20 49 33 fffff2d9 b3 19 59 5f 54 85 15 1e d 18 20 1c
FIXUPS: 2dcb6 a 24 1c 50 1d 1f 62 34 3b 2b 3b 45 2b c 41 6b 56 36 fffff215
FIXUPS: 2d2a9 25 2f 1c 69 28 5f 54 21 128 1e 1b 33 2f 51 15 1e d 35 21
FIXUPS: 2d743 1c 6b 28 32 4f 18 1f 5b 66 25 22cf 17 1d 14 13 14 1a 19 fffffd2c
FIXUPS: 2f8d4 4a 94 2b fffff903 56 1e 13 22 fffffe07 36 28 1f 29 26 17
FIXUPS: 2f285 1c ffffdf63 26 28 15 18 35f1 13 16 26 1e 41 93 20 68 82 10
FIXUPS: 30afb 10 30 10 fffff3a6 21 21 24 2a 19 c fffffe4b 72 13 24 17 fffffc73
FIXUPS: 2fb40 77 3a 59 14e3 14 14 f 27 11 4c fffffe3d 31 21 1f d 21 10
FIXUPS: 30f77 1d fffffec2 fffffe19 28 29 ffffff78 17 fffff815 41 8c 14
FIXUPS: 307b4 19 1c 13 2a 3a 13fd 5d 17 b5 fffffb32 21 13 50 5e fffffd07
FIXUPS: 316d6 18 a6 10 31 2c 44 2c fffffcfd 37 fffffccd b 14 14 f 6d 1a2
FIXUPS: 314ce 10 3e b fffffbfb ef1 82 24 27 2a 17 58 50 44 1d 16 c4 13
FIXUPS: 3233f 16 1d a 96 f2 10 fffff9a2 2a 44 4b fffffe4d 2a 44 4b fffffc49
FIXUPS: 31ad6 11b 21 1132 11 11 11 11 11 11 11 11 11 11 11 11 11 11 11
FIXUPS: 32e54 11 11 14 14 14 14 14 14 14 14 14 14 14 fffff075 43 9dd 1f
FIXUPS: 32a25 1f 1f 1f 1f 1f 22 22 22 22 22 22 22 22 22 22 25 2f 11 11
FIXUPS: 32c9b 11 11 10 11 11 11 11 11 11 fffff8cf 1f 10 e 1e 11 25 11 5e
FIXUPS: 32721 1f 1f 1f 1f 1c 1f 1f 1f 1f 1f 1f 1f 1f 1f 1f 1f 1f 1f 1f
FIXUPS: 3298a 1f 1f b16 1f 1f 1f 1f 1f 1f 1f bd 11 11 11 11 11 11 fffff8b9
FIXUPS: 32fb0 1d 17 16 11 11 46 13 14 5b 11 10 34 30 16 3b 595 19 19 19
FIXUPS: 338a2 65 a6 22 17 e 15 e e e 2b 11 fffff840 1f 10 e 4c 11 4f 11
FIXUPS: 333f6 1f 1f 1f 1f 17 17 1f 959 39 6a 55 5a 62 28 2b 83 59 16 74
FIXUPS: 34197 54 2f 51 55 1b 52 12 4b 51 52 10 93 3d 33 a3 1a 11 198 ffffef8a
FIXUPS: 34e82 2f 14 f fffffe9a 2b 29 30 c d fffffeec 1b fffffdc5 13 ffffff61
FIXUPS: 34a58 11 2f 25 fffffe4f fffff264 29 34 35 3e 7 1c 7 1f c7 51 5a
FIXUPS: 36ef6 45 4b ffffe94c 191 19 de0 ffffe922 8 12 27 b 2a ffffff1b
FIXUPS: 3511b 19 a c fffffdd7 17 22 c 2c 18 3f 10 70 10 a c 53 fffffd94
FIXUPS: 38610 fffff1f7 21 35 35 13a c 10 c 27 6c fffff522 c 18 15 5 7 114
FIXUPS: 37145 7 10a 4a 7 15 5 7 e 267 35 35 1e8 fffff73d 1ff0 b 65 b 7c
FIXUPS: 38fe3 e b 18 32 45 2f fffff6a8 43 33 24 bd 2d 9b 32 43 c 10 c fffff35c
FIXUPS: 37ec7 eb 1c8 8c 152 6d 238 1b4f 21 154 31c 20 1f0 ffffea20 e c
FIXUPS: 39236 22 28 78 6e 21 68 33 40 25 f fffffc9a 5c 41 1f fffff975 82
FIXUPS: 38c12 83 7d 11 b8 b c35 9 2c 9 3d 54 84 8d 7e 23 23 23 3a 51 24
FIXUPS: 39de2 2a 28 45 2d 2d 28 28 1c 29 41 84 3a 24 31 36 50 fffff45e
FIXUPS: 395a9 71 15 1b 51 9 2e 9 6e 15 37 15 1e 14 1c 1c 1c 1b 36 3a 9
FIXUPS: 398f2 9 48 9 2e 9 2e 9 2c 9 1c5a fffffc1f 70 4f 1df fffffa8b 25
FIXUPS: 3afc0 31 fffffeb0 24 a 23 fffffdca 1b 76 be fffffb61 33 2c 32 20
FIXUPS: 3aa4b 14 1b 43 6f ffffe9bd 15 1b 50 9 2427 18 17 a 15 3b 5b 52
FIXUPS: 3bb3b 2c c d b0 53 66 53 25 23 fffff91e 17 2e 2d a 16 fffffe11
FIXUPS: 3b576 c f 4c 27 f f fec 29 19 2c fffffeb1 3a fffffeab b 14 c f
FIXUPS: 3c46a 1b c 10 29 2d fffffe1f fffffe5e fffff5eb 11 14 12 8 7 1b
FIXUPS: 3b7eb 17 150 e 15 18 1768 29 fffffaf6 45 29 3a 40 3e 33 4b 59 5a
FIXUPS: 3ce77 19 42 3c a7 19 28 c 21 fffff822 19 d9 13f 9e fffffc3c 43
FIXUPS: 3c6de fffffed9 c d fffc587f 3a d5 2ee 103 15d ca fd 10f 17 17 54
FIXUPS: 281b 17 ffffe8b5 73 21 25 1b 3d 8d 7a 58 be 66 51 2e 468 13 3b6f1
FIXUPS: 3d075 58 fffc8c76 1b 1b 48 32 22 22 21 45 c 48 161 b7 cc 2b 3f
FIXUPS: 624b 87 c 4c 2b 85 a3 9f 36 9c 3d 19 1a9 ffffb560 5d 60 2fdd 70
FIXUPS: 4f01 8 5a 3a c 9a de 20 33 2d 1c a 6 84 77 b1 23 7b 184 e1 46a
FIXUPS: 5b1b 6c c 6d 48 25 1a 62 54 ffffe6a6 17 25 4d c4 a 18 7 a 42 b
FIXUPS: 45dd 1c d f 5d f2 59 2c 14 86 40 5b 8c 115 9a 20 e0 ab 1a 8e 18
FIXUPS: 3998 b8 19 a 2a 41 b 1e f 64 20 32 a 299 f 102 a 18 7 35 41 b 19
FIXUPS: 405f d f 5d f4 58 2c 14 97 ffffee08 7 5 5 5 5 5 5 5 10 20 21 2e
FIXUPS: 323a 9 a e b8 48 68 2c 14 55 5d 24d 13 15 13 15 5c 82 15a 3715
FIXUPS: 725a 5f f2 3d 1f 1f c 1f ffffb577 2b8 17 15d dd 25 d0 5 5 18 5
FIXUPS: 301c 14 5 12 5 16 1e 5 1e 16 33 7 45d6 24 f 20 32 5f f d d d d
FIXUPS: 77fd d d d d d d d d d fffff074 5e 168 213 26 82 26 5f c 6f c 443b
FIXUPS: b2db 4e 31 2d 35 41 13 13 4a 16 2d ffffbfba 18 c 12 9 2f e 32 e
FIXUPS: 7550 c c c b 3e 80 1c 24 f 21 34e9 c c 94 7b 47 10 13 23 3f 6 a
FIXUPS: ae34 19 71 25 2b 45 4e 18 2a 11 5c 26 38 6 59 29 48 29 c7 f fffff2cf
FIXUPS: a566 26 32 96 49 2c 48 98 1c 52 2c 3a f 27 9 6 8 20 13 31 29 2d
FIXUPS: a99f 38 c 1a 8f 32 23 19 44 fffff16b d 1dc 33 20 d 3b 31 54 79
FIXUPS: a06d f 3f e 6 68 15 c 2b 24 a d7 a7 2f a 7b 3f 29 38 1a 62 18 fffff24e
FIXUPS: 9772 13 63 2d f 3e 3d 14 d 13 62 33 f 26 d 5b f 78 2e 4a 14 d 1e
FIXUPS: 9b52 6c 2e 4a 14 d 1d f fffff43b f d6 5e 1f 67 13 55 27 a a0 a
FIXUPS: 93e4 26 3b a 1a 21 30 a 4e 26 55 12 1e 6e f f 7d f 3e 3e fffff31f
FIXUPS: 8a8f 55 1f a 2a 1a 2a cb 3b 3a 18 18 18 18 d7 11 14 20 a 13 52
FIXUPS: 8eb5 20 f 36 a9 f 20 f 8e f fffff29e 5 9 50 74 4b d 18 1a 6f 76
FIXUPS: 8592 a 4d 1f 15 2b f 18 c c 1f 18 a 35 146 c 85 fd 2a 1a 2a fffff5fd
FIXUPS: 806e 34 18 49 1f 46 3c 1f 43 3d 26 1c a 22 19 5 5 15 5 5 5 5 5
FIXUPS: 8307 e 5 5 5 5 5 5 fffff62f 2d 2b 4a 16 16 13 58 1f e e e 17 c
FIXUPS: 7b2c 6c 22 f f 5a 50 48 20 35 61 2b a f3 8b 2b 5d 8 38c6 54 37
FIXUPS: b96d 37 126 1f 23 28 98 145 e6 fd 18 22 129 2d da 26 11 1e 11 5a
FIXUPS: c281 6c 3b 32 25 1f 11e 39 ffffb3d6 6386 3b 22 27 27 3b 22 27 27
FIXUPS: dde2 22 27 27 3b 22 27 27 41 ffffd5e0 18 27 a 33 2a 64 6c 5d 81
FIXUPS: b7b1 6c 15 2d 1e05 27 27 3b 22 27 27 41 1c 3d 1f 3a d5 27 27 2d
FIXUPS: d9ba 18 30 27 27 3b 22 27 27 3b 22 27 27 3b 22 27 fffff44c 3a d5
FIXUPS: d1ac 27 2d 1a 18 30 27 27 3b 22 27 27 3b 22 27 27 3b 22 27 27 3b
FIXUPS: d50e 27 27 3b 22 27 27 3b ffffefa8 3b 1f ce 2a 2a 64 2b 4e 111
FIXUPS: c96b 17 48 c7 68 8 b 18 a4 a 4f f7 69 87 69 1c 7b 24 53 1c 7f 3d
FIXUPS: f1de 21 f c6 95 11c 28 29 16 84 48 4a 1b c0 a7 16 8a 23 3d 5d 6e
FIXUPS: f98d 37 61 10 38 39 f ffffcab1 b a 56 2207 2d 10 e e e e e e e
FIXUPS: e885 59 3a 89 47 b7 f 5e 3a 24 52 74 6c 63 47 31 49 3f 18 47 30b
FIXUPS: f19f ffffeea0 5b b5 1a 84 19 3e 54 23 a8 17 17 17 152 12 1a d 20
FIXUPS: e5a6 3d 21 1f 3e 27 25 1f 5c 20 14 1d 1d 36 2b99 c 18 11 17b 42
FIXUPS: 1156c 21 d 11 187 43 12 16 13 1e 15 d 11 24 132 13 11a e 1b 9 2b
FIXUPS: 11afe 12b c 16 ffffc33c 2f59 43 2a 2b 32 1b 29 1b 14 f 13 31 35
FIXUPS: 110e2 3b 3c 1b c 1b 40 1b 34 13 1b 34 13 2d 19 12 2d 18 11 fffff646
FIXUPS: 109ad 1b 16 30 1b 16 2b 1b 30 1b 2b 1b c 38 36 1a 15 13 1b 3d 1a
FIXUPS: 10c59 1a 1c 42 42 4b 2f 3a 38 9f fffff7e0 1b c 1b c 1b 19 c 1b
FIXUPS: 10740 c 1b 18 1b 28 1b 8 11 13 f 13 1b 16 24 1b 16 24 1b 16 1c
FIXUPS: 1093d 32 fffffa74 1b 2e 18 18 1b c 1b c 1b c 1b c 1b c 1b c 1b
FIXUPS: 1056d 1b c 1b c 1b c 1b c 1b c 1b c 1b fffff930 13 13 49 dd 1c
FIXUPS: 1011d 13 1b 13 13 1b 13 13 1b 19 1b 19 1b 19 1b 13 13 1b 4f 13
FIXUPS: 1031d 13 1f 1b 40 1a 1e80 24 12 93 74 ffffd803 26 26 16 1f 7c 13
FIXUPS: fd0a 1c 81 1d 1a 1b 11 1a 1b 11 1a 1b 11 1a 1b 11 1a 1b 19 3c 1f17
FIXUPS: 11e93 d 1a d 35 8 24 13 23 20 f 19 22 1a 2e 13 2c 1c 2c 1a 2e 7e
FIXUPS: 12177 9 24 12 23 9 24 12 23 e5a b0 57 31 57 b3 57 1f 1d a4 34 c3
FIXUPS: 11c78 8 41 2b 2a 16 10 11 42 18 2f d c 1a 9 c 21 d 14 14 d3b 14
FIXUPS: 12bd7 f 5c 14 14 14 f 54 2f 10 e e e e e e e e 7f 4d 39 1f e 4d
FIXUPS: 12f6b 1f e 57 79 1f 1aef ffffd840 81 62 2a 9d 3c 4a 2d 34 3f c
FIXUPS: 126d9 50 17 200 20 1e 21 5f 16 11 18 10 15 12 10 10 12 6b 11 79
FIXUPS: 147f4 12 12 12 12 12 12 12 12 12 12 19 14 a 10 42 c f 12 12 12
FIXUPS: 14994 12 12 d 3d f 2b 97 24 58 1b fffffa22 12 12 12 12 12 12 28
FIXUPS: 14632 12 12 12 12 12 12 24 12 12 12 12 12 12 12 12 12 12 12 12
FIXUPS: 147ac 12 12 12 fffffb3f a d d 2b 19 12 12 12 12 12 12 12 12 12
FIXUPS: 1443d 12 12 12 12 12 12 12 12 12 12 31 9 19 12 12 12 fffff9c2 f
FIXUPS: 13f72 f 27 f 27 f 27 f 27 f 19 10 42 2e 34 19 12 12 12 12 12 12
FIXUPS: 141bd 12 43 7a 16 30 10 37 fffff9a5 12 12 12 12 12 12 12 12 12
FIXUPS: 13d72 12 12 12 12 12 12 12 12 12 12 12 12 12 12 12 12 12 12 12
FIXUPS: 13f06 f fffffb73 31 a 14 1a a f d a d 17 8 5 5 f 5 c 5 a d d 34
FIXUPS: 13be6 12 24 12 12 12 12 12 12 12 fffff9a5 5e 35 14 9c 16 3a 16
FIXUPS: 13822 1b 35 1b 2b 3a 2d 11 d e 10 13 28 14 14 14 14 1e 12 12 12
FIXUPS: 13a4c d 5 12db 2b 10 12 18 14 127 14 11 11 11 1bd d 92 6a 40 5a
FIXUPS: 1529b 1b a9 1b 1b 23 ffffe190 c 9 13 c 7 10 82 1b 595f c 16 73
FIXUPS: 19056 f 96 1ad 124 122 2f 14a 20 20 18 dc 20 4d 4d 6f 89 31 1f
FIXUPS: 199bc 81 4f 69 48 ffffb079 81 85 2c 36c7 27 35 25 21 53 63 6f d1
FIXUPS: 186c0 71 50 2e 1a4 53 51 16 16 1e 2d c c 13 12 246 102 30 91 5c
FIXUPS: 18f42 c 2a ffffed2f 2c 5a 14 14 10 10 10 37 44 11 87 57 17 25 2e
FIXUPS: 1802a 20 2d 1f 17 20 20 17 21 16 ef 82 16 76 18 3d ffffebbd 16
FIXUPS: 16fce 8c 2f 161 41 38 7e 3f 3a d8 15 dc 20 4d 4d 6f df 25 4e 97
FIXUPS: 178c8 98 c9 57 45 98 19 58 30 76 ffffe9d6 79 20 21 2a 60 11 1b
FIXUPS: 167f4 11 35 3b 22 8d ab 16 16 1e 2d c c 13 12 21f 102 30 91 5b
FIXUPS: 16ef2 c 29 17 fffff156 1f 15 27 27 24 24 28 16 28 17 25 10 9d 2d
FIXUPS: 162f4 60 1a 1c 1a 1c 17 2e 1e 23 3a c 24 c 24 c 13e fffff5de 22
FIXUPS: 15c40 59 9 35 9 8a 32 c 26 1e c 26 1e c 26 23 21 1e 10 15 1f c
FIXUPS: 15f46 23 23 2a 21 1a 70 1f fffff603 11 7f 4b 18 18 18 29 1a 2a
FIXUPS: 15830 11 25 1d 34 18 1d 11 25 1d 18 10 62 17 1b 16 1b 5f b8 30
FIXUPS: 15bb5 33 486c 43 42 66 42 38 9a 1c 25 8 d ffffad40 68 26 41 26
FIXUPS: 154f9 14 1e 14 1c 14 15 1a 15 1a 15 1a 15 1a 15 1a 5a81 10 10 8f
FIXUPS: 1b202 d3 25 31 4f 42 6b 45 50 ffffe830 12c a9 1e2 98 3b 27 3a 5f
FIXUPS: 1a273 37 13 42 4f 1f 1f 1e 22 23 2112 49 36 9 6 ffffe2a5 4a 8e
FIXUPS: 1a959 93 76 6e 62 29 81 21 94 1c 35 18 9e 70 37 45 39 82 b1 12
FIXUPS: 1b028 1f 28 14 d34 2a 20 3a 39 20 71 32 2c 3f 3a 127 1c 3a b8 4c
FIXUPS: 1c2ad a 25 61 14 35 14 25 13 2a 14 25 13 6d 14 25 fffff1cf f 35
FIXUPS: 1b728 2d 1f f 35 2c 25 24 25 9c 2b 34 2b 39 2b 34 2b 34 30 31 7f
FIXUPS: 1bb71 4c 7c 27 52 27 77 36 f8f 10 c 11 10 10 14 1c 18 14 1c 26
FIXUPS: 1ce26 30 17 25 35 2f 46 f 3e 26f 8 5 2d 16 11 ffffe38d 46 f 35
FIXUPS: 1b6af 133b 9 f 9 19 33 9 1e 9 1e 9 1e 9 1e 9 1e 9 99 9 38 9 22
FIXUPS: 1cc31 21 9 21 9 21 9 21 9 33 fffffa9a 26 23 12 9 16 c 13 e e 16
FIXUPS: 1c885 a e 16 15 a 9 a e 16 c 13 c 10 c 10 c 10 21 1f 9 f5a 40 4a
FIXUPS: 1d9be f ffffebdf 14 9 16 9 16 9 16 9 16 9 16 9 16 9 16 1b 28 9
FIXUPS: 1c6f4 9 f 9 f 2b 9 42 1a59 d d 65 14c 60 ffffee83 8 f 8 80 c a4
FIXUPS: 1d413 23 19 23 13 14 20 2b 1c 46 32 16 14 95 6f 81 53 19 4e 152b
FIXUPS: 1ed3a 105 7 f 20 3c 24 115 87 20 26 b8 61 6c 3a 3d0 72 1e4 20 21
FIXUPS: 1f915 10f ffffe6ea d d d 7d d d d d 595 a 5 5 1c 17 17 35 11 e
FIXUPS: 1e832 5 a 11 21 23 8 3c 9 1d 1f 1b 12d 5f 29 121 f 27 8 6e 8 40
FIXUPS: 2360c 20 182 173 65 4e 11 2a 28 15 28 15 19 16 18 16 ffffa990 8
FIXUPS: 1e491 e d d c 9 30 7b 31 49 53 3d 53 95 46c6 ad 2d 2d 15f 2c 28
FIXUPS: 23117 4b 2a 26 2a 4f 64 5f 20 27 12 14 24 27 b0 40 e 11 2a 28 15
FIXUPS: 23547 18 34 22 ffffea77 64 31 13 c7 5b 1f 43 227 87 1a aa 30 50
FIXUPS: 22683 60 25 19 34 a 91 110 5b 9 a2 5c 71 37 2e b1 1cd 51 ffffe8e0
FIXUPS: 2170c 19 58 75 3e 3b 1a 1a 28 b5 49 16 68 24 45 49 d1 4d 47 18
FIXUPS: 21cbc 1f 1f 2d f 77 c8 5f e 22 22 fffff159 e 3d e 3d 32 3f 3c 4a
FIXUPS: 21224 15 1e 3c 4e 2d 97 31 31 20 25 23 23 32 23 23 81 41 1f 27
FIXUPS: 2162b 35 6b fffff13e 17 31 13 12 13 33 66 1a 2d 6e 1c 15 24 cb
FIXUPS: 20b88 38 14 1a a0 14 33 2f 2d 66 22 2f cb 91 33 1a 1a fffff40f
FIXUPS: 203f0 13 16 13 12 12 12 12 35 77 13 39 13 13 13 1d 35 22 13 77
FIXUPS: 206b6 17 4f 13 17 31 13 17 31 13 12 fffff606 8 36 a0 7a 25 7c 4f
FIXUPS: 20076 1f 5c 5d 19 f 1d 50 15 58 19 10 11 c 2b 10 11 c 19 10 11
FIXUPS: 20334 1c 54 463f 3b 46 2fd 1a 36 1b8 9b 75 2cd 53 376 17 22 17
FIXUPS: 25782 17 186 29 37 c ffffa0fe 30 10 14 30 36 108 1a a 78 36 4016
FIXUPS: 23d44 11 2e 11 11 11 136 c 93 1d 63 34 36 17 17 19 1a 1a a5 46
FIXUPS: 241f5 a2 76 1d 143 29d 16 216 1b 1c 36 1ef9 55 46 16 ff 135 16
FIXUPS: 26ba5 ff 14 38 16 3b 16 e 12 11 13 12 11 13 12 11 15 12 27 f e
FIXUPS: 26e76 15 ffffccb3 30 1f23 47 1d 33b 6c 232 13 1b 2b bc 26 f 1c
FIXUPS: 26263 38 13 25 40 13 161 15 17 154 3a 50 3d 1a 1a 127 1d 22 1d
